:020000040800F2
:104000000050002031EF000869C400086BC40008AC
:104010006DC400086FC4000871C4000800000000EF
:1040200000000000000000000000000075C400084F
:1040300073C400080000000077C4000885920008DF
:1040400079C400087BC400087DC400087FC4000850
:1040500081C4000883C4000885C4000887C4000820
:1040600089C400088BC400088DC40008000000004B
:104070000000000000000000000000000000000040
:1040800000000000000000009DC400089FC400085C
:10409000ADC40008BDC40008CDC40008DDC40008DC
:1040A000DFC40008E1C40008E3C40008E5C4000858
:1040B000E7C40008E9C40008EBC40008EDC4000828
:1040C000EFC40008F1C40008F3C40008F5C40008F8
:1040D000F7C40008F9C40008098B0008FDC40008F3
:1040E000FFC4000801C5000803C500080000000067
:1040F00000000000000000000000000000000000C0
:0C41000000000000000000005FF800005C
:1041100030BF704720BF704740BF7047BFF36F8FFD
:104120007047BFF34F8F7047BFF35F8F704701DF5A
:104130007047EFF31480704780F31488BFF36F8FDC
:104140007047EFF30980704780F309887047EFF3F9
:104150000880704780F30888704772B6704762B66F
:10416000704771B6704761B6704780F31188704729
:10417000EFF31280704740BA704700BA70470000F2
:104180000C4B10B59B680C4813F400440B490C4AC7
:104190000C4B07D0012404700B4808600B491860D1
:1041A000116010BD04700A4808600A4911600A4A8B
:1041B0001A6010BD00080140EC10002050110020D2
:1041C00008130020C8110020719200084B970008C6
:1041D000E58D0008858C0008358D00082DE9F74F26
:1041E000624F6348012109F0ABFA04200121032446
:1041F00009F08EFD102642F20263384601A94FF005
:104200000408ADF804308DF806408DF8076009F019
:1042100008FA40F202637B610DEB08014CF20803DF
:104220003846ADF8043001254FF04809DFF850A1B9
:104230008DF807808DF8064009F0F3F90DEB0801C1
:1042400038468DF80790ADF804508DF8064009F017
:10425000E8F90820294609F05BFD41F6FD4B504680
:104260000DEB0801ADF804B08DF806408DF807603D
:1042700009F0D7F9CAF810B03046294609F048FDD0
:104280004FF0FF0A0DEB08013A488DF807804FF414
:104290007F4BADF804A08DF8064009F0C2F90DEB94
:1042A00008018DF807903348DFF8D890ADF804B0D6
:1042B0008DF8064009F0B5F92020294609F028FDBF
:1042C0004FF6FF7348460DEB0801ADF804308DF84A
:1042D00006408DF8076009F0A4F9C9F810B0402035
:1042E000C9F814A0294609F013FD8DF80780DFF8FE
:1042F000988040F2FF33404601A9ADF804304FF4F6
:104300007C498DF8064009F08CF9404601A9ADF8CA
:1043100004908DF806408DF8076009F082F929466F
:10432000C8F81490144809F00BFA00230A211A4621
:104330004FF400507861BC683861B868640458BFB5
:104340000132400448BF01330139F1D10A2A0B4A36
:1043500003D10A2B01D1012300E0002304480121ED
:10436000137009F0EDF903B0BDE8F08F00080140CB
:1043700000023000001001400004300070110020E5
:10438000000C01400014014000180140124B82B0A3
:104390001B78F3B1114B4FF400625A614FF4806205
:1043A0001A610022019201990D4A914202D8019AA4
:1043B0000132F7E74FF400621A614FF480625A61EC
:1043C00000230193019A064B9A42E3D8019B0133E3
:1043D000F7E702B0704700BF70110020000C0140E9
:1043E0003F0D0300072816D8DFE800F00406080A8E
:1043F0000C0E101201220CE002220AE0042208E056
:10440000082206E0102204E0202202E0402200E020
:104410008022014B5A61704700140140072816D8CA
:10442000DFE800F00406080A0C0E101201220CE06E
:1044300002220AE0042208E0082206E0102204E03A
:10444000202202E0402200E08022014B1A617047E6
:104450000014014038B50546002445FA04F3DB0793
:10446000E0B202D5FFF7DAFF01E0FFF7BBFF01344E
:10447000082CF2D138BD08B507282ED8DFE800F0A7
:1044800004060B10151E232800200FE0144B98681B
:10449000C0F3400008BD124B9868C0F3800008BD0F
:1044A0000F4B9868C0F3C00008BD042004F0D2FF91
:1044B000B0F5006F94BF0020012008BD084B98683C
:1044C000C0F3401008BD064B9868C0F3801008BDCB
:1044D000034B9868C0F3C01008BD002008BD00BFA2
:1044E0000010014007282DD8DFE800F004090E1362
:1044F000181D2227144BD86800F001007047124B9A
:10450000D868C0F3400070470F4BD868C0F38000F4
:1045100070470D4BD868C0F3C00070470A4BD8688D
:10452000C0F300107047084BD868C0F340107047C4
:10453000054BD868C0F380107047034BD868C0F3B0
:10454000C0107047002070470014014038B50024A7
:104550002546E0B2FFF78FFF18B10123A3401D43AA
:10456000EDB20134082CF4D1284638BD052822D8F4
:10457000DFE800F003080D12171C104B986800F0DC
:10458000010070470D4B9868C0F3400070470B4B1B
:104590009868C0F380007047084B9868C0F3C0006B
:1045A0007047064B9868C0F300107047034B98683B
:1045B000C0F3401070470020704700BF0018014052
:1045C000052802D8C90805F0EDBD704708B109F00B
:1045D000DDB909F0E3B962B6704772B67047C0B290
:1045E00005F00EBFC0B205F0FBBE084B10F0010F86
:1045F0004FF0100214BF1A615A6110F0020F4FF011
:10460000200214BF1A615A61704700BF000C0140BC
:10461000074B9A88C2F30722172A06D19A88D2B28A
:10462000DE2A02D1188980B270470020704700BF8F
:10463000006C0040154B9A6812F4807F9A680CBF9A
:104640008020002091059A685CBF40F04000C0B215
:1046500052059A6858BF40F0200011059A6858BF6B
:1046600040F01000D2049A6858BF40F0080091044E
:104670009A689B6858BF40F00400520458BF40F04D
:1046800002001B0458BF40F00100704700100140B9
:1046900008B5082004F0DEFE5E2804D9064B1A781F
:1046A0004AB9012206E0082004F0D4FE542802D8BA
:1046B000014B00221A7008BD60050020034B1878DA
:1046C000013801288CBF00200120704760050020C0
:1046D000034B1878012806BF02221A700020704789
:1046E00060050020002070472DE9F04F4FF4804016
:1046F00089B0012109F018FB434C0120014609F063
:1047000007FB03264FF420434FF0180A204602A966
:10471000ADF808308DF80BA04FF0040B8DF80A604F
:1047200008F07FFF4FF48043204602A9ADF808301F
:104730008DF80A608DF80BB008F073FF0823ADF810
:104740001830324B002401254FF482794FF00208D3
:104750004FF40077184603A9ADF80C40ADF81040AF
:10476000ADF81A40ADF81C400193ADF80E90ADF8CD
:104770001280ADF81450ADF8167009F081FB019B62
:104780002946184609F002FC29464FF4805009F0EA
:10479000BFFA2846214608F0D3FF8DF80BA0DFF8BA
:1047A00074A0A023504602A9ADF808308DF80A6025
:1047B00008F037FF4023504602A9ADF808308DF8C5
:1047C0000A608DF80BB008F02CFFADF80C40ADF886
:1047D0001040ADF81A40ADF81C400D4C282320467F
:1047E00003A9ADF81830ADF80E90ADF81280ADF811
:1047F0001450ADF8167009F043FB2046294609F025
:10480000C5FB09B0BDE8F08F000C01400038004046
:10481000003001400008014070B504460E461546C0
:1048200008287BD8DFE800F005101316191C1F0AB2
:104830000D003C4B4FF480525A6119E04FF4007266
:1048400013E04FF4807210E04FF480620DE04FF4FB
:1048500000620AE04FF4805207E04FF4005204E097
:104860004FF4804201E04FF400422F4B5A6110E0B8
:104870002E48022109F00EFC0028F9D02B483146C1
:1048800009F0B4FB2948012109F004FC0028F9D003
:1048900019E02748022109F0FDFB0028F9D024483F
:1048A000314609F0A3FB2248012109F0F3FB00285F
:1048B000F9D045B3082C31D8DFE804F006111417FD
:1048C0001A1D200B0E0015B3164B4FF480521A61BF
:1048D0001DE04FF4007213E04FF4807210E04FF4CB
:1048E00080620DE04FF400620AE04FF4805207E06E
:1048F0004FF4005204E04FF4804201E04FF40042D4
:10490000094B1A6105E014B1082C09D801E00748E9
:1049100000E0074809F06CFBC0B270BD002070BD1C
:10492000284670BD000C01400014014000380040D2
:104930000030014037B5B54DA8786B7805282C4676
:1049400001D904225AE3A22B00F0AE8200F2848047
:10495000842B00F01F8128D8062B00F0808110D80E
:10496000022B00F0178106D8002B00F0F080012BFD
:1049700000F0FB8041E3042B00F04C8140F23481D5
:1049800062E1802B00F0E38009D80C2B00F08381DA
:104990000D2B00F09A81072B40F02F836DE1822BC5
:1049A00000F0AD8140F2E18034E1932B00F08D8185
:1049B00026D8872B00F0B48106D8852B00F014810F
:1049C000862B00F0418118E38C2B00F0B4818D2BF5
:1049D00000F0BC818A2B40F0108302288ABFC11EE0
:1049E0004101490194BF0023012341F014011846FD
:1049F000C9B201AA06F0ACFFEB788DF80630CBE126
:104A0000992B00F0E08108D8952B00F0AA81C0F026
:104A10004281962B00F0D081EFE2A02B00F038828B
:104A200000F23C829A2B40F0E88202288ABFC11E25
:104A30004101490194BF0023012341F018011846A8
:104A400001AAC9B206F084FF9DF80530EA7803F0A8
:104A50000F0343EA0213CDE1B12B00F0A7822ED859
:104A6000A92B00F0788210D8A52B00F0498206D837
:104A7000A32B00F01F82A42B00F02282BDE2A72B03
:104A800000F05D8240F24C825FE2AD2B00F07C8250
:104A90000AD8AB2B00F0658200F26982D5F80310CA
:104AA000C9B205F023FBABE2AF2B00F0738200F23A
:104AB0007782D5F8031049B205F06AFBA0E2C22B59
:104AC00000F0BA811FD8B72B00F089820DD8B52B22
:104AD00000F0728200F27782B22B40F08E82D5F81D
:104AE0000310C9B205F0A2FB8AE2C02B00F0C5801A
:104AF00000F29C81B82B40F08082D5F80310C9B237
:104B000005F040FA7CE2CC2B00F0AD810FD8C72B2A
:104B100000F0A580C82B00F09581C32B40F06D827A
:104B20003B4B03EB4010D5F80330436068E2D52BD4
:104B300000F0A081D62B00F0A481D42B40F05D8240
:104B4000334B03EB4010D5F80330436158E205F0D6
:104B5000CBFC40B9A178022988BF033994BF00205B
:104B60000120490110E0062248E205F0BDFC0028C2
:104B7000F9D1A178022988BF03394FEA411194BFC6
:104B80000020012041F00201C9B2D4F8032006F050
:104B900042FE35E205F0A8FC0028E4D1A178D4F863
:104BA0000320022988BF03394FEA411141F008016F
:104BB00094BF00200120C9B206F01BFEA178D4F8F2
:104BC0000320022988BF03394FEA411141F0060151
:104BD00094BF00200120C9B2002AB8BF524206F09B
:104BE00008FEA37801212CE005F07EFC0028BAD154
:104BF000A178022988BF03394FEA411141F00A0127
:104C000094BF00200120C9B285E000BF980A0020AF
:104C1000CC11002002288ABFC11E4101490194BF66
:104C20000023012341F00601C9B21846D4F803203D
:104C300006F0DFFDD4F80310A378A94A42F8231048
:104C40000021A84AD154DBE1D4F8031006F007FF95
:104C5000A378D4F80310A44A42F82310E1E0A34B50
:104C600001221A54A24BE17803EB40135972A14B75
:104C70001B5C022B40F0C481BCE19C4B01221A5406
:104C80009B4BE17803EB401399729A4B1B5C002B12
:104C900040F0B681AEE102288ABFC11E4101490140
:104CA00094BF0023012341F01401184601AAC9B2A0
:104CB00006F04EFED4F803209DF8053012B143F003
:104CC000020367E023F0020364E002288ABFC11EEA
:104CD0004101490194BF0023012341F0140118460A
:104CE00001AAC9B206F034FED4F803209DF80530BD
:104CF00012B143F001034DE023F001034AE0022822
:104D00008ABFC11E4101490194BF0023012341F024
:104D10000401C9B21846D4F8032006F06AFD6FE119
:104D200002288ABFC11E4101490194BF002301230B
:104D300041F00E01EDE76E4BE97803EB4013D972B9
:104D4000C1F10801C9B205F0C9F859E102288ABFCA
:104D5000C11E4101490194BF0023012341F01A0102
:104D6000D7E702288ABFC11E4101490194BF002331
:104D7000012341F01401184601AAC9B206F0E8FD6A
:104D8000D5F803209DF8053012B143F0040301E08B
:104D900023F004038DF80530A17801AA022988BF09
:104DA00003394FEA411141F0140194BF0020012062
:104DB000C9B206F0F9FC23E1D5F803204E4B02B14D
:104DC00001221A541CE102288ABFC11E4101490177
:104DD00094BF0023012341F01801184601AAC9B26B
:104DE00006F0B6FDEA789DF8053002F00F0223F0D8
:104DF0000F031343A1788DF80530022994BF0020DA
:104E0000012000D90339490141F01801C9B201AAB2
:104E100006F0CAFC344BA07853F8201006F01FFEB1
:104E2000A378304A134400229A71E9E0304B03EB37
:104E30004010EB780372E3E0D5F803202C4B4001DF
:104E40001A50DDE0294B01221A54294BD5F80320D2
:104E500003EB4013DA77274B1B5C032B40F0D08029
:104E6000264BD978C6E0224B03EB4010D5F803302F
:104E7000C381C5E01E4B03EB4010D5F803308377A8
:104E8000BEE01B4B03EB4010D5F803308383B7E043
:104E9000D5F80310C9B205F031F8B1E0D5F8031028
:104EA000C9B205F039F8ABE0D5F80310C9B205F086
:104EB00055F8A5E0D5F80310C9B205F059F89FE000
:104EC00005F0B8F8D5F8031020B9A878C9B205F0F4
:104ED00063F895E0A878C9B205F086F890E000BFC5
:104EE000D410002064050020BC0C0020F812002023
:104EF000CC1100200013002018130020980A002075
:104F000005F098F8AB78D5F8031020B91846C9B267
:104F100005F04CF874E01846C9B205F079F86FE076
:104F200005F088F8D5F8031020B9A878C9B205F0C3
:104F300047F865E0A878C9B205F060F860E0D5F8F8
:104F40000310C9B205F046F85AE0D5F80310C9B20B
:104F500005F0B8F854E0D5F80310C9B205F0BCF874
:104F60004EE0D5F80310C9B205F0CAF848E0D5F80C
:104F70000310C9B205F0CEF8AA78224B03EBC203A6
:104F8000D5F803205A713BE0D5F80310C9B205F0FB
:104F9000F5F835E0D5F80310C9B205F029F92FE08E
:104FA000D5F80310C9B205F02DF929E0D5F80310A2
:104FB000C9B205F031F923E0134B03EB4010D5F8EB
:104FC000033083611CE0D5F803200E4B43F83020FA
:104FD000B2B903EBC003597905F09CF810E0094B16
:104FE000D5F8032003EBC0031A71084B1B5C012B9F
:104FF00006D1E978FFF7E4FA02E00322044B1A70C5
:1050000003B030BD10110020CC110020001300208F
:10501000B00C002037B57F4D7F4CA8786B78052801
:1050200002D904232370DAE2D62B00F2C682DFE82D
:1050300013F0D700E200F50000010B010D010F0194
:1050400014011901520173015A012A013E01C402DF
:10505000C402C402C402C402C402C402C402C40220
:10506000C402C402C402C402C402C402C402C40210
:10507000C402C402C402C402C402C402C402C40200
:10508000C402C402C402C402C402C402C402C402F0
:10509000C402C402C402C402C402C402C402C402E0
:1050A000C402C402C402C402C402C402C402C402D0
:1050B000C402C402C402C402C402C402C402C402C0
:1050C000C402C402C402C402C402C402C402C402B0
:1050D000C402C402C402C402C402C402C402C402A0
:1050E000C402C402C402C402C402C402C402C40290
:1050F000C402C402C402C402C402C402C402C40280
:10510000C402C402C402C402C402C402C402C4026F
:10511000C402C402C402C402C402C402C402C4025F
:10512000C402C402C402C402C402C402C402C4024F
:10513000C402D700E20084010B01F50000010D015B
:105140008F01C402C4029A01C402AC01B101C402BD
:10515000C402C402C402C4023E012A01C001D40137
:10516000C402C402D601EA015A0173011901C40242
:10517000C402420245025F026202650271027C02C1
:1051800087028A028D029002930296029B029E027F
:10519000A102A402A702AA02AD02B002B302B802A1
:1051A000BC02C102C402C402C402C402C402C402DA
:1051B000C4021401FD01020206020B020D02C40228
:1051C0000F010F02C402C402C4021402C402190275
:1051D0001D023102C402C402C402330238023D027D
:1051E000022894BF0023012302D84001C1B20DE080
:1051F000C11E490109E002288ABFC11E41014901BF
:1052000094BF0023012341F00201C9B2184606F001
:1052100011FE79E1980A0020B00C002002288ABF14
:10522000C11E4101490194BF0023012341F008013F
:10523000BAE002288ABFC11E4101490194BF002380
:10524000012341F00A01AFE09E4B0CE19E4B0AE1C5
:105250009E4B03EB4010437A5CE09C4B03EB401009
:10526000837A57E0022894BF0020012006F063FBF8
:10527000AB780122022B92BF9340033B5B0002FA02
:1052800003F3034243E002288ABFC11E41014901E2
:1052900094BF0023012341F014011846C9B201AAAA
:1052A00006F056FB9DF80530C3F3400332E00228B8
:1052B0008ABFC11E4101490194BF0023012341F06F
:1052C00014011846C9B201AA06F042FB9DF8053048
:1052D00003F001031EE0022894BF01300230C0B287
:1052E000FFF7C9F810E1022894BF002001207C21BB
:1052F00001AA06F02DFBAB789DF80610022B4FF0AB
:10530000020200D9033B5B0002FA03F30B420CBF1D
:1053100000230123636052E1022894BF0020012092
:105320007C2101AA06F014FBAB789DF80610022B35
:105330004FF00102E6D89340E6E702288ABFC11E7B
:105340004101490194BF0023012341F004012BE0F6
:1053500002288ABFC11E4101490194BF00230123D5
:1053600041F00E0120E002288ABFC11E410149011F
:1053700094BF0023012341F014011846C9B201AAC9
:1053800006F0E6FA9DF80630C4E704F0CFFDC0F160
:105390000800B9E002288ABFC11E4101490194BF3B
:1053A0000023012341F01A01C9B2184606F0E7FABA
:1053B000AAE002288ABFC11E4101490194BF00230F
:1053C000012341F014011846C9B201AA06F0C0FA3F
:1053D0009DF80530C3F380039CE73D4BDAE00228DB
:1053E0008ABFC11E4101490194BF0023012341F03E
:1053F00018011846C9B201AA06F0AAFA9DF80530AC
:1054000003F00F0386E702288ABFC11E410149014C
:1054100094BF0023012341F018011846C9B201AA24
:1054200006F096FA9DF805301B0973E7274B03EB4E
:105430004010037A6EE7254B40011B586AE7234B67
:1054400003EB4010436865E7224B0CE0224B0AE077
:105450001E4B03EB4010C37F5CE71C4B03EB40107B
:10546000C38957E71D4B53F8203053E7AB781C4AEC
:105470000021D05C616010B11A4801254560D1540B
:10548000194AD15C19B1616841F0020161600021E3
:10549000D15494E0154B7DE00C4B03EB4010436975
:1054A00038E70A4B03EB4010837F33E7074B03EBEE
:1054B0004010838B2EE704F041FD25E004F046FD0B
:1054C00022E000BFD4100020BC0C0020CC11002032
:1054D00018130020F0100020901200205811002016
:1054E000BC110020B00C002046110020C211002089
:1054F00004F098FD08E004F09DFD05E004F09AFD3D
:1055000020B9A87804F0A6FD606058E0A87804F0FF
:10551000C1FDF9E704F08EFD18B9A87804F0A2FDEA
:10552000F2E7A87804F0C6FDEEE704F083FD18B9B1
:10553000A87804F09FFDE7E7A87804F0B3FDE3E75F
:1055400004F0A0FDE0E704F0EFFDDDE704F0F6FD78
:10555000DAE704F0FBFDD7E704F000FED4E7214BC7
:1055600003EBC0004379D5E604F026FECCE704F057
:105570002DFEC9E704F092FEC6E704F097FEC3E7EC
:1055800004F09CFEC0E704F0A1FEBDE704F0AEFE0F
:10559000BAE7154B1B5CBDE6144B03EB4010836967
:1055A000B8E6104B53F83030B4E60E4B03EBC000B6
:1055B0000379AFE604F046FDA6E7032323700C4B06
:1055C0001B7863B10B4B62681A600B4B1AB91A68EF
:1055D00042F0080202E01A6822F008021A6003B0E2
:1055E00030BD00BF101100200A110020CC11002096
:1055F000AB0C00209C0C0020A00A002038B5AF4A5C
:1056000095781446022D00F05181032D00F0688139
:10561000002D40F0088253784F2B00F0A58037D83A
:10562000462B78D014D8422B63D009D8402B5CD0BD
:10563000412B40F0F681D178A14B002019705CE03D
:10564000442B9F4A5DD062D8E1780420117154E068
:10565000492B73D00AD8472B68D0482B40F0E18102
:10566000D3789749262001F8263FD6E04C2B71D0FD
:105670004D2B74D04B2B40F0D481914CD17803202A
:10568000E17002F0F2FFE078BDE8384003F0D0BAF4
:10569000572B00F0D08012D8522B00F0968005D8FE
:1056A000502B7ED0512B00F08180BAE1542B00F0BA
:1056B000A980C0F09180552B00F0B180B1E1832B1F
:1056C00000F0E78006D8592B00F0BB805A2B00F081
:1056D000C080A6E1852B00F0E580C0F0DE80FF2BC6
:1056E00040F09F81D278774B9FE140F2FF70D178F4
:1056F00003E0D178724B01205970BDE8384002F0C8
:10570000B4BFD4F803301C20D3616F4909E0E178BD
:1057100005205171F1E7D2F8033069490C2041F8B6
:105720000C3F0422BDE8384002F0FEBF644DD2F8C1
:105730000330294641F8083F082054E0D278604BF6
:105740000AB9DA7503E061490122DA754A60172067
:10575000D97DD2E7D1785A4B02209970CDE7D17824
:10576000574B15205975C8E7D2F80310544CC9B2ED
:105770001920617602F079FF607E10F001000EBF03
:1057800001462846012106F091FB637E012003F0CB
:10579000020303F0FF0103B10146BDE8384006F003
:1057A00085BBD178464B16209975A6E7444B1A7DE8
:1057B0001D4612F0010F04D0E378DB0701D402F09C
:1057C000B8FEE1781420297597E7D2F803303C49F8
:1057D000202041F8203FA4E7394DD2F80330294674
:1057E00041F8103F1020042202F09EFF384B1B7836
:1057F000002B40F01B816879A9682A69BDE8384010
:1058000003F050BBD2F80330012B00F20C812B4B7C
:105810002B49DB781A2001F81A3F012282E7D2F8DF
:105820000330012B00F2FF80244B2549DB781B203D
:1058300001F81B3FF1E7D3782149272001F8273FE2
:10584000EBE7D2F803301E49242021F8243F02223E
:1058500068E71B4DD378294601F8283F282001220C
:1058600002F062FF95F8280010F001000EBF01461B
:105870000020012106F02CFB95F82830012003F0D0
:10588000020303F0FF0103B10146BDE8384006F012
:105890001FBBD2F803200F4B5EE0D2F803200E4B63
:1058A0001A6038BDD2F803200A4B5AE051780B4BEE
:1058B000D2F8032043F8212038BD00BF980A002009
:1058C00004000020AA0C002020000020B00C0020C2
:1058D000EC10002064050020AC0C0020D40C00204B
:1058E00053782E2B00F29D80DFE803F018212A9BCD
:1058F0009B9B9B9B9B33383D42474C9B9B9B9B9B1D
:105900009B9B9B9B9B9B9B5153555C5E606264661B
:10591000686A6C73787D82878C919600444BD4F8CA
:1059200003201A6003F0FAFC424B586138BD404B2B
:10593000D4F803205A6003F0F1FC3E4B986138BD67
:105940003B4BD4F803209A6003F0E8FC394BD86154
:1059500038BDD4F80320364BDA6038BDD4F80320C4
:10596000334B1A6138BDD4F80320314B5A6138BD2E
:10597000D4F803202E4B9A6138BDD4F803202C4B69
:10598000DA6138BDD4F80320294B1A6238BD0020F3
:1059900002E0002017E00120D4F80310BDE83840F1
:1059A00006F07FB901200EE00220F5E702200AE0B0
:1059B0000320F1E7032006E00420EDE7042002E0E5
:1059C0000520E9E70520D4F80310BDE8384006F0CB
:1059D000A1B9D4F80320164B5A6238BDD4F803207D
:1059E000134B9A6238BDD4F80320114BDA6238BDEC
:1059F000D4F803200E4B1A6338BDD4F803200C4BA7
:105A00005A6338BDD4F80320094B9A6338BDD4F8E3
:105A10000320074BDA6338BDD4F80320044B1A6423
:105A200038BD032200E00422034B1A7038BD00BFCA
:105A3000A812002064050020B00C00202DE9F843D6
:105A4000054614460F4600295ED000285CD08142EE
:105A50005AD0022A8ABFD11E5101490194BF0026A3
:105A6000012641F00601C9B2304606F0E3F9022CE6
:105A70008ABFE11E6101490141F00C01C9B28146B2
:105A8000304606F0D7F9804628460BF063F8054605
:105A900038460BF05FF8014628460BF067F90746D9
:105AA00048460BF057F839460BF060F90BF070FAE6
:105AB000054640460BF04EF839460BF057F90BF00F
:105AC00067FA002D08BF01251049002814BF804641
:105AD0004FF0010838460BF033FA0D4F30B1204635
:105AE000414605F0BCFF3B1901229A71022C8ABF86
:105AF000E11E6101490141F00601C9B230462A4662
:105B000005F089FE01233B55BDE8F8830000A04164
:105B10006405002038B5114D04462B5C93B1022872
:105B200088BFE11E0E4B94BF6101490141F006019F
:105B300053F8242094BF00200120C9B205F059FE7B
:105B400000232B552544AB793BB1064BE0B253F80B
:105B5000241005F084FF0023AB7138BD64050020DC
:105B6000D4100020BC0C00202DE9FF4704F0BCFC41
:105B700008B1062279E2994CA078052803D9637808
:105B8000022B40F029816378032B00F26D82DFE85D
:105B900013F004006F00F6001F01FFF7BBFFA178B0
:105BA0008F4A002353548F4A022953544FF0010265
:105BB00002FA01F28C4B88BF033918784FEA411181
:105BC00020EA02021A7094BF00200120C9B2D4F862
:105BD00003201E4605F01FFEA1780022022988BF7F
:105BE000033994BF0020012088BFC9B205F0DFFE51
:105BF0007E4FA37807EB43139B7F002B00F0378287
:105C00000025A3789D422FD04FEA451907EB0902E2
:105C100007EB4313927F9B7F9A4225D12846FFF7DB
:105C200079FF0123AB40022D88BFE91E327888BF7F
:105C3000490194BF4FF000084FF0010888BFC9B276
:105C400022EA030398BF5FFA89F14046D4F80320A3
:105C5000337005F0E0FD022D8ABFE91EE9B2C9B23A
:105C60004046002205F0A3FE0135062DC9D1FEE114
:105C7000FFF750FFA1785A4A00235354594A02298A
:105C8000535488BF03394FEA411141F0020194BFD8
:105C900000200120C9B206F0CDF8A17801228A4087
:105CA000514BD4F8035002290544187888BF0339B2
:105CB00020EA02024FEA41111A7094BF002001202D
:105CC000C9B22A46994605F0A6FDA178002202290C
:105CD00088BF033994BF0020012088BFC9B205F0F6
:105CE00066FE434BA2785D60404B03EB4212927F0D
:105CF0009A46002A00F0BB81FD260025A078854247
:105D000037D04FEA45180AEB08020AEB4013927F9E
:105D10009B7F9A422DD1FFF7FDFE022D88BF7101B6
:105D200094BF0027012794BF48F0020141F002010F
:105D3000C9B2384606F07EF80123AB4099F800104E
:105D4000022DD4F8032021EA030388BF7101024425
:105D500094BF5FFA88F1C9B2384689F8003005F07F
:105D60005AFD022D94BFE9B231463846002205F0B3
:105D70001EFE01350136062DF6B2BFD177E110F0D7
:105D8000C00539D1052827D8D4F80330142B23DCDB
:105D9000062202FB0303174A52F82360FFF7BAFEFC
:105DA0000E4B012299780E4B8A405D540D4B02290F
:105DB0005D540D4B88BF033918784FEA411120EA32
:105DC00002021A7094BF00200120C9B232463CE1A1
:105DD00010F0C00F00F0FF80042246E1980A002076
:105DE00046110020BC11002009110020CC11002018
:105DF000B00C0020A40A0020402D40F0AB80D4F865
:105E00000380B8F1140FE7DC002501950295039596
:105E10002B4640FA03F2D10706D504AA2A440135DD
:105E2000032D02F8103C02D00133062BF1D10026DD
:105E3000AE4221DA1DF806703846FFF76BFE022FDE
:105E40008ABFF91E7901490141F0020194BF002087
:105E50000120C9B205F0EEFF062303FB0877854B4E
:105E600001AA53F82730C01A80EAE073A3EBE0736D
:105E700042F826300136DBE7012D35DD022D019E8B
:105E8000029D08D1AE4201DD304628E02846314669
:105E90009DF8002026E0AE42039F0EDDBE4207DDE6
:105EA000304629469DF80120FFF7C8FD30460DE039
:105EB000384631469DF800200EE0BD429DF8002096
:105EC00008DD28463146FFF7B9FD284639469DF8DA
:105ED000022007E038463146FFF7B0FD38469DF80E
:105EE00001202946FFF7AAFD0025A3782B41DA07F8
:105EF0002CD5614B0622D3F80330604902FB0352D4
:105F00005C4B022D53F822204FF000036B545C4988
:105F100094BF002601266B544FF0010101FA05F1F0
:105F2000584B187820EA010119708ABFE91E6901EF
:105F30004901C9B2304605F06EFC022D8ABFE91E48
:105F4000E9B2C9B23046002205F031FD0135062D17
:105F5000CBD18CE0802D40F08A80D4F80330142B14
:105F60003FF73AAF0025A3782B41DB072FD5424BF3
:105F70000622D3F80330284602FB03523D4B53F868
:105F80002270FFF7C7FD3D4A0023AB543C4A022D67
:105F9000AB544FF0010202FA05F23A4B94BF0026CF
:105FA00001261978304621EA02028ABFE91E6901FA
:105FB0004901C9B21A703A4605F02DFC022D8ABF7C
:105FC000E91EE9B2C9B23046002205F0F0FC013505
:105FD000062DC8D14BE0052849D8D4F80330142B3E
:105FE00045DC02288ABFC11E4101490194BF00233C
:105FF000012341F00201C9B2184605F01BFFA37846
:10600000D4F80320062101FB02311A4A52F821502C
:1060100005441846FFF77EFDA178184A0023535423
:10602000174A022953544FF0010202FA01F2154BAC
:1060300088BF033918784FEA411120EA02021A702A
:1060400094BF00200120C9B22A4605F0E4FBA178E4
:106050000022022988BF033994BF0020012088BF95
:10606000C9B205F0A4FC02E00322074B1A7004B089
:10607000BDE8F087A40A0020980A002046110020FD
:10608000BC11002009110020B00C0020F7B5BE4E55
:10609000BE4F327864233B70D6F80330222A7A70E0
:1060A0007B6035463C4601F0408260D80F2A00F004
:1060B00051862AD8072A00F0B28114D8032A00F0AA
:1060C0006F8107D8012A00F0C480022A00F00D81F8
:1060D00001F090BC052A00F09A8100F29C81FFF744
:1060E00043FD01F089BC0B2A00F0798506D8092A06
:1060F00000F01D8440F2B68200F01DBC0D2A00F0B5
:10610000A18540F2898500F0FEBD192A00F065875F
:1061100014D8152A00F0B58607D8132A00F0568641
:10612000142A00F08C8601F065BC172A984A00F00A
:106130003A8700F24587536201F05EBC1E2A00F0E8
:106140005F850DD81B2A00F06A87C0F057871C2A8C
:1061500041F050848E4B002283F8202001F04CBC8B
:10616000202A01F0118141F2C18001F079B9812A20
:1061700001F0678236D8412A01F0518217D8252ACA
:1061800001F00E8207D8232A01F0D681242A01F0DB
:10619000DA8101F02FBC272A01F03082C1F0098298
:1061A000402A41F0278403F04CFC01F025BC452A2D
:1061B00001F03E8208D8432A01F0348201F2358290
:1061C00003F041FC01F018BC472A01F03782C1F00E
:1061D0003282802A41F00E846D4B002283F8202009
:1061E00001F00ABC882A01F0AE821CD8842A01F092
:1061F0005D820DD8822A01F03A82832A41F0FA8327
:10620000634B002183F84C1083F8341101F034BA49
:10621000862A01F05D8201F2DD825D4B002283F867
:10622000202001F0E9BB8C2A01F0318306D88A2AAC
:1062300001F0118341F2F78201F024BBF22A01F050
:106240008D83FF2A01F0CD838D2A41F0D38301F0A5
:1062500042BBB378052B4BD804F046F918B106239E
:10626000237001F0C9BBFD260446AB789C420AD0DE
:10627000484A02EB43139B7F002B2FD002EB4412C2
:10628000927F9A422AD1424B0122E254424A002391
:10629000022CA354414A94BF0027012794BFE1B2C6
:1062A0003146A3543846022205F081FB022C94BFEC
:1062B0006101710141F00601C9B2384640F2FF7236
:1062C00005F097FA022C94BF6101710141F00801B9
:1062D000C9B23846D5F8032005F08BFA01340136EF
:1062E000062CF6B2C1D101F087BBB378052B03D9D8
:1062F0000423237001F080BB04F0F6F80028AED12F
:10630000FD260446AB789C420AD0224A02EB431396
:106310009B7F002B30D002EB4412927F9A422BD10C
:106320001B4B0122E2541C4A0023022CA3541B4A9B
:1063300094BF0027012794BFE1B23146A3543846E9
:10634000022205F034FB022C94BF6101710141F07F
:106350000601C9B2384640F2FF7205F04AFA022C33
:1063600094BF61017101D5F8032041F00801C9B261
:106370003846524205F03DFA01340136062CF6B299
:10638000C0D101F039BB00BF980A0020B00C00203A
:1063900064050020CC110020BC1100204611002013
:1063A000B378052BA4D80024AB789C4209D0CD4A01
:1063B00002EB43139B7F2BB302EB4412927F9A4272
:1063C00020D1C94A0023A354C84AE6B2A354304698
:1063D00005F022F9022C88BFF11E94BF0027012787
:1063E0008CBFC9B231463846022205F0E0FA022CD1
:1063F0008ABFF11E7101490141F00801C9B2384656
:1064000005F082FA0134062CCED101F0F5BAFEF780
:1064100091FA01F0F1BAFEF7FDFD01F0EDBAB378A3
:106420007278052B3FF664AF9A2A2ED8992A80F00D
:10643000B580822A00F098800BD8062A78D003D83D
:10644000042A6FD0052A0BE0072A7FD00C3A012AD4
:1064500013E08C2A00F08E800AD8832A62D0862A24
:1064600040F0FC8018460C2105F0C9FB01F0C4BACD
:106470008D2A00F08D80933A022A00F2EF801846B0
:10648000142105F0BCFB01F0B7BAC72A50D01AD8C6
:10649000C12A00F0978005D8B52A00F08580C02A6F
:1064A00054D0DBE0C22A00F09780C32A40F0D680A7
:1064B0008C49580101EB431144300431042202F0AD
:1064C00033F901F099BAD22A00F09E8013D8C82A75
:1064D00000F08C80CC2A40F0C180824A580111180B
:1064E0000E311044081A023300EB4310022202F06E
:1064F0001BF901F081BAD52A00F09480D62A00F069
:106500009F80D42A40F0AA80764A5801111814318D
:106510001044081A023300EB4310042202F004F97D
:1065200001F06ABA1846062105F069FB01F064BA69
:106530006C4A5901501809300A44801A023300EBA2
:106540004310517A02F091F801F056BA654A5901A8
:1065500050180A300A44801A023300EB4310917A33
:1065600002F083F801F048BA1846042105F047FB11
:1065700001F042BA5B4A580111180B311044081A55
:10658000023300EB4310012202F0CEF801F034BADE
:1065900018461A2105F033FB01F02EBA18461821CF
:1065A00005F02DFB01F028BA580100F118024D4901
:1065B000101A0233114400EB4310042202F0B4F825
:1065C00001F01ABA474A580102EB43124830117AD7
:1065D00002F04BF801F010BA4249981C400101EB5F
:1065E0004311042202F0A0F801F006BA3D4A580116
:1065F00011181F311044081A023300EB4310012216
:1066000002F092F801F0F8B9580100F11002354992
:10661000101A0233114400EB4310042202F084F8F4
:1066200001F0EAB92F4A580111181E311044081A16
:10663000023300EB4310012202F076F801F0DCB9DE
:10664000284A580111181C311044081A023300EB73
:106650004310022202F068F801F0CEB90323237040
:1066600001F0CAB9AB78224E052B6A783FF640AEEE
:10667000952A4FD8932A80F0DC800D2A0DD80C2A59
:1066800080F0D780052A00F0A68001D8042A0CE00B
:10669000062A00F0C080072A5FE0862A00F09B806F
:1066A0002CD8822A00F0CB80832A40F03C8106213E
:1066B000184605F079FAAC78022C8ABFE11E610118
:1066C000490141F00601C9B294BF0020012005F044
:1066D00056F9084B084A43F82400AB780021D154FE
:1066E00001F08AB9CC110020BC1100204611002015
:1066F000980A0020D4100020640500208C2A00F0A5
:10670000A4808D2A40F00F8118461A2105F04CFA1A
:1067100001F072B9C32A00F0D1802ED8B52A00F05A
:10672000AB8014D8993A012A00F2FD80184618214E
:1067300005F03AFAC54BB07853F8201005F08FF900
:10674000C34AB378134400229A7101F055B9C12AA3
:1067500000F0A08000F2A880C02A40F0E480BD4A8A
:106760005C0111190A311444081B023300EB431079
:1067700002F054F8A07201F03FB9CC2A00F0A980D1
:1067800012D8C72A47D0C82A40F0CD80B14A580154
:1067900011181F311044081A023300EB4310012274
:1067A00002F055F801F028B9D52A00F0A080D62AC9
:1067B00000F0AB80D42A40F0B680A64A58011118E8
:1067C00014311044081A023300EB4310042202F083
:1067D0003EF801F011B90C21184605F0E5F9AC7846
:1067E000022C8ABFE11E6101490141F00C0194BFF6
:1067F00000200120C9B205F0C2F8944B944A43F836
:106800002400A87800210244917153F8201005F06B
:1068100026F901F0F1B88F4A5C01111909311444CD
:10682000081B023300EB431001F0F8FF607201F027
:10683000E3B81846142105F0B7F901F0DDB81846A1
:10684000042105F0B1F901F0D7B8824C5A01A11822
:106850000B312244881A023300EB4310012201F06D
:10686000F6FFB07804EB4014E17AC1F10801C9B237
:1068700003F034FB01F0C0B8580100F1180275496B
:10688000101A0233114400EB4310042201F0DFFF21
:1068900001F0B2B858016F4C483004EB431401F0DA
:1068A000BDFF207201F0A8B86A49981C400101EBB5
:1068B0004311042201F0CBFF01F09EB86549580155
:1068C00001EB431144300431042201F0C0FF01F018
:1068D00093B8604A580111180E311044081A023357
:1068E00000EB4310022201F0B2FF01F085B8594AD3
:1068F000580111181E311044081A023300EB4310DE
:10690000012201F0A4FF01F077B8524A5801111892
:106910001C311044081A023300EB4310022201F02C
:1069200096FF01F069B80323237001F065B8FEF704
:1069300065FE01F061B8B278474B022A00F0C280D0
:10694000032A00F0C480002A40F031815B78512B8B
:1069500000F096802CD8472B71D014D8432B69D0E7
:106960000AD8412B61D062D8402B40F01E8140F202
:10697000FF7001F053FFE5E0452B384A5DD000F28F
:106980009680D3690FE14C2B71D008D8492B6BD07E
:1069900057D34B2B40F00981304BDB7803E14F2B71
:1069A00068D06AD84D2B40F000812C4B5B7DFAE01B
:1069B000802B76D013D8552B69D005D8532B274A76
:1069C00061D062D8136AEEE0592B63D05A2B64D0A1
:1069D000572B40F0EA80214B93F82730E3E0842BDB
:1069E00067D009D8822B1A4A5FD060D892F820303D
:1069F0001E1F73427341D6E0F02B5CD00DD8852B5F
:106A000040F0D380124A164913694B4303F54053B3
:106A10003933136123F00043C5E0FE2B4BD0FF2B2D
:106A200040F0C3800F4B1B7848E00C4B44E00B4B0D
:106A30005B78B8E0094B1B79B5E05379B3E0074BBD
:106A400069E0064B93F82630ADE000BFBC0C002097
:106A500064050020CC110020980A002004000020CA
:106A60006D4EC641AA0C00207C4BDB7D26E07B4BA3
:106A70009B7898E0794B5B7E95E0784B9B7D92E02C
:106A8000764B1B7D8FE013698DE0937E8BE0734B1B
:106A9000DB7E88E0714B9B8C85E0704B93F828304F
:106AA00081E06F4B93F820307DE0536A7BE0D36840
:106AB00079E06C4B29E06C4B1B7874E0003318BF15
:106AC000012370E05A78694B53F822306BE05B7811
:106AD0002E2B6AD8DFE803F0181B1E696969696903
:106AE000692124272A2D3069696969696969696999
:106AF00069696933383A3C3E40424446484A4C5002
:106B00005356595C5F626500594B1B684BE0584B0C
:106B10005B6848E0564B9B6845E0554BDB6842E0BC
:106B2000534B1B693FE0524B5B693CE0504B9B6908
:106B300039E04F4BDB6936E04D4B1B6A33E00020F8
:106B400005F021F9606034E0002012E00120F7E751
:106B500001200EE00220F3E702200AE00320EFE725
:106B6000032006E00420EBE7042002E00520E7E72D
:106B7000052005F023F9E5E73D4B5B6A13E03C4B4C
:106B80009B6A10E03A4BDB6A0DE0394B1B6B0AE065
:106B9000374B5B6B07E0364B9B6B04E0344BDB6B96
:106BA00001E0334B1B6C636003E0032300E004232C
:106BB0002370304B1B78002B00F01E872E4B626831
:106BC0001A602E4B2AB91A6842F008021A6000F0C7
:106BD00013BF1A6822F008021A6000F00DBFB378E4
:106BE000022B15D17378372B0ED8204903F5A770E7
:106BF000800001EB8301042201F096FD00F0FCBE51
:106C00007278142A40F225830323237000F0F4BE27
:106C100004233B7000F0F0BEB378022B0ED1184B6A
:106C20005B78372BF0D8114903F5A770800001EB92
:106C30008301042201F00BFE00F0DEBE04233B7052
:106C400000F0DABEB07805283FF652AB6B780C4EF8
:106C5000012B39D016D3022B3AD050E0040000208B
:106C600064050020AC0C0020F0120020D40C0020A1
:106C7000A8120020AB0C00209C0C0020A00A0020D1
:106C8000980A002003F030FC054600287FF4E7AAAC
:106C9000B07804F0B9FCB3782846834209D09B4908
:106CA00001EB4012927F52B101EB4311897F914277
:106CB00005D1974A01218154964A0021815401301F
:106CC0000628EAD100F098BE04F0A6FC00F094BEBD
:106CD00004F0AAFC904B78601B78002B00F08C86A7
:106CE0008E4B18608E4B1A6820B942F008021A6069
:106CF00000F082BE22F008021A6000F07DBE03237D
:106D00003B7000F079BEB27812B1022A05D01DE0C6
:106D10001846FDF76AFC00F06FBE824A50780728DB
:106D200008D81BB9FDF75EFB00F066BEFDF776FBE9
:106D300000F062BEFF287FF467AF5D1C0ABF774B8F
:106D4000D8B21878FDF786FB00F056BE04233B70DE
:106D500000F052BEB378012B1CD005D3022B1DD1FD
:106D60007078FDF7BFFB0EE07078082802D8FDF7B9
:106D700082FB08E00A2802D100237B6010E00B2888
:106D800003D1FDF7AFFC60600AE0FF2808D1FDF7F2
:106D9000DDFBF8E7707802F05DFBF4E704233B705D
:106DA0005D4B1B78002B00F027865C4B62681A60F5
:106DB0005B4B2AB91A6842F008021A6000F01CBE48
:106DC0001A6822F008021A6000F016BE7178534A61
:106DD000092925D8DFE801F005080B0E12181B1E43
:106DE000212311680B441AE01168CB1A17E01168CF
:106DF0004B4314E0116891FBF3F310E0116891FB31
:106E0000F3F003FB10130AE011680B4007E0116870
:106E10000B4304E011684B4001E01368DB4313604F
:106E200012683F4B2AB91A6842F008021A6000F053
:106E3000E3BD1A6822F008021A6000F0DDBD374A8F
:106E400012689A42364B196804DD21F0030141F0C3
:106E5000040108E00BBF21F0060121F0050141F01B
:106E6000010141F0020119602AB91A6842F00802D2
:106E70001A6000F0C1BD1A6822F008021A6000F022
:106E8000BBBD72780C2A00F2B785DFE802F007106C
:106E900019222B344D565F68717A8300204A12689C
:106EA000140740F1A9851A4A536200F0A5BD1C4A97
:106EB0001268100700F1A085154A536200F09CBDCE
:106EC000174A1268D10740F19785114A536200F0C2
:106ED00093BD134A1268D20700F18E850C4A5362A3
:106EE00000F08ABD0E4A1268570740F18585084AAE
:106EF000536200F081BD0A4A126812F0050F00F0DB
:106F00007B85034A536200F077BD00BFCC1100209F
:106F10006405002046110020AB0C00209C0C0020D2
:106F2000A00A0020980A0020A84A1268960740F19B
:106F30006385A74A536200F05FBDA44A12689507B3
:106F400000F05A85A24A536200F056BD9F4A12686B
:106F5000D40640F151859E4A536200F04DBD9B4AD4
:106F60001268900640F14885994A536200F044BD8A
:106F7000964A1268510640F13F85954A536200F0E7
:106F80003BBD924A1268120640F13685904A536220
:106F900000F032BD8D4A1268D70540F12D858C4A2C
:106FA000536200F029BD916A072900F22585481C2B
:106FB0009062506A02EB8101C862536200F01CBD0E
:106FC000926A834B002A00F01785013A9A6203EB1C
:106FD0008202D26A5A6200F00FBD73782E2B04D859
:106FE0007C4A0121D15400F007BDFF2B7FF40CAE89
:106FF000774B012283F84C2000F0FEBC73782E2BD7
:1070000004D8744A0021D15400F0F6BCFF2B7FF461
:10701000FBAD6F4B002283F84C2000F0EDBC6C4CB4
:1070200094F84D2082B95E1C4FF00A0204D16A4BDD
:107030001B685A43226501E05343236502F06EF951
:107040000123606584F84D306B78042B00F2D48402
:10705000DFE813F0050045007F00C4001B0002F0CC
:107060005DF9626D216D801A80EAE072A2EBE07238
:107070008A42574B04D9002283F84D2000F0BCBC53
:107080005A6A013A5A6200F0B7BCA87804F0CCFA08
:1070900040B94E4B84F84D001A6822F010021A6075
:1070A00000F0AABC236D4A4DA3B102F037F96B6D15
:1070B0002A6DC01A80EAE073A3EBE073934209D90A
:1070C000002385F84D30414B1A6842F010021A60D7
:1070D00000F092BC636A013B636200F08DBCA8784B
:1070E000022894BF0020012004F025FCAA78012189
:1070F000022A92BF02FA01F3D31E5B0001FA03F3E6
:1071000013EA000609D0002384F84D302F4B1A688B
:1071100022F010021A6000F06FBC226D2C4D9AB163
:1071200002F0FCF86A6D296D801A80EAE072A2EB29
:10713000E0728A4208D9254B85F84D601A6842F002
:1071400010021A6000F058BC636A013B636200F0F1
:1071500053BCA8787C21022894BF002001206A46F5
:1071600004F0F6FBAA780220022A8ABFD31E53003D
:107170005B0000FA03F39DF8021013EA010709D03F
:10718000002384F84D30114B1A6822F010021A6067
:1071900000F032BC226D0E4D9AB102F0BFF86A6D5C
:1071A0002E6D801A80EAE072A2EBE072B24208D93A
:1071B000064B85F84D701A6842F010021A6000F014
:1071C0001BBC636A013B636200F016BCA00A00208E
:1071D000640500201E1300209C0C0020A8787C2150
:1071E000022894BF002001206A4604F0B1FBAA786F
:1071F0000120022A92BF02FA00F3D31E5B0000FABC
:1072000003F39DF8021013EA010708D0002384F865
:107210004D30AB4B1A6822F010021A60ECE3226D7D
:10722000A84D92B102F07AF86A6D2E6D801A80EA4C
:10723000E072A2EBE072B24207D9A14B85F84D7023
:107240001A6842F010021A60D6E3636A013B636277
:10725000D2E3B678052E1DD8062000FB02609A49BD
:1072600041F82030994B9B7E002B00F0C583002A0B
:1072700000F0C283531E18205843062303FB02620A
:1072800000F5C36001EB820100EB8600042201F0EF
:107290004BFAB1E3FF2E7FF42BA88B4E8AB9182549
:1072A000002405F5C06071192044214404220434EF
:1072B00001F03AFA182CF4D11835B5F5FC7FEFD16E
:1072C0009AE300246B7818205A1E5043062202FBD2
:1072D000034100F5C36000EB840006EB810104224A
:1072E000013401F021FA062CECD185E37378142BDC
:1072F0003FF68AAC764A9278052A19D8062101FB16
:107300000323714951F82320724B7A601B78002BBC
:1073100000F07283704B1A60694B22B91A6842F010
:1073200008021A6068E31A6822F008021A6063E330
:10733000FF2A7EF4DDAF644E8BB91825002405F5D5
:10734000C0607119204421440422043401F07FFA02
:10735000182CF4D11835B5F5FC7FEFD14CE300249F
:107360006B7818205A1E5043062202FB034100F599
:10737000C36000EB840006EB81010422013401F0BC
:1073800066FA062CECD137E37778142F3FF63CAC45
:10739000B678300634D50024A87840FA04F3D9072B
:1073A00015D5022894BF00200120022C8ABFE11EBF
:1073B00061014901464B41F00201C9B25E7804F017
:1073C00039FD062303FB06463F4B43F826003F4B9F
:1073D0009B7E8BB16B787BB15A1E182050430622DE
:1073E00002FB0343384900F5C36000EB840001EB66
:1073F0008301042201F098F90134062CCCD1FBE280
:10740000052E3EF675AF022E8ABFF11E71014901AD
:1074100041F00201C9B294BF0020012004F00AFD2E
:10742000062101FB0766294B274A9B7E42F826006E
:10743000002B00F0E1826B78002B00F0DD82244805
:1074400018258478581E684301FB034100F5C3608A
:1074500002EB810100EB8400042201F065F9CBE22C
:1074600072781D4B0A2A53D8DFE802F0060B11167A
:107470001C243A3F44494D0018491A6809680A44D7
:1074800003E016491A680968521A1A6040E0134965
:107490001A6809684A43F8E710491A68096892FBB4
:1074A000F1F2F2E70D4A1968126891FBF2F002FB63
:1074B0001012EAE7094A11681A680A40E5E700BFB6
:1074C000A00A002064050020A40A00200400002077
:1074D000980A0020AB0C00209C0C0020B80C002067
:1074E000A04A11681A680A43CFE79E4A11681A68D1
:1074F0004A40CAE79B4A1168C943116008E01A680C
:1075000098490A6004E0974A186811681060196089
:107510001A68954B22B91A6842F008021A606BE2A9
:107520001A6822F008021A6066E2904B1B68C6F8DF
:107530000330FDF7FFF95FE28C4B1B68C6F80330A0
:10754000FEF75CF858E27378052B00F25582DFE80D
:1075500003F003090F151B21834B1A6802F00F0279
:107560001A6049E2804B1A6822F010021A6043E266
:107570007D4B1A6822F020021A603DE27A4B1A68AD
:1075800022F040021A6037E2774B1A6822F080023C
:107590001A6031E2744B1A6822F480721A602BE28E
:1075A00072782E2A3FF630AB714901EB8202936567
:1075B00022E26F4B6D49D3F814210A60D3F81821E9
:1075C00068490A60D3F81C2167495A62D3F8202120
:1075D0000A60D3F82421674983F84D20D3F8282185
:1075E0005A65D3F82C211A6593F83021885C08B1CC
:1075F00001208854002283F83421FDE1B378052B63
:107600003EF676AE7278142A3FF6FEAA062101FBFA
:107610000233564A5849126841F82320ECE102F03F
:1076200011FAE9E102F010FAE6E102F01FFAE3E1F3
:1076300002F01DFAE0E102F01BFADDE102F019FAB6
:10764000DAE1727812B1012A05D00DE0484B01222F
:1076500083F82020D0E1B3F5006FBEF449AE444971
:1076600081F820204B62C7E103233B70C4E1404B0B
:10767000022283F82020BFE13D4A4FF0FF3002F1A3
:10768000580343F821003B480023435401312F297C
:10769000F2D182F820305362936282F84D30334A3F
:1076A0001360304A1360304A1360A5E1334A127DFB
:1076B00092070AD4B3F5006FBEF41AAE2C4A042127
:1076C00082F82010C2F8383196E108233B7093E12C
:1076D0002B4A01211170294A2A4C9178B3F5006F89
:1076E000217026D2127D12F0010522D1184669467A
:1076F00000F0DEFE9DF80030257263709DF80130C9
:10770000A3709DF80230E3709DF8063023719DF858
:10771000053063719DF80430A3719DF80330E37167
:107720000123E15C227A01330A44082B2272F8D14A
:1077300062E101230021E1540133082B114AF9D100
:107740001378137258E17378012B2FD01CD3022BBE
:107750003DD10B4B01221A70084B0A4A9B781370DB
:1077600000232BE0B80C0020A00A00209C0C002075
:10777000640500201E130020A40A0020040000203D
:10778000A00C0020A10C00209C4B01221A709C4BE5
:107790009C4A9B7813709C4B186800230133C118D6
:1077A00011F8011C082BD154F8D125E11722FA71E8
:1077B0007B71DE222A23BA713B711DE193490133AB
:1077C000194411F8091C082BD154F7D114E10323F3
:1077D0003B7011E17378032B00F20E81DFE803F0B8
:1077E000020F1B1F8A4B93F82020FA7193F84D204B
:1077F000D3F83831BA711A0A7A713B71FCE0844BC4
:1078000093F82020FA7193F84D205B6ABA711A0A36
:107810007A713B71F0E07F4B1B687B60ECE07E4B44
:107820001B687B60E8E07278002A40F0E5807B4AC4
:107830009178002940F0E08040F2D242934240F03B
:10784000DB8040F2FF7000F010FF00F072FE0120BC
:10785000FCF7BCFED0E07278714B02B101221A70C5
:10786000EA78704B1A706A4B93F83C116E4B1970A2
:107870006E4900230B706E490B706E4B19780A43EA
:107880001A70B9E0624B012283F83D21B4E07578AB
:1078900015B1012D0FD01BE0042240F2FB706946A8
:1078A00000F0D5FF009BD6F803209A4206BF0123C3
:1078B0007B607D60A0E0B3782A2B06D140F2FB709C
:1078C0005D49042200F030FF96E003233B7093E013
:1078D00003233B7090E07278032A3CD8DFE802F083
:1078E00008022D384A480022D0F84011054610E021
:1078F000474AD2F84011092907D8481CC2F840016C
:1079000002EB8102C2F8443176E009233B7073E058
:1079100001328A4270D04948960050F822409C4279
:10792000F6D18319481E824204D25C68013243F8C2
:10793000044BF7E7C5F840015EE0354A0023C2F882
:1079400040313E4A002199500433282BF9D153E0AD
:107950000A237B6050E003233B704DE07378812B5A
:107960004AD1B2782D4B922A46D19A79A32A43D193
:107970005A79B42A40D11A79C52A3DD1DB78D62B61
:107980003AD12F4B4FF400725A61C022C3F8102431
:1079900001F0F6FF01F0C2FC044601F0BFFC001B41
:1079A0000028B8BF4042B0F57A7FF6DBFCF715FE41
:1079B00005F006FF002006F0D7FB0021214805F066
:1079C000D8FA204805F03AFA1F4804F0ADFD05F05A
:1079D00015FB4FF0804006F01DFC0020FCF7F6FD83
:1079E0000AE040F2D242934206D1094B012283F8C9
:1079F0006C2101E00223237003B0F0BDA00C002035
:107A000004000020A10C002000000020004000081D
:107A1000640500209C0C0020B80C0020980A00206F
:107A20000811002054110020FF1200204C110020EA
:107A30004D130020091100209B0A0020A8060020F9
:107A40000008014008000240002401404849F8B500
:107A500000230B604749484A0B60484953629362D0
:107A60000B6082F84D3082F84C3082F83431164683
:107A7000434A4FF0FF3142F82310424A0024D454C5
:107A800001332F2BF4D1022C8ABFE11E6101490181
:107A900094BF0025012541F00601C9B2284604F033
:107AA000C9F9022C8CBFE11E6101374B88BF490127
:107AB00041F00C0143F82400C9B2284604F0BAF999
:107AC000A700324B0134062CD851DCD10024304BB6
:107AD000E0B203EB4413D97A0134C1F10801C9B211
:107AE00002F0FCF9062CF2D100232A4A0021995019
:107AF0000433B3F5806FF8D1274FBB7E8BB11825C7
:107B00000024264905F5C06029442044214404226C
:107B1000043400F09CFE182CF3D11835B5F5FC7F29
:107B2000EED1FB7E2BB13B7903F0EF02012A0DD1A0
:107B30000EE04FF4A7641A4920462144042204347D
:107B400000F085FEB4F5C36FF5D1ECE7212B01D130
:107B5000012300E0002386F86D317B7D23B1FCF723
:107B6000ADFD08B1012300E0002386F82030F8BD08
:107B70009C0C0020B80C002064050020A00A002006
:107B8000BC0500201E130020D4100020BC0C0020D7
:107B9000CC110020D40C002004000020A40A0020F6
:107BA0009C070020F7B50F4E0F4CC6F803300F4B63
:107BB00086460F46B270002294E803001A708DE8E2
:107BC000030086F800E07770FEF760FA21786368BA
:107BD000074A82F86E119DE8030084E80300184606
:107BE00003B0F0BD980A0020B00C0020AB0C0020C0
:107BF00064050020014B93F86E0170476405002076
:107C0000F7B51F4E024653780C4696E803008DE800
:107C100003001C4900270B7093786D464B70D37896
:107C20008B7013798B7153794B7193790B71D37975
:107C3000CB70154B1F70FEF729FA144B1978334699
:107C400071B9217032786170A2707278E270F27945
:107C50002271B27962717279A2713279E27109E0AE
:107C6000012907D13A460A4911444978A154013201
:107C7000082AF8D195E8030083E8030003B0F0BDBB
:107C8000B00C0020980A0020AB0C0020A00C0020B3
:107C9000A10C00202DE9F047A34B8EB01B78A34C1C
:107CA00013B994F86F3163B1A14B1B78062B08D040
:107CB0000A2B06D003F0EF030F2B1CBF002384F820
:107CC0003C3194F83C31994A591E0129994E41D8CA
:107CD0009949012BCA6814BF082307238DF818306F
:107CE00094F87031079232788DF8193000238DF8AE
:107CF0001A30C2B98B688DF827208DF820308F4B51
:107D000019788DF8211059788DF82210D9798DF8CD
:107D1000231099798DF8241059791B798DF8251045
:107D20008DF826300AE0012A08D1854901330EAAD0
:107D3000595C1A44082B02F8191CF6D1814B1B78A8
:107D4000002B40F0B88006A801F026FA002800F0C9
:107D50009C83B0E0032B2AD192F86D511DBB337880
:107D60008BB9754F754DB87897F801802A788044A3
:107D700090446A789044EA799044AA7990446A7968
:107D800090442A7920E0012B40F095806C4B585D9F
:107D9000013500F01BFF092DF8D18CE0072B6AD1CB
:107DA00092F86D3173B3654804F040FB83E0042B17
:107DB000F4D1614F614DB87897F80180002301221A
:107DC0006B702A706B608044904400F0FFFE7878FE
:107DD00000F0FCFE287800F0F9FE687800F0F6FE6E
:107DE000E87900F0F3FEA87900F0F0FE687900F081
:107DF000EDFE5FFA88F8287900F0E8FE404600F0D2
:107E0000E5FE58E032782ABB4B4B93F802C093F85A
:107E100001804A4B8DF800C01F785D78C444D87942
:107E20008DF80270674499798DF803503D445A7972
:107E30008DF8040028441B798DF8051001448DF855
:107E400006200A448DF8073013448DF801808DF820
:107E5000083008E0012A06D1394A9A5C0DF803205F
:107E60000133092BF8D1374B1B7823B3684609211E
:107E700001F0BAFD1FE0082B1DD1304A002301207C
:107E80005370107053602C4A8DF80200917852782C
:107E90008DF800108DF801200A4402448DF803305B
:107EA0008DF804308DF805308DF806308DF80730E8
:107EB0008DF80820D7E7244B224F1A789946002ADC
:107EC00000F09780214B224D1B78013B062B00F2DE
:107ED0008C80DFE803F004043F8A8A8A6800164A2F
:107EE000297893688DF836108DF8303080238DF81E
:107EF00031308A238DF8323000238DF833308DF8FD
:107F000034308DF835308DF829308DF82A30D3682B
:107F100007210B933B788DF82810002B65D10AA818
:107F200001F03AF961E000BFAA0C002064050020CE
:107F3000980A0020A00C002004000020B00C0020B3
:107F4000A10C0020EC1000204D130020FF12002097
:107F50004C110020DFF840832A7898F8020098F846
:107F600001A082440AF10A0A924400F02FFE98F818
:107F7000010000F02BFE802000F028FE8A2000F097
:107F800025FE002000F022FE002000F01FFE002051
:107F900000F01CFE5FFA8AFA287800F017FE5046BF
:107FA00000F014FE21E0BC4B2A78987859788023A1
:107FB0008DF80E308A238DF80D108DF80F300144A6
:107FC00000238DF810308DF811308DF812300A3101
:107FD0003B788DF813200A448DF80C008DF814209E
:107FE0001BB103A8092101F0FFFC00232B7089F8C5
:107FF0000030002384F83C31337084F86F3194F8FA
:108000006C3113B10120FCF7E1FA94F83D21A34B48
:1080100052B193F86D21D2F1010238BF002283F8EA
:108020006D21002283F83D213B78002B45D106A825
:1080300001F0FCF8002840D09DF81830062B3CD900
:10804000974B9DF820201A709DF821205A709DF8BA
:1080500022209A709DF823209A719DF824205A714D
:108060009DF825201A719DF82620DA709DF81930A8
:1080700084F87031884B1A69079B934203D1874B70
:10808000012283F86F2101F049F9864B0022186024
:10809000854B1A709DF8183094F82020072B0CBFE0
:1080A0000123022384F83C31531E012B7F4B02D95C
:1080B000052A40F0CF800022EBE094F86D51002DAE
:1080C00071D103A800F09CFD00286CD000F0B6FD33
:1080D00010B1724B83F8715194F871119DF80C0036
:1080E0004A1CD2B22144092A6C4B84F8712181F8D0
:1080F000720140F0E480002283F87121664A93F80F
:1081000072315178994207D092F82710002900F077
:10811000D6808B4240F0D38092F827209A4204BF49
:10812000012384F86F3100231A465C4D05F5B971BF
:10813000595C01330A44082BD2B2F6D195F87A3152
:1081400093422CD1564B95F873211A7095F87421EF
:108150005A7095F875219A7095F876219A7195F86C
:1081600077215A7195F878211A7195F87921DA708A
:1081700001F0D4F84E4B4F4A186095F820100023B8
:108180001370032285F83C214A1E012A85F87131BB
:10819000464A02D9052918BF012313708FE0042332
:1081A00085F83C318BE094F86D313C4D83B13C480F
:1081B00003F0EFFF60B101F0B1F83D4B3D4A1860AC
:1081C00000231370032285F83C2195F820203AE023
:1081D00094F86D61002E44D13B78002B41D00AAD5C
:1081E000284601F0EBFB00283BD033463246E95CE1
:1081F00001330A44082BD2B2F9D19DF830109142D4
:108200002CD1274B9DF829201A709DF82A205A70EE
:108210009DF82B209A709DF82C209A719DF82D20A6
:108220005A719DF82E201A719DF82F20DA7001F0F6
:1082300075F81F4B1F4A186000231370072284F83B
:108240003C2194F82020511E01291946174B03D9CF
:10825000052A01D001221CE0197030E084F83C317D
:108260002DE094F820300D4D013B012B27D86B6A8F
:10827000B3F5006F20D2FCF721FAE8B1686A08492B
:10828000431C6B6200F014F9092385F83C31074B5D
:1082900001221A7013E000BF0400002064050020D2
:1082A000980A0020EC120020ED100020AB0C0020FA
:1082B000F4120020FE120020002384F8203094F8ED
:1082C0002030734D042B04D1724E3278170640F1E2
:1082D000B18094F83C3113F0FB0F05D0082B03D08C
:1082E000062B01D0FDF7D2FE94F83C31092B79D151
:1082F00001F014F8664A684D52692B68801A80EACA
:10830000E072A2EBE0729A4208D9644B1A78012A13
:1083100004BF02221A7001F001F8606100F0FEFF54
:10832000A3696A68C01A80EAE073A3EBE073934222
:1083300008D95A4B5A78012A04BF02225A7000F019
:10834000EDFFA06100F0EAFFE369AA68C01A80EAC5
:10835000E073A3EBE073934208D9504B9A78012A5B
:1083600004BF02229A7000F0D9FFE06194F84C300B
:10837000002B37D0464B93F83421002A32D147499D
:108380008B5C022B2BD1424B03F1580050F822009A
:10839000451C22D0424983F8302109680022C3F8E5
:1083A000141140490968C3F81811596A5862C3F892
:1083B0001C113D490968C3F8201193F84D1083F84A
:1083C0004D20C3F82411596D0122C3F82811196DED
:1083D00083F83421C3F82C1104E000238B540132BC
:1083E0002F2ACCD194F83C11294B092906D193F8B6
:1083F0002020022A04BF052283F82020D4F840213F
:10840000234B002A41D009293FD193F8201001299C
:108410003BD1586A00231E4901F5A27454F8234049
:10842000A04203D1052381F820302EE0013393428E
:10843000F1D12AE095F83C3113F0FB0F25D0082B41
:1084400023D0062B21D0D5F83801184CD6F80330AC
:10845000B0F5006F6270636012D2314600F03BF9F4
:10846000D5F83801314600F0A8F830B1D5F83831E8
:108470000133C5F83831652300E00723237004E099
:1084800007232370002385F820300EB0BDE8F08765
:1084900064050020980A0020A81200201E13002066
:1084A0009C0C0020B80C0020A00A0020B00C00207A
:1084B000C0EBC00038B500F5006500200C46024650
:1084C0000321FCF7A9F90020C5F307210246FCF7B8
:1084D000A3F90020E9B20246FCF79EF9002001460C
:1084E0000246FCF799F92070002001460246FCF78D
:1084F00093F96070002001460246FCF78DF9A070E8
:10850000002001460246FCF787F9E0700020014692
:108510000246FCF781F92071002001460246FCF773
:108520007BF96071002001460122FCF775F9A0710A
:1085300038BD38B54FF40064002006210122FCF755
:108540006BF9002005210246FCF766F90020014680
:108550000122FCF761F98307F3D5002002210246CE
:10856000FCF75AF90020C4F307210246FCF754F93E
:108570000020E1B20246FCF74FF90025B5F13F0EAD
:10858000DEF100024FF0000052EB0E020146013511
:10859000FCF742F9402DF1D1002005210246FCF7FD
:1085A0003BF9002001460122FCF736F9C307F3D45A
:1085B0004034B4F5804FBFD138BDF7B5C0EBC00033
:1085C00000F5006500200C4602460321FCF724F963
:1085D0000020C5F307210246FCF71EF90020E9B28E
:1085E0000246FCF719F9002001460246FCF714F98F
:1085F0000746002001460246FCF70EF90646002019
:1086000001460246FCF708F90546002001460246ED
:10861000FCF702F98DF80300002001460246FCF742
:10862000FBF88DF80400002001460246FCF7F4F840
:108630008DF80500002001460122FCF7EDF82378B3
:108640008DF80600BB420DD16378B3420AD1A378FE
:10865000AB4207D1DDF80300D4F80330C31A584207
:10866000584100E0002003B0F0BD38B501220446B7
:108670000D4600200621FCF7CFF800200521024618
:10868000FCF7CAF8002001220146FCF7C5F8820772
:10869000F3D5002002210246FCF7BEF80020C4F307
:1086A00007210246FCF7B8F80020E1B20246FCF7C9
:1086B000B3F8002029460122FCF7AEF8002005217E
:1086C0000246FCF7A9F8002001460122FCF7A4F8B5
:1086D000C307F3D438BD38B5C0EBC0050C4605F56B
:1086E00000600978FFF7C1FF05F601006178FFF728
:1086F000BCFF05F60200A178FFF7B7FF05F60300FF
:10870000E178FFF7B2FF05F604002179FFF7ADFF2E
:1087100005F605006179FFF7A8FF05F60600A179C7
:10872000BDE83840FFF7A1BF2DE9F04104460F46F0
:108730001646002006210122FCF76EF800200521D4
:108740000246FCF769F8002001460122FCF764F8B4
:108750008507F3D5002002210246FCF75DF80020D2
:10876000C4F307210246FCF757F80020E1B20246A5
:10877000FCF752F80025B54242D0013414F03F080E
:10878000795D04D0721EA81A4242424100E00122E3
:108790000020FCF741F8B8F1000F2FD1731E9D4265
:1087A0002CD2002005210246FCF736F800200146B5
:1087B0000122FCF731F810F00100F2D1062101226C
:1087C000FCF72AF8002005210246FCF725F80020D6
:1087D00001220146FCF720F88207F3D50020022190
:1087E0000246FCF719F80020C4F307210246FCF703
:1087F00013F80020E1B20246FCF70EF80135BAE7A3
:10880000002005210246FCF707F80020014601225E
:10881000FCF702F8C307F3D4BDE8F08110B50446B5
:10882000002003210246FBF7F7FF0020C4F30721D5
:108830000246FBF7F1FF0020E1B20246FBF7ECFF36
:10884000BDE81040002001460122FBF7E5BF70B5EE
:10885000044600200E46154603210246FBF7DCFFC6
:108860000020C4F307210246FBF7D6FF0020E1B247
:108870000246FBF7D1FF0024AC420AD06A1EA31ABD
:1088800000205A4201465A41FBF7C6FF30550134D9
:10889000F2E770BD37B5002005210246FBF7BCFFAB
:1088A000002001460122FBF7B7FF10F07104F2D15E
:1088B00000F034FD054600F031FD401B0028B8BF34
:1088C0004042B0F5FA6F09DA4CB940F2FF70FFF799
:1088D000A5FFB0F142035C425C41ECE71CB1294BBF
:1088E0001B78002B3CD040F2FF700021FFF7BDFE4B
:1088F000FFF71FFE002024494022FFF715FF002448
:10890000B42202FB04F0214900F58070FFF70CFF50
:10891000A01C40011E4920220134FFF705FF062C50
:10892000EED1002301934FF4C364204601A9042231
:108930000434FFF7F9FEB4F5FF6FF6D1002301937D
:108940004FF4A764204601A904220434FFF7ECFE8B
:10895000B4F5C36FF6D140F2FF704221FFF785FEF8
:10896000002009494022FFF772FF402409492046B0
:10897000214420222034FFF76AFFB4F5807FF5D12F
:1089800003B030BD70110020040000206013010806
:10899000401301088C11002030B5054687B05548BA
:1089A00006F024F94FF40030012105F0BDF9042050
:1089B000012105F0ADF90420002105F0C1F90820DE
:1089C000002104F0BDFE03238DF8063018230DEBC3
:1089D00003048DF80730042324F8143D464821464B
:1089E00004F01FFE48238DF8073043480823214632
:1089F000ADF8043004F015FE02A806F085F90B2D41
:108A000025D8DFE805F02406090C0F1215181B1EE7
:108A100020224FF461531CE04FF4964319E04FF4C9
:108A2000E14316E04FF4164313E04FF4614310E0C6
:108A30004FF496330DE04FF4E1330AE04FF4613325
:108A400007E02E4B05E02E4B03E02E4B01E04FF4E8
:108A500016530293029B02A95B082648029306F074
:108A60000FF92623002401258DF8003068460723DE
:108A70008DF801308DF802408DF8035004F0DCFED3
:108A80001C4840F2FF3106F027FA224619482821F7
:108A900006F067F92A46174840F2277106F061F997
:108AA0002A46144840F2266106F05BF92A4611482E
:108AB00040F2255106F055F922460E4840F2244175
:108AC00006F04FF922460B4840F6460106F049F9F8
:108AD0002246084840F66A1106F043F92246054846
:108AE000602106F03EF90348294606F02EF907B04A
:108AF00030BD00BF004400400008014090D003009A
:108B000020A1070040420F00684620F007018D4673
:108B1000294919B50B889C061AD5284BDB6898079C
:108B200001D58B8814E0264B1A6858680132202A38
:108B300008BF0022824205D01C6888881919C0B27B
:108B400008721A601F4A0A2111609A6A1E4B1A6045
:108B5000194803881A061BD51B4B1A68C2B9184B53
:108B6000DC6A196B8C420FD0144902240C61196B1A
:108B70004C1C1C63194491F83410C9B28180196BE4
:108B8000202905D11A6303E040F2277106F0E9F8C5
:108B9000094803885B060BD540F2266106F0C0F950
:108BA000074B1A6BDB6A9A4202D1044B02225A61CC
:108BB000BDE8194085467047004400400008014068
:108BC000E006002054130020501300200A4BDA6AFC
:108BD000196B0132202A08BF00228A420AD0D96AC2
:108BE000194481F83400DA62044840F22771012206
:108BF00006F0B7B8704700BFE00600200044004010
:108C00000A4B59681A6891420BD05A68511C596036
:108C10001A44127A02705A68202A04D100225A603B
:108C200001E0002070470120704700BFE0060020EF
:108C3000014B9862704700BFE0060020044B1A7891
:108C400002F0FF0012B100221A700120704700BF2D
:108C50005813002008B5FBF7C0FC044B00225A60F3
:108C60001A60BDE80840FBF7B6BC00BFE006002074
:108C700010B5441E14F8010F10B1FFF7A7FFF9E774
:108C800010BD00BF684620F007018D4631B5264C67
:108C9000264B25681B680135082D08BF00259D421D
:108CA00086B04FF0000037D001A903F0A9FF9DF86E
:108CB0000C302268042B1E4B03EB021206D101215B
:108CC00051702168029A03EB011105E000215170F7
:108CD0002168019A03EB01114A609DF80D20022AD8
:108CE000226808BF012103EB021218BF0021917016
:108CF00022689DF80E10120199540022216801A8E3
:108D0000104403EB01111144C07A0132082A0872A1
:108D1000F4D1054B1D6001E003F058FF06B0BDE83B
:108D200031408546704700BFE81300205C130020E7
:108D300068130020684620F007018D4631B5264CA7
:108D4000264B25681B680135082D08BF00259D426C
:108D500086B04FF0010037D001A903F051FF9DF814
:108D60000C302268042B1E4B03EB021206D10121AA
:108D700051702168029A03EB011105E00021517046
:108D80002168019A03EB01114A609DF80D20022A27
:108D9000226808BF012103EB021218BF0021917065
:108DA00022689DF80E10120199540022216801A832
:108DB000104403EB01111144C07A0132082A0872F1
:108DC000F4D1054B1D6001E003F000FF06B0BDE8E3
:108DD00031408546704700BFE81300205C13002037
:108DE00068130020684620F007018D4631B52A4BF4
:108DF0002A4A1968126886B0914204D101200021E4
:108E000003F01EFE43E01A68254901EB0212507878
:108E100000F0FF0248B104228DF80C2000220192DC
:108E20001A6801EB0212526806E018688DF80C20EF
:108E300001EB00104068019002921A6801EB0212E7
:108E4000927802F0FF001AB102228DF80D2001E0A5
:108E50008DF80D001A6812018A5C8DF80E20002230
:108E60001C680D4801EB04141444257A01AC144429
:108E70000132082AE572F3D1036801330360036805
:108E8000082B04BF0023036001A803F0E5FD06B032
:108E9000BDE8314085467047641300206013002010
:108EA000EC130020F0B501388BB00F4615460C23AB
:108EB000072813D8DFE800F0100E0C0A0812060489
:108EC00002220CE004220AE0102208E0142206E04C
:108ED000282204E0642202E0C82200E008228DF883
:108EE000143003238DF815300023ADF816208DF8CB
:108EF000133003F0B7FC4FF00070012104F014FFB1
:108F00000120014604F004FF0820012104F000FFC5
:108F10000820002104F014FF4FF4EA10012104F0AE
:108F20000FFC03238DF8063018230AAC8DF80730A8
:108F30004FF4007324F8243D2146784804F071FB77
:108F4000042321468DF8073074484FF480730024C1
:108F50000126ADF8043004F064FB03A88DF812403C
:108F60008DF80C408DF80D608DF80E408DF80F4097
:108F70008DF810608DF8116003F081FCB7F5006F7B
:108F80008DF818408DF819408DF81A600FDA7B01C2
:108F9000ADF81C304FF6FF73ADF81E40ADF8203031
:108FA000ADF82230ADF824408DF826600DE04FF684
:108FB000FF73ADF81C40ADF81E40ADF82030ADF8A1
:108FC0002230ADF824408DF8264006A803F0B6FC08
:108FD000012300228DF818308DF819208DF81A30F1
:108FE00095B1B5F5006F0FDA6901ADF81E204FF6A7
:108FF000FF72ADF81C10ADF82020ADF82220ADF8BE
:1090000024308DF826300DE04FF6FF71ADF81C20AE
:10901000ADF81E20ADF82010ADF82210ADF82430C8
:109020008DF8262006A803F089FC02238DF818305D
:109030007B13FF0047F0040700260124ADF81E70E3
:1090400006A84FF6FF77ADF81C308DF819608DF843
:109050001A40ADF82070ADF82270ADF824608DF89C
:10906000264003F06BFC0323B5428DF818308DF8D1
:1090700019608DF81A4010DD6B13ED0045F0040502
:10908000ADF81C30ADF81E50ADF82070ADF8227070
:10909000ADF824408DF826400CE00423ADF81C60A8
:1090A000ADF81E30ADF82070ADF82270ADF8244058
:1090B0008DF8266006A803F041FC01240726002550
:1090C000142302A88DF808308DF809608DF80A5035
:1090D0008DF80B4004F0B0FB152302A88DF8083082
:1090E0008DF809608DF80A508DF80B4004F0A4FB50
:1090F000132302A88DF808308DF809608DF80A5006
:109100008DF80B4004F098FB2146022003F098FCF8
:109110001020214603F094FC0BB0F0BD000C014080
:1091200037B50220002103F08BFC1020002103F052
:1091300087FC0021012003F083FC00240725142371
:1091400001A88DF804308DF805508DF806408DF893
:10915000074004F071FB152301A88DF804308DF849
:1091600005508DF806408DF8074004F065FB132389
:1091700001A88DF804308DF805508DF806408DF863
:10918000074004F059FB03F06DFB4FF000702146DF
:1091900004F0CAFD03B030BDF0B5437887B0044693
:1091A000426833B104238DF80C30002302920193FE
:1091B00003E08DF80C3001920293A37803B10223EF
:1091C0008DF80D3023788DF80E300023E11801AAB8
:1091D0001A44097A0133082BD172F7D101A803F0A0
:1091E0003BFC042816D10E4F0E4B3D681B68013521
:1091F000082D08BF00259D420ED03E680A4B03EBA8
:10920000061694E80F0086E80F00012001463D6035
:1092100003F016FC012000E0002007B0F0BD00BF05
:109220006013002064130020EC13002030B50D4BB8
:109230000D4C054622681B689A420ED023685A1CC2
:1092400022600A4A02EB03130FCB85E80F00236864
:10925000082B04D10023236001E0002030BD012051
:1092600030BD00BFE81300205C130020681300200D
:10927000684620F007018D4601B5BDE801408546EE
:10928000704700BF684620F007018D4601B5124BBC
:1092900019781A4679B15B68013353600F4B19682E
:1092A000013119600E4B196811B119680139196043
:1092B0000023137001E001221A700A4B1A683AB1B8
:1092C0001A68013A1A601B6813B9074B01221A7019
:1092D000BDE801408546704734070020AC0C0020F3
:1092E00050130020541300205813002008B5042008
:1092F00004F014FF48F6A04004F01CFF012004F025
:109300001FFF05480321002204F06CFBBDE8084064
:10931000012004F029BF00BF9AC30200014B586826
:10932000704700BF34070020F0B593B00325002438
:109330000227424801A9ADF804708DF806508DF857
:10934000074004F06EF911233D4801A9ADF804303F
:109350008DF806508DF8074004F063F901200146AE
:1093600004F0CAFC01214FF4007004F0D1FC354830
:1093700003F064FD344B33480793344B07A908933B
:1093800080230C934FF480730D934FF480630E93FE
:1093900020230F934FF40053109309940A950B94D4
:1093A000119403F0BBFD2748012103F0E2FD0126E3
:1093B0004FF46023264802A9049302948DF80C60B0
:1093C0008DF80D6005948DF8185003F0D9F82048F9
:1093D0000A2132462B4603F04BF91D480E213A462E
:1093E0002B4603F045F92B46194809212A4603F07C
:1093F0003FF9224616484FF4FC6103F000F9144887
:10940000314603F0F3F81248314603F0E6F810480D
:1094100003F0FEF80E4803F000F90028FAD10C48DA
:1094200003F0FFF80A4803F001F90028FAD10848D0
:10943000012103F0FFF813B0F0BD00BF000C0140A4
:1094400000100140080002404C2401403C0700206D
:1094500000240140042805D0082807D070B9084B23
:10946000188801E0064B588880B27047044B9888F2
:1094700040F26B1380B258430013704700207047CE
:109480003C070020014B00221A607047440700206F
:10949000034B9B7A13B1034B05225A60704700BF00
:1094A0007814002044070020014B04225A607047C2
:1094B00044070020034B1A7A202A04BF00221A72A4
:1094C000704700BF440700207047212810B508D11D
:1094D000104B1B681B7803F07F03212B10D0022058
:1094E00010BD2028FBD10B4B0B4A1B681B78107258
:1094F00003F07F03212B094B18BF00230BB9EEE7C4
:10950000074B044A0024126820469361548298470E
:10951000204610BDD8140020440700207195000893
:1095200059950008074B1B681B7803F07F03212B1C
:1095300006D100F0DF0002280CBF00200220704797
:1095400002207047D814002021B9022834BF00201F
:10955000022070470220704720B9034B08221B6885
:109560001A82704701487047D81400204400002038
:1095700020B9034B08221B681A82704701487047C4
:10958000D81400204400002008B5032006F06AFC2F
:10959000064B0246D8604FF48871054806F014FA6D
:1095A000BDE80840032006F0DCBA00BF44070020F5
:1095B000DE14002038B5334B00241B68C0259C7294
:1095C0005D72DC72204606F03BFA20464FF40071D3
:1095D00006F053FA2046102106F066FA2046402194
:1095E00006F0C2FB8021204606F0ADFB204606F0C7
:1095F000E4FA254B204693F8341006F002FC20468E
:1096000006F0AFFA0120214606F037FA012029467C
:1096100006F099FB0120202106F046FA01202146A0
:1096200006F057FA02204FF4C06106F026FA022035
:109630004FF4807106F087FB0220214606F049FABC
:109640000220202106F030FA0320214606F015FA08
:1096500003204FF4887106F087FB0320402106F0B9
:10966000D0FB03204FF4405106F033FA032021468B
:1096700006F01AFA204606F045F8044B01225A601B
:1096800038BD00BFD814002044000020440700204B
:10969000014905F031BE00BF7C000020014905F002
:1096A0002BBE00BF84000020054B1B68DB78042B19
:1096B00004D8044901EBC30105F01EBE0020704729
:1096C000D81400208C00002008B5002004F09EFA79
:1096D000BDE808404FF40000012104F025BB024B17
:1096E00003225A60704700BF44070020044B9A7A57
:1096F000044B0AB1052200E001225A60704700BF06
:10970000781400204407002007B514238DF8043096
:1097100000238DF805308DF8063001A801238DF85F
:10972000073004F089F803B05DF804FB20B1054868
:109730004FF4806103F0DDBF02484FF4806103F015
:10974000DABF00BF000801407047684620F00701FB
:109750008D4679B5154D164B2A681C4692B21A8073
:10976000144A188811881646014011F4806F05D0FC
:109770004FF6FF332B60104BDB6898472388328805
:109780001340990507D54FF6FF532B600B4B197CFF
:109790000131C9B2197423881A40130401D506F0A7
:1097A00019F8BDE879408546704700BF445C004029
:1097B0006E1400201E1500204400002044070020E5
:1097C00008B509484FF4806103F093FF074B01226D
:1097D0001A60074A00200749186010604FF4E052F1
:1097E0000A801A6008BD00BF00080140405C0040CC
:1097F000445C00401E150020084B10B51B68002477
:109800009C72FFF7DDFF064B064A1C604FF40643CF
:109810001380054A1360054B5C6010BDD81400200E
:10982000445C00401E150020405C004044070020BE
:1098300038B5064D01232B60054B00241C602046E3
:10984000FFF774FF03232B60204638BD405C0040C7
:10985000445C0040074B1A6892B242F008021A605A
:109860001A6892B242F004021A60034B03225A6053
:10987000704700BF405C00404407002010B5064C14
:109880004FF6FB73226813402360FFF72FFF4FF45E
:109890000643236010BD00BF405C004010B51E4C65
:1098A000072818BF20702378052B32D8DFE803F093
:1098B00003060A0E1621FFF7E1FF2AE0FFF7DEFF9D
:1098C000042327E002236370032323E06378013B32
:1098D000DBB263706378F3B9042217E00F4B1A68A8
:1098E00092B242F010021A60052323700A236370BB
:1098F00010BD6378013BDBB2637063785BB9074AE4
:109900004FF6EF7311680B4013600622024B1A707A
:1099100010BD0623237010BDDC140020405C004005
:1099200007B5FFF7D1FEFFF7EFFE05F037FF042084
:10993000012104F0EDF94FF48063ADF80430032306
:109940008DF806300448102301A98DF8073003F084
:1099500068FE03B05DF804FB0008014007B514235E
:109960008DF8043000238DF805308DF8063001A8FD
:1099700001238DF8073003F05FFF03B05DF804FBAF
:10998000FFF756BF0B4910B5CA6882B14B68052B6B
:109990000CD10023CC68A34204D2074C1C5DC454F4
:1099A0000133F7E7034B0021D96000E000221046A5
:1099B00010BD00BF44070020DE140020084BDA6809
:1099C000082A1A460AD900230649595CC1540133B2
:1099D000092BF9D10023D360012070470020704784
:1099E00044070020DE14002010B5084C0A46216010
:1099F00092B2C02105F0D0FF0120218806F0E0F9E5
:109A0000BDE81040012006F09DB800BF44070020CB
:109A1000704710B5FFF782FC074C2368C01AB0F5F9
:109A2000FA7F07D9054BDA6882F40062DA60FFF743
:109A300075FC206010BD00BF20150020000C014007
:109A40007047704770477047054B064AD3F80310BC
:109A5000054B09B9928800E0128992B25A607047AA
:109A6000980A0020006C0040B00C0020704770473E
:109A700070477047F8B50F4B0D461E5CC1F30741A8
:109A800000223046FAF7C8FE0B4C0702C5F3072147
:109A9000002230462760FAF7BFFE38430702E9B2DA
:109AA000304601222760FAF7B7FE384307092760DE
:109AB000F8BD00BF411401085807002038B5484CD4
:109AC0000B2303FB004203FB0043117904330329FA
:109AD00084BF032111719A78032A84BF03229A70EC
:109AE0000B2303FB004203FB0043117A04320F29CE
:109AF00084BF0F2111715A7A0433072A84BF0722C9
:109B00005A710B2303FB004203FB0043917A04329A
:109B10000F2984BF0F2191715A7B0C330F2A84BF08
:109B20000F225A700B2202FB004302FB0042997B7A
:109B30000C330F2984BF0F21997013795279DB03FD
:109B400043F40021A1641AB1254943F404238B6432
:109B50000B2101FB0041C979214B19B1996C41F4EA
:109B6000005199640B2372B903FB0043197A9A7967
:109B7000C90141EAC2210433A26C5B790A4342EA7B
:109B80000312A2641AE003FB00431B7B144A1BB1BF
:109B9000936C43F4805393640B2202FB0042917B4D
:109BA000557BA26C0E4B42EAC51201F0070542EA52
:109BB0000512090748BF42F400629A640B2202FBB7
:109BC0000042D17A064B043219B991799A6C0A4352
:109BD0009A64A16CFFF74EFFA36CE36438BD00BF2D
:109BE0005807002010B5144C0023A364C300E218EA
:109BF00092F8552012B14FF40072A264E11891F866
:109C000056100D4A19B1916C41F480719164E218BB
:109C100092F8571023440F2984BF0F2182F8571060
:109C200093F85710A36C1943A164FFF723FFA36CAB
:109C3000C4F8803010BD00BF5807002038B5234C51
:109C40004FF46023A364C300E21892F88B2012B192
:109C50004FF47022A264E21892F8851092F88450B2
:109C6000090341EA853192F88620A56C012A41EA70
:109C70000501A16403D1154A41F480619164E118A2
:109C800091F88750A26C91F8881042EA05220129C8
:109C9000A26403D10D4942F080028A64E11891F870
:109CA00089100A4A012903D1916C41F04001916465
:109CB000234493F88A10A36C43EA0111A164FFF7CF
:109CC000D9FEA36CC4F8B43038BD00BF58070020DB
:109CD00038B52A4C43001A18224492F9B910B83208
:109CE0003F29C4BF3F2151701A18224492F9B9107C
:109CF000B8323F31BCBFC12151701A18224492F8CA
:109D0000BA10B8321F2984BF1F2191704FF440222E
:109D1000A2641A18224492F8B820012A03D1174AE3
:109D20004FF45021916404EBC00191F88B10134A59
:109D300051B91918114491F8B950916C05F07F058B
:109D400041EA052191640CE01D18154495F8B950BD
:109D500001F0030105F07C052943956C45EA0125D6
:109D600095640344234493F8BA10A36C1943A16487
:109D7000FFF780FEA36CC4F8CC3038BD5807002034
:109D800010B58300254C1A18224492F8D0100129EE
:109D900084BF012182F8D0101A18224492F8D11001
:109DA000D032032984BF032151701A18224492F83B
:109DB000D210D0320F2984BF0F2191701A1822447B
:109DC00092F8D310D032032984BF0321D1701A181E
:109DD000224492F8D41003440F2988BF0F2102F1C6
:109DE000D00288BF1171234493F8D41003F1D0023C
:109DF00093F8D03041F4202141EAC331537841EA4D
:109E00004331937841EA0321D37841EA4311A164B5
:109E1000FFF730FEA36CC4F8F03010BD58070020E7
:109E200000202C4AF8B5054604462B4E0327A6F120
:109E300034016F54331929444FF0050E4FF0010CD3
:109E400004F806C081F805C083F801E04FF0020C69
:109E500083F802E000234F708B70CB700B7181F898
:109E600006C0CB713C4406F11801683E43542E44B1
:109E70000144122C82F800C05370D370937082F8A2
:109E800004C0577182F806E0D3711372977253724F
:109E90004B708B70CB700B717371B371F37105F1F3
:109EA0000805704402F10B02BFD11D46ECB22046FA
:109EB000FFF766FF2046FFF70BFF2046FFF7BEFEC9
:109EC0002046FFF78FFE01352046FFF7F7FD062DF0
:109ED000ECD1F8BD5C07002010080020064B0429D7
:109EE00003EBC00318BF002283F8571018BF83F894
:109EF0005520FFF777BE00BF58070020054B03EB46
:109F0000C00383F8551011B1042283F85720FFF7DE
:109F100069BE00BF58070020034B03EBC00383F862
:109F20005610FFF75FBE00BF58070020024B03EB3F
:109F3000C00090F85700704758070020024B03EB11
:109F4000C00090F85500704758070020024B03EB03
:109F5000C00090F85600704758070020034B0B22B2
:109F600002FB00331971FFF7A9BD00BF580700209D
:109F7000034B0B2202FB00335971FFF79FBD00BF5B
:109F800058070020034B0B2202FB0033D971FFF767
:109F900095BD00BF58070020034B0B2202FB003386
:109FA0009971FFF78BBD00BF58070020034B0B22B0
:109FB00002FB00331972FFF781BD00BF5807002074
:109FC000034B0B2202FB00335972FFF777BD00BF32
:109FD00058070020034B0B2202FB00339972FFF756
:109FE0006DBD00BF58070020034B0B2202FB00335E
:109FF0001973FFF763BD00BF58070020034B0B2206
:10A0000002FB00335973FFF759BD00BF580700200A
:10A01000034B0B2202FB00339973FFF74FBD00BFC8
:10A0200058070020024B0B2202FB003000797047DA
:10A0300058070020024B0B2202FB0030407970478A
:10A0400058070020024B0B2202FB0030C0797047FA
:10A0500058070020024B0B2202FB0030807970472A
:10A0600058070020024B0B2202FB0030007A704799
:10A0700058070020024B0B2202FB0030407A704749
:10A0800058070020024B0B2202FB0030807A7047F9
:10A0900058070020024B0B2202FB0030007B704768
:10A0A00058070020024B0B2202FB0030407B704718
:10A0B00058070020024B0B2202FB0030807B7047C8
:10A0C00058070020034A00EB8003134483F8D010A4
:10A0D000FFF756BE58070020034B00EB80021344E5
:10A0E0005970FFF74DBE00BF28080020034B00EB5E
:10A0F000800213449970FFF743BE00BF2808002078
:10A10000034B00EB80021344D970FFF739BE00BF48
:10A1100028080020034B00EB800213441971FFF75D
:10A120002FBE00BF28080020034B00EB800018441E
:10A1300090F8D000704700BF58070020024B00EB9A
:10A14000800018444078704728080020024B00EB3C
:10A15000800018448078704728080020024B00EBEC
:10A1600080001844C078704728080020024B00EB9C
:10A17000800018440079704728080020034A00EB4B
:10A180004003134483F8B810FFF7A2BD580700201E
:10A19000034B00EB400213445970FFF799BD00BF19
:10A1A00010080020034B00EB400213449970FFF7A6
:10A1B0008FBD00BF10080020034B00EB4000184487
:10A1C00090F8B800704700BF58070020034B00EB21
:10A1D0004000184490F90100704700BF10080020AB
:10A1E000024B00EB400018448078704710080020B4
:10A1F000034B03EBC00383F88410FFF71FBD00BFC0
:10A2000058070020034B03EBC00383F88510FFF7CA
:10A2100015BD00BF58070020034B03EBC00383F8B4
:10A220008610FFF70BBD00BF58070020034B03EB60
:10A23000C00383F88710FFF701BD00BF5807002057
:10A24000034B03EBC00383F88810FFF7F7BC00BF94
:10A2500058070020034B03EBC00383F88910FFF776
:10A26000EDBC00BF58070020034B03EBC00383F88D
:10A270008A10FFF7E3BC00BF5807002010B5064B5B
:10A28000044603EBC00383F88B10FFF7D7FC20468E
:10A29000BDE81040FFF71CBD58070020024B03EB40
:10A2A000C00090F88400704758070020024B03EB71
:10A2B000C00090F88500704758070020024B03EB60
:10A2C000C00090F88600704758070020024B03EB4F
:10A2D000C00090F88700704758070020024B03EB3E
:10A2E000C00090F88800704758070020024B03EB2D
:10A2F000C00090F88900704758070020024B03EB1C
:10A30000C00090F88A00704758070020024B03EB0A
:10A31000C00090F88B007047580700202DE9F047E7
:10A320002E4D1E462B1893F8F43004468A4691466B
:10A33000DDF82080099F042B1AD8DFE803F003081A
:10A340000D121700FFF7BAFB2B19012212E0FFF7DD
:10A3500075FC2B1902220DE0FFF712FD2B190322C9
:10A3600008E0FFF7B5FC2B19042203E0FFF73AFCE5
:10A370002B19002205EBC40483F8F42094F88A20FA
:10A38000164B012A13D002D3022A15D021E0BAF1CC
:10A39000000F03D01B689B0C8AF80030B9F1000F46
:10A3A00017D02B68C3F38923A9F8003011E086B1D8
:10A3B0001B689B0A33600CE01EB11B68DB0B5B0162
:10A3C0003360B8F1000F04D02B68C3F3842388F8FE
:10A3D00000300FB12B683B70BDE8F08758070020B4
:10A3E00005280AD8054B0B2101FB0033DA7A043328
:10A3F0001AB90122DA71FFF761BB704758070020D4
:10A4000005280AD8054B0B2101FB0033DA7A043307
:10A410001AB10022DA71FFF751BB704758070020CC
:10A420002DE9F041114AC700D31993F88A60054617
:10A43000032E904604D0032283F88A20FFF7FEFB08
:10A440002846FFF7FBFBD8F80040230344BF6FEA20
:10A4500004346FEA1434032E05D0474487F88A6029
:10A460002846FFF7EBFB2046BDE8F08158070020A7
:10A4700070B50A4C9DF810609DF8145004EBC004B0
:10A4800084F8501084F8512084F8523084F85360D6
:10A4900084F85450BDE87040FFF7A4BB5807002073
:10A4A00006281ED8DFE800F004070B0E12161A006B
:10A4B0000C4B1B6814E00B4BD3F8803010E0094BB9
:10A4C000DB6C0DE0074BD3F8F03009E0054BD3F817
:10A4D000CC3005E0034BD3F8B43001E0014BDB7A1C
:10A4E0000B60704758070020014B1878704700BF79
:10A4F0005408002010B50024064B0022E254064BFD
:10A50000E0B203EB4413997A0134FAF759F8062CB8
:10A51000F2D110BD00130020CC1100202DE9FF471F
:10A520009A4C63784BB96FF000436360A360E360BB
:10A5300023616361A36101236370257F944F4DB94B
:10A54000E8B2F9F798FF78550135082DF8D18F4B0F
:10A5500001221A7727250026F0B2F9F78CFFBB5DA0
:10A5600083421CD08A4B8B4AF05406F1080302EB5D
:10A5700083035B68022B05D0032B0AD0012B0ED17D
:10A5800068B106E058B9844A515D012907D1535595
:10A5900005E0814B5A5D012A04BF02225A5501365B
:10A5A000082E05F10105D7D17C4EF369B3B17C4B80
:10A5B0001D781F4695B9FEF7B1FE7A4B1B68C01A8D
:10A5C000F3690028B8BF4042984207D928460135B0
:10A5D00001F040FB062DF9D101233B70336AC3B172
:10A5E000714B1D781E46A5B9FEF798FE6F4B6B4A5E
:10A5F0001B68126AC01A80EAE073A3EBE07393420F
:10A6000007D92846013501F025FB062DF9D1012394
:10A61000337094F82500664D5C4E05EB40131F7BAC
:10A620006FB1644B002103440093634B0A4603441B
:10A630000193624B03EB8003FFF770FE7AE3FAF7B6
:10A640003DF8D0B93678CEB95FFA86F840465C4F0F
:10A6500000F0E2FF304601F0FDFAF35D3BB105EB9F
:10A660004613997A4046F9F7ABFF0023F3550136BC
:10A67000062EE9D10123237000E0377094F82600FC
:10A6800000F06AFB94F82630404E0133DBB2052B14
:10A6900088BF002386F82630FEF740FEA36AC01A62
:10A6A00080EAE073A3EBE0730A2B07DC454B9A6862
:10A6B0009B685B0602D5170600F13C832378002BCC
:10A6C00040F02B83314B93F82510022988BF0339C2
:10A6D0004FEA411141F00A0194BF00200120C9B2A4
:10A6E00001F04DF9064694F82500052800F2F481A2
:10A6F00001F066FC254B242793F825004FF00C0E43
:10A70000022894BF0023012307FB03F794BF0146EF
:10A71000C11E0EFB01712C4A1144097A61B1242734
:10A720005F43022894BF0146C11E4FF00C0E0EFB82
:10A73000017152F801800CE024275F43022894BF86
:10A740000146C11E4FF00C0E0EFB01710A44D2F8F7
:10A7500004801B4F3A5C032A00F2ED80DFE802F030
:10A76000028A3667002E00F0E68005EB4013D97FA1
:10A7700029B1F9F725FF94F825300322AAE0597A88
:10A78000F9F71EFF94F825300222A3E054080020B8
:10A7900071080020A81200201E13002004000020D1
:10A7A000FE120020F4120020ED100020EC12002018
:10A7B000CC1100200A110020C211002058110020E5
:10A7C00000130020001801407411002086B9B14A1E
:10A7D000125C002A53D102288ABFC11E41014901DF
:10A7E00041F00801C9B2184601F0C9F8002846D066
:10A7F00086EAE672A2EBE672B8F1000FB8BFC8F1C4
:10A800000008424594F8250002D0002E40F08180D7
:10A81000A14B53F830108A4280F0868003EBC003CE
:10A820001979F9F7CDFE9D4B93F8253018E086EAAB
:10A83000E672A2EBE672B8F1000FB8BFC8F10008EB
:10A84000424501D0002E6FD1934B53F830108A420D
:10A8500008D203EBC0031979F9F7B2FE94F825305A
:10A86000012260E005EB4013597AF9F7A9FE94F84C
:10A8700025304CE0002E2FD1864A125CE2B1FEF763
:10A880004DFD94F825304FF00A0E04EB8302526818
:10A89000801A05EB4312918B0028B8BF40420EFB93
:10A8A00001F1884247DD1846917AF9F789FE7B4B22
:10A8B000002293F825300DE002288ABFC11E410115
:10A8C000490141F00801C9B2184601F058F80028C2
:10A8D000D5D001E0FA542EE086EAE673A3EBE673E6
:10A8E000B8F1000FB8BFC8F10008434594F825003F
:10A8F00000D076B9684A52F83020934214D305EB61
:10A900004013597AF9F75CFE644B93F82530022224
:10A9100009E005EB4013D97F31B1F9F751FE5F4BE8
:10A92000032293F82530FA5494F82570FEF7F6FCCC
:10A9300004EB8707786094F82500594B0021034405
:10A940000093584B0A4603440193574BDFF84C8160
:10A9500003EB8003FFF7E2FC94F82500534F05EB6F
:10A9600040139B69002B37D0F9F700FEA0B398F88D
:10A97000250086EAE672A2EBE67207EB40139B69BC
:10A980009A4229D901F066F998F82530484A012100
:10A9900007EB4317D154BB7F4BB994F82530454A98
:10A9A0000F33D15C012917D10221D15414E00027C3
:10A9B00094F8252005EB471305EB4212927F9B7F0D
:10A9C0009A4205D1384601F045F9F8B200F024FE6C
:10A9D0000137062FECD1E0E72EB194F82570364B05
:10A9E000DB5D8BB938E094F82510022988BF033964
:10A9F0004FEA411141F0080194BF00200120C9B283
:10AA000000F0BDFF0028E8D194F8253005EB431293
:10AA1000D28912B9284AD35C23B3FEF77FFC94F89D
:10AA2000253004EB8302D26A05EB4315801AE989CD
:10AA300080EAE072A2EBE0720A2041438A4211DD13
:10AA40001E4DEA5C72B91846FFF7CAFC134B01228F
:10AA500093F82530EA5405E0FEF760FC0F4B03EB5A
:10AA60008707F86294F825000B4D002EB8BF764298
:10AA700055F83030094F9E4222D2FFF777FB97F806
:10AA8000253005EBC3056A79824225D1184600219D
:10AA900020E000BF181300201011002054080020EF
:10AAA0000A110020C211002058110020CC110020F2
:10AAB000BC1100201E1300200C13002012130020D4
:10AAC000FFF754FB97F8253005EBC30569798842F9
:10AAD00002D01846FFF71EFB002000F02CFF94F870
:10AAE0004420C60702F0F802944B48BF42F001022E
:10AAF00045078DF8080083F8442005D594F84430C4
:10AB000043F0020384F84430C00605D594F844307D
:10AB100043F0040384F84430012000F00CFF94F863
:10AB20004420864B02F0C702C10748BF42F008022A
:10AB300083F8442043078DF8090005D594F8443084
:10AB400043F0100384F84430C70605D594F8443028
:10AB500043F0200384F84430794EDFF8F4C1DFF885
:10AB6000F4E1784F784B94F844809CF800109EF8FC
:10AB700000203878357893F80090B246002341FAE7
:10AB800003F6F60713D548FA03F6F6070FD542FA8F
:10AB900003F6F6070BD4012505FA03F6B9F1000F09
:10ABA000F6B246EA000046EA020208BF002101337D
:10ABB000062BE4D194F844303870D8078CF8001094
:10ABC0008EF800208AF800500AD55C4A92F8452099
:10ABD000D10705D45D4AD178012904BF0221D17083
:10ABE0009A0709D594F84520970705D4574A117953
:10ABF000012904BF022111715E0709D594F845208F
:10AC0000550705D4514A5179012904BF02215171D8
:10AC1000180709D594F84520110705D44B4A9179B6
:10AC2000012904BF02219171DA0609D594F8452063
:10AC3000D70605D4454AD179012904BF0221D17133
:10AC40009E0609D594F84520950605D43F4A117A09
:10AC5000012904BF0221117294F8251084F84530AF
:10AC60000323B1FBF3F304AA134413F9083C002BAC
:10AC700053DA022988BF03394FEA411141F0160126
:10AC800094BF0020012003AAC9B200F061FE9DF824
:10AC90000E202A4B12F0400F09D093F825102B48B4
:10ACA00049001B31455C012D04BF022545541006A7
:10ACB0000AD593F8250025490E3011F81050012DC2
:10ACC00004BF022501F81050D10609D593F82510CC
:10ACD0001E4849001B31455C012D04BF0225455427
:10ACE00092060AD593F82510184A0E3112F8110071
:10ACF000012804BF022002F8110093F8251003AACE
:10AD0000022988BF03394FEA411141F0160194BF6F
:10AD100000200120C9B200F047FD94F82520074B20
:10AD20000132D2B2052A88BF002283F82520FEF71F
:10AD3000F5FAA06204B0BDE8F08700BF5408002017
:10AD40004D1300204C110020081100201E1300207C
:10AD500054110020091100202DE9F04FA34E85B0B9
:10AD6000335C0446002B00F04A84022884BFC11ED5
:10AD700049014FEA401794BF0025012594BF47F0D1
:10AD80007C0141F07C01C9B203AA284600F0E0FD35
:10AD9000974B0220DA1992F808809A4618F0400F73
:10ADA0009DF80E1020D084428ABFE21E620052003D
:10ADB00000FA02F2022C4FF0010092BF04FA00FBED
:10ADC000A4F1030B4FEA4B0B00FA0BFBD2B25FFA74
:10ADD0008BFB0A400BEA010BD959D8194942019162
:10ADE0004168C1F100091EE0022C8ABFA4F1030BE7
:10ADF0004FEA440B4FEA4B0B00FA0BFB022C4FF0CF
:10AE0000010092BF04FA00F2E21E520000FA02F2C0
:10AE10005FFA8BFBD2B20BEA010B0A40D919DB595E
:10AE2000D1F804900193022C94BF601CA01CC0B206
:10AE30000092F9F720FB0AEB070191F9081008F0DE
:10AE40003F080029009A03DAD0F1010038BF002042
:10AE500008F1FF31072900F2D283DFE811F0080082
:10AE6000080008000800DB01DB01DB01DB01335DCA
:10AE70000F2B00F2C483DFE813F0C2031000280296
:10AE80005D00650273007C009500BF001301700136
:10AE90007501C203A101B2019B03022C85BFE11E13
:10AEA000490147F0140141F01401C9B203AA284630
:10AEB00000F04EFD022C84BFE11E49019DF80D20DB
:10AEC00094BF47F0060141F006014FEA8409C9B278
:10AED00006EB090328469A6000F051FD022C88BF5A
:10AEE000E11E06EB090318628CBFC9B22146284651
:10AEF000022200F05CFD022C03D847F00607F9B2ED
:10AF000004E0E11E490141F00601C9B2284640F2C1
:10AF1000FF7200F06EFC022C86BFE11EC9B2214612
:10AF200028460322A8F1020800F06DFDB8F1010FD8
:10AF300014D83EE2002A00F06283022C03D847F0C6
:10AF40000207F9B204E0E11E490141F00201C9B271
:10AF5000284600F06FFF274B43F8240004234DE3FD
:10AF6000BBF1000F00F04B83204600F073FE062378
:10AF700044E3022C86BFE11EC9B2214628460322C3
:10AF800000F041FD022C03D847F00807F9B204E0B5
:10AF9000E11E490141F00801C9B228464A4600F0C5
:10AFA00028FC0DE2BBF1000F40F02983022C85BF85
:10AFB000E11E490147F0080141F00801C9B22846E5
:10AFC000002200F016FC022C03D847F00807F9B263
:10AFD00004E0E11E490141F00801C9B22846C9F167
:10AFE000000200F006FC082308E300BF9C080020D4
:10AFF000CC110020F0100020BBF1000F00F0FF8208
:10B00000022C85BFE11E490147F0020141F0020117
:10B01000C9B2284600F00EFF022C85BFE11E49018F
:10B0200047F0080141F00801C9B2804600222846D5
:10B0300000F0DFFBA14B022C53F8242088BFE11E57
:10B04000C8EB020243F824208CBFC9B2214628462F
:10B05000032200F0D8FC022C85BFE11E490147F015
:10B06000060141F00601C9B289EAE972A2EBE97270
:10B07000284600F0BEFB022C83BFE11E4901C9B285
:10B08000F9B22846424600F0C6FB022C86BFE11EFC
:10B09000C9B221462846002200F089FC0923ADE20E
:10B0A000284600F048FC022C4FF0010292BF04FA3F
:10B0B00002F3E31E5B0002FA03F3034200F09F82F7
:10B0C000022C85BFE11E490147F0020141F0020157
:10B0D000C9B2284600F0AEFE022C88BFE11E784BB4
:10B0E0008ABF490147F0080141F00801C9B243F89D
:10B0F00024000022284600F07CFB022C86BFE11EC3
:10B10000C9B221462846022200F051FC022C85BF1C
:10B11000E11E490147F0020141F00201C9B228468F
:10B12000002200F078FB022C85BFE11E4901F9B234
:10B13000C9B228460022A8F1030800F06CFBB8F160
:10B14000010F00F24D82022C86BFE11EC9B22146DA
:10B150002846022200F02BFC72E1BBF1000F40F008
:10B1600095814CE2BBF1000F40F04982022C85BF73
:10B17000E11E490147F0020141F00201C9B228462F
:10B1800000F058FE022C85BFE11E490147F008017E
:10B1900041F00801C9B280460022284600F029FB90
:10B1A000022C88BFE11E4FF0020288BF490198FBC4
:10B1B000F2F294BFF9B2C9B228469DE1284600F0E8
:10B1C000BAFB022C4FF0010292BF04FA02F3E31E15
:10B1D0005B0002FA03F3034240F002820FE2022C0A
:10B1E00003D847F00607F9B204E0E11E490141F037
:10B1F0000601C9B24FEA840806EB08031A6A28461A
:10B2000000F0F7FA022C86BFE11EC9B2214606EB18
:10B210000803EEE1315D0F2900F2F181DFE811F062
:10B22000EF011000520081008F00BF00EF01D2003B
:10B23000EF01EF0122013801F8007901E201C801B4
:10B24000022C85BFE11E490147F0140141F01401B1
:10B25000C9B203AA284600F07BFB022C9DF80D2002
:10B2600088BFE11E06EB84039A608CBFC9B22146F9
:10B270002846022200F09BFB022C03D847F0060769
:10B28000F9B204E0E11E490141F00601C9B22846C5
:10B2900040F2FF7200F0ADFA022C86BFE11EC9B287
:10B2A00021462846032200F0AEFBB8F1060F00F05D
:10B2B0008080B8F1080F7FF451AE7AE0F0100020E2
:10B2C00090120020B8F1060F0ED106EB84039A68A5
:10B2D000022C88BFE11E02F004028CBFC9B22146D5
:10B2E000284642F0010209E0B8F1080F08D1022C0B
:10B2F00086BFE11EC9B221462846032200F083FB27
:10B30000022C03D847F00807F9B204E0E11E490116
:10B3100041F00801C9B22846019A00F06AFA0323F5
:10B320006CE1A8F10503012B04D81AB1B8F1060F9E
:10B3300041D113E6002800F062810C235EE1B8F1F0
:10B34000050F0ED106EB84039A68022C88BFE11E1C
:10B3500002F004028CBFC9B22146284642F0020224
:10B3600009E0B8F1070F08D1022C86BFE11EC9B26F
:10B3700021462846032200F046FB022C03D847F062
:10B380000807F9B204E0E11E490141F00801C9B221
:10B39000019B28465A4200F02CFA05232EE1A8F121
:10B3A0000503012B09D8BBF1000F06D0B8F1050F3A
:10B3B00001D1022322E10F2320E1002800F01F81A8
:10B3C00007231BE1002840F01A81A8F10708B8F113
:10B3D000010F0FD906EB84039A68022C88BFE11E87
:10B3E00002F004028CBFC9B22146284642F0010295
:10B3F00000F009FB022C03D847F00807F9B204E07B
:10B40000E11E490141F00801C9B228464A4625E03B
:10B41000002840F0F480A8F10708B8F1010F0FD917
:10B4200006EB84039A68022C88BFE11E02F0040236
:10B430008CBFC9B22146284642F0020200F0E3FA6E
:10B44000022C03D847F00807F9B204E0E11E4901D5
:10B4500041F00801C9B22846C9F1000200F0C9F95B
:10B460000A23CBE0002800F0CA80022C03D847F062
:10B470000207F9B204E0E11E490141F00201C9B23C
:10B48000284600F0D7FC06EB840398630B23B5E055
:10B49000002840F0B480022C85BFE11E490147F02E
:10B4A000020141F00201C9B2284600F0C3FC022C9F
:10B4B00085BFE11E490147F0060141F006010AEB94
:10B4C00007030022C9B25A73804689EAE972A2EBE7
:10B4D000E972284600F09FF906EB8403022C9B6B6F
:10B4E00084BFE11E490198444FF0020294BFF9B2B3
:10B4F000C9B2284698FBF2F200F08DF9022C86BF03
:10B50000E11EC9B221462846002200F050FA0D2360
:10B5100074E0284600F00FFA022C4FF0010292BFAF
:10B5200004FA02F3E31E5B0002FA03F3034266D05F
:10B53000022C85BFE11E490147F0020141F00201E2
:10B54000C9B20E232846335500F074FC022C88BF84
:10B55000E11E2C4B8ABF490147F0080141F0080168
:10B56000C9B243F824000022284600F042F9022C18
:10B5700086BFE11EC9B221462846022200F017FA12
:10B58000022C85BFE11E490147F0020141F0020192
:10B59000C9B22846002200F03EF9022C85BFE11E08
:10B5A0004901F9B2C9B22846002200F034F926E078
:10B5B000022C86BFE11EC9B221462846022200F0B5
:10B5C000F6F9022C03D847F00807F9B204E0E11EAF
:10B5D000490141F00801C9B22846002200F009F9EA
:10B5E0000E230BE0022C86BFE11EC9B2214606EBFA
:10B5F00084031A7A284600F006FA0023335505B072
:10B60000BDE8F08F90120020024B1A5C0AB90122AB
:10B610001A5470479C080020024B1A5C0AB10F2292
:10B620001A5470479C080020014B185C704700BFFB
:10B630009C080020000000002DE9F04113780F461F
:10B640001446C3F34115064610B10335062D2DD01F
:10B65000504901EB451101F10802107930BBD807C0
:10B6600024D45F2B22D84C48405DF8B913F0970FD3
:10B670001CD1DFF82C8118F8053063B9C97F284642
:10B6800019B1F8F79DFF032303E05178F8F798FF0D
:10B69000022308F80530DFF80C8118F805302BB1CB
:10B6A0002846FEF7ADFE002308F805302178B6B134
:10B6B000012E2BD100220820F9F7AEF838706178FE
:10B6C00000220820F9F7A8F87870A1780022082055
:10B6D000F9F7A2F8B870E1780820324613E0324654
:10B6E0000720F9F799F83870617832460720F9F7A2
:10B6F00093F87870A17832460720F9F78DF8B87082
:10B70000E17807200122F9F787F8F8702378DA0743
:10B710003DD45F2B3BD803F01E02082A12D0142A16
:10B720002BD0062A33D1242256435B090C2202FB7C
:10B730000363A178E278194E42EA012233445A6049
:10B74000BDE8F081242171435B090C2000FB031349
:10B75000A678E578114A45EA0625D550A3781B0757
:10B7600015D52678760900FB061693596FEA035320
:10B770006FEA13539351BDE8F08124214E435B09D6
:10B780000C2101FB0363054EE27833441A72BDE8D5
:10B79000F08100BFCC1100200C1300207411002098
:10B7A000001300201213002007B513788DF8001045
:10B7B0008DF80130537801A98DF8023093786A46EC
:10B7C0008DF80330FFF738FF03B05DF804FB07B5D1
:10B7D0008DF802309DF810308DF800108DF80120A2
:10B7E00001A96A468DF80330FFF726FF03B05DF824
:10B7F00004FB07B500238DF800108DF801308DF89B
:10B800000320131201A96A468DF80230FFF714FFD6
:10B8100003B05DF804FB5F292DE9F34105460E46B0
:10B82000144658D811F01E07C1F3411202D0022F5E
:10B830001DD050E000EB40031A4430491201881833
:10B8400043688C50C3EB040EBEF1000FB8BFCEF1BD
:10B85000000EBEF5000F08DB9C42CCBF284C294CE3
:10B860000A441C440123137335E0077333E000EBF3
:10B870004007224B17443F01D91924F07F4EC1F8ED
:10B8800008E04C6001F10800D9599846C4EB010E5C
:10B89000BEF1000FB8BFCEF1000EBEF5000F18DBF1
:10B8A000A142CCBF164B174B520123448DF8002008
:10B8B0001A148DF801201A128DF80220284601A9C9
:10B8C0006A468DF803304744FFF7B6FE01233B7309
:10B8D00001E00023037123148DF801302846231260
:10B8E00001A96A468DF800608DF802308DF803409A
:10B8F000FFF7A2FE02B0BDE8F08100BF24150020D2
:10B90000FFFF7F00010080FF07B511F01C0202D18C
:10B91000FFF781FF0CE000238DF800106A4601A9B3
:10B920008DF801308DF802308DF80330FFF784FE7A
:10B9300003B05DF804FB014618B1012806D10820C8
:10B9400001E0072001210A46F8F766BF0020704792
:10B9500013B541F0010114468DF8041001AA69469F
:10B96000FFF76AFE9DF801309DF8000023709DF8F6
:10B97000023063709DF80330A37002B010BD07B5AC
:10B9800041F001018DF8041001AA6946FFF754FE49
:10B990009DF803309DF8020043EA0020030544BFF0
:10B9A0006FEA00506FEA105003B05DF804FB73B506
:10B9B00002298ABFCB1E4B015B0143F015030C46E5
:10B9C0001646DBB201A96A4605468DF80030FFF73E
:10B9D00033FE022C9DF8053088BF033C64018DF8CE
:10B9E000013044F014049DF80630E4B2284601A961
:10B9F0006A468DF800408DF802308DF80360FFF73D
:10BA00001BFE02B070BD73B502298ABFCB1E4B016D
:10BA10005B0143F015030C461646DBB201A96A46EA
:10BA200005468DF80030FFF707FE022C9DF8053023
:10BA300088BF033C64018DF8013044F014049DF884
:10BA40000730E4B2284601A96A468DF800408DF817
:10BA500002608DF80330FFF7EFFD02B070BD2DE9F5
:10BA6000F74F0228C1F30A078ABFC11E41014901ED
:10BA700094BF4FF000084FF0010841F0180106464E
:10BA8000C9B2404601AAFFF763FF9DF8059038460A
:10BA90004FEA191A09F00F09D1450FDB04F0A4FC95
:10BAA000CAEB09090446012000FA09F00D4604F02A
:10BAB000ABFC00223A4B04F00DFD10E004F094FCC6
:10BAC000C9EB0A090446012000FA09F00D4604F00A
:10BAD0009BFC02460B460020314904F025FE02463D
:10BAE0000B462046294604F01FFE04F02DFF04F00B
:10BAF0009DFC29A3D3E9002304F0ECFC04F024FF0F
:10BB000004F094FC0022274B04F0E4FC4FF0FF3AD1
:10BB100004460D46D3464FF00009012000FA09F013
:10BB200004F072FC0B4602462946204604F0D2FC83
:10BB300004F0E2FEA0F18003802B38BFCA4609F171
:10BB4000010928BF5846B9F10E0F01D08346E4E73A
:10BB5000022E8ABFF11E7101490141F01201C9B2E2
:10BB600000238DF8050001AA40468DF804308DF8B9
:10BB700006A0FFF719FE022E8ABFF11E71014901CE
:10BB800041F00C014046C9B23A46FFF732FE0020B0
:10BB900003B0BDE8F08F00BF04560E2DB29DEF3FFD
:10BBA000000060400000204073B54D0805EB4505DE
:10BBB000B42305F5807503FB0055044628460E4660
:10BBC000FCF72CFE8DF80400681CFCF727FE8DF8AE
:10BBD0000500A81CFCF722FE022C8DF8060094BF7D
:10BBE0000020012002D86401E1B202E0E11E490117
:10BBF000C9B2314301AAFFF7D7FD02B070BD37B516
:10BC0000022804460D468ABFE11E61014901C9B2FE
:10BC100041EA05014FEA550594BF0020012001AA21
:10BC200005EB4505FFF794FE05F58075B42303FB8E
:10BC300004549DF804102046FCF717FD601C9DF885
:10BC40000510FCF712FDA01C9DF80610FCF70DFD79
:10BC500003B030BD022888BFC11E38B594BF00258F
:10BC60000125044694BFC1B2C9B228460222FFF79B
:10BC70009EFE022C8ABFE11E6101490141F00801CC
:10BC8000C9B22846FFF740FE022C8ABFE11E6101BF
:10BC9000490141F00A012846C9B2BDE83840FFF722
:10BCA00033BE73B502280E468ABFC11E4101490149
:10BCB00094BF0025012541F016010446C9B201AA2E
:10BCC0002846FFF745FE9DF8053016F0010F14BF1A
:10BCD00043F0400323F040038DF805309DF8053014
:10BCE00016F0020F14BF43F0100323F01003022CD0
:10BCF0008ABFE11E6101490141F016018DF805304E
:10BD0000C9B20023284601AA8DF80630FFF74CFD82
:10BD100002B070BD73B502280E468ABFC11E410134
:10BD2000490194BF0025012541F016010446C9B21E
:10BD300001AA2846FFF70CFE9DF8053016F0010F0A
:10BD400014BF63F07F0303F07F038DF805309DF887
:10BD5000053016F0020F14BF43F0200323F0200338
:10BD6000022C8ABFE11E6101490141F016018DF8E4
:10BD70000530C9B20023284601AA8DF80630FFF726
:10BD800013FD02B070BD07B502288ABFC11E410174
:10BD9000490194BF0023012341F01601C9B218469E
:10BDA00001AAFFF7D5FD9DF80530C3F38010DB062F
:10BDB00048BF40F0020003B05DF804FB07B502285D
:10BDC0008ABFC11E4101490194BF0023012341F0F4
:10BDD0001601C9B2184601AAFFF7BAFD9DF8053051
:10BDE000D8099B0648BF40F0020003B05DF804FB91
:10BDF00070B50F4C000123189A68914209DD8A1A28
:10BE0000C2F18075AA425E6801DC324409E0751B0C
:10BE10000AE00ADA521AC2F18075AA425E6802DCB0
:10BE2000B21A5A6001E035445D602044816070BD03
:10BE30002415002037B541F001030C4601AA6946DC
:10BE40008DF804300546FFF7F7FB9DF802309DF8AA
:10BE500001201B0243EA02439DF8032043EA02014A
:10BE60000B0248BF41F07F415F2C19D8C4F3411247
:10BE700014F01E040ED0022C12D105EB450515441A
:10BE8000E8B221F07F41FFF7B3FF074B03EB051545
:10BE9000696805E005EB45052A44034B12019958F2
:10BEA000084603B030BD00BF2415002038B50C464D
:10BEB00068210546FFF7BEFF14B140F0010201E022
:10BEC00020F0010228466821BDE83840FFF7A3BCF6
:10BED00038B50C4668210546FFF7ACFF14B140F0B9
:10BEE000100201E020F0100228466821BDE8384029
:10BEF000FFF791BC73B5314C40F22312637E0020F2
:10BF000013F0010F94F8283008BF4FF49172D9074D
:10BF100048BF42F010026821FFF77DFC0020022399
:10BF2000024600937E210346FFF751FC637E40F2F8
:10BF3000231213F0020F94F8283008BF4FF49172C7
:10BF40009B0748BF42F0100201206821FFF763FC05
:10BF500002230022009301207E211346FFF737FCC5
:10BF600000240026E5B2F1B228460136FFF71CFE98
:10BF70001D2EF7D1022C8ABFE91E6901490194BF29
:10BF80000026012641F00C01C9B23046FFF752FFEE
:10BF900001462846FFF763FD022C8ABFE91E6901AE
:10BFA000490141F01601C9B2304643F2FF12013493
:10BFB000FFF71FFC062CD4D102B070BD0400002096
:10BFC000F0B502288ABFC31E43015B01022885B079
:10BFD00094BF0025012543F003030446DBB203AA06
:10BFE000284602A98DF80C30FFF726FB9DF80A10B1
:10BFF0009DF80930090241EA03419DF80B302046C3
:10C000001943FFF7F5FE1C4A2301D118097B0029CB
:10C0100030D024206843022C8CBFE11E21460C2620
:10C0200006FB010115480144097A19BBD018D658FE
:10C030004268B71A002FB8BF7F42B7F5000F05DB83
:10C040009642CCBF0E4B0F4B134402E00A4A0173D9
:10C05000D358022C02D86401E1B202E0E11E49018A
:10C06000C9B2DAB200922846C3F30742C3F30723EA
:10C07000FFF7ADFB05B0F0BD2415002074110020C2
:10C08000FFFF7F00010080FF074B10B518681C46BA
:10C0900001460A780B4601311AB12C2AF9D1002247
:10C0A0001A700133236010BDEC08002070B5124BEC
:10C0B00006461B78E3B1FCF7A3FD104C054618B10A
:10C0C00000232371012070BDA368E268934207D268
:10C0D0005A1C23441B7C012033702071A26070BD68
:10C0E00004F11000FDF74EFCA560E060284670BD2D
:10C0F000BDE87040FCF784BDEC100020EC08002087
:10C1000010B50E4B1B7813B10D4C23791BB9BDE84C
:10C110001040FCF75BBD226D0D2802F101032244A3
:10C12000236582F8540002D03F2B00D829B9194664
:10C130000448FDF759FC0023236510BDEC100020D6
:10C14000EC0800204009002070B50121044686B0AB
:10C150002020FFF7D5FF002C04DA2D200121FFF766
:10C16000CFFF644200230A2194FBF1F201FB12414C
:10C1700001AE30311D46995514460133002AF2D1E3
:10C18000705D0121FFF7BCFF15F1FF35F8D206B055
:10C1900070BD2DE9F34105460DF10700FFF786FF5D
:10C1A000974C002800F0C88094F894309DF8070060
:10C1B000944E03BB7378403398420DD1D4F8983035
:10C1C000002B40F0B9803179012331F0010184F86E
:10C1D000943040F0B180ADE00D2801D01B2801D192
:10C1E000002305E0D4F898307E2B00F2A5800133BF
:10C1F000C4F89830A0E0317931F0010101D1FFF7A6
:10C200007FFF9DF807301F2B0CD9D4F898207C496C
:10C210007E2A00F28280501C0A44C1F8980082F8FD
:10C220009C307AE0082B08D1D4F89830002B74D0D9
:10C23000734A013BC2F898306FE00D2B6DD1D4F8F2
:10C240009830002B69D03379112B16D16D4B012119
:10C25000587800274030C0B2FFF752FFD4F898302A
:10C260009F4206D2684B0121D85DFFF749FF013795
:10C27000F4E70D200121FFF743FF0023D4F8988055
:10C280002768C4F81C311A461946424537D001299F
:10C2900011D002D3022925D02FE0DFF864C10CF1C0
:10C2A0009C00105C202828D00CEB030181F82001B1
:10C2B0000133012121E0524800F19C0C12F80CC01E
:10C2C000BCF1200F0AD1012B04D91844002180F8B9
:10C2D000201101334D4F02211F440EE0184480F815
:10C2E00020C109E0DFF818C10CF19C00105C202887
:10C2F00003D09C448CF8200101330132C5E70022B1
:10C30000C4F81C31234483F820210123276084F8DA
:10C310009F3184F89420C4F898209DF807301B2B97
:10C320000AD133790021012BC4F8981084F89410B5
:10C3300002D10D20FFF7E4FE94F89F0100260028AB
:10C340005AD02F4B83F89F61F7B2DFF8DC80C7EB40
:10C35000C70708EB07042D48214604F039FF28B928
:10C36000A6796379F1072B7036D506E018F8073007
:10C370000136002BE8D12B703DE0FFF785FE2B78CE
:10C380000446042B14D1224904F022FF08B90023EB
:10C390000CE020461F4904F01BFF08B9012305E00B
:10C3A0001D49204604F014FF90B902236B7013E07E
:10C3B0000D2B0ED1194904F00BFF0028E7D02046C1
:10C3C000174904F005FF0028E8D020461549E9E7A1
:10C3D000204604F0F9FE6870B20704D5FFF754FE5A
:10C3E00004F0F2FEA870730705D5FFF74DFE04F0C8
:10C3F000EBFEC5F80300012002B0BDE8F08100BFEC
:10C40000EC08002004000020880900200C0A00200D
:10C410004C15010850150108541501085A1501085A
:10C4200060150108651501084714010838B50D4D60
:10C430000446A87801214030C0B2FFF761FE687859
:10C4400001214030C0B2FFF75BFE2078FFF77CFE91
:10C450006068FFF779FEBDE838400D200121FFF745
:10C460004FBE00BF040000207047FEE7FEE7FEE776
:10C47000FEE77047704770477047704770477047D6
:10C4800070477047704770477047704770477047F4
:10C49000704770477047704770477047704708B5DE
:10C4A000014B1B68984708BD5011002008B5024B8E
:10C4B0001B68984708BD00BF0813002008B5024B51
:10C4C0001B68984708BD00BFC811002008B5024B83
:10C4D0001B68984708BD00BF8C120020704770474A
:10C4E0007047704770477047704770477047704794
:10C4F0007047704770477047704770477047704784
:10C500007047704770477047704770477047704773
:10C510007047704770477047704770477047704763
:10C5200070477047704700BF08B5144B98420FD052
:10C5300003F5A053984213D0A3F5C05398421BD1E2
:10C540004FF40070012101F0FBFB4FF400700EE08E
:10C550004FF48060012101F0F3FB4FF4806006E0AE
:10C560004FF40040012101F0EBFB4FF400400021AB
:10C57000BDE8084001F0E4BB08BD00BF0028014051
:10C5800043680A6823F4702323F4807313430A7901
:10C5900010B543EA022343608A68CB6884681A4373
:10C5A000084B234013434A7943EA420383600B7CE0
:10C5B000C26A013B22F47002DBB242EA0353C36257
:10C5C00010BD00BFFDF7F1FF00230360037143714D
:10C5D0008360C360012303747047836811B143F023
:10C5E000010301E023F0010383607047836811B108
:10C5F00043F4807301E023F4807383607047C9B211
:10C6000043680AB1194301E023EA01014160704720
:10C61000836843F00803836070478068C0F3C000FC
:10C620007047836843F00403836070478068C0F3F9
:10C6300080007047836811B143F4A00301E023F444
:10C64000A003836070478068C0F3805070474368E0
:10C65000013923F4604343EA413343607047436840
:10C6600011B143F4006301E023F4006343607047B9
:10C67000092970B50DD9A1F10A0404EB440407257A
:10C68000A540A340C66826EA050545EA0304C46040
:10C690000BE001EB41040725A54003FA04F4066909
:10C6A00026EA050545EA04030361062A0CD8013A87
:10C6B00002EB82021F23934001FA02F2446B24EA48
:10C6C00003031A43426370BD0C2A0CD8073A02EBED
:10C6D00082021F23934001FA02F2046B24EA03034F
:10C6E0001A43026370BD0D3A02EB82021F2393408E
:10C6F00001FA02F2C46A24EA03031A43C26270BD5B
:10C70000836811B143F4801301E023F48013836044
:10C710007047C06C80B27047014B1868704700BF0B
:10C720004C240140436811B143F4806301E023F4D9
:10C73000806343607047436811B143F4805301E064
:10C7400023F4805343607047836823F4E043194324
:10C7500081607047836811B143F4004301E023F422
:10C76000004383607047836811B143F4021301E012
:10C7700023F40213836070478068C0F34050704711
:10C78000092970B50DD9A1F10A0404EB4404072569
:10C79000A540A340C66826EA050545EA0304C4602F
:10C7A0000BE001EB41040725A54003FA04F40669F8
:10C7B00026EA050545EA04030361846B931CC4F370
:10C7C00001555B1BDBB203EB83031F229A409940A8
:10C7D00024EA020444EA0103836370BD836B0139D8
:10C7E00023F4401343EA0153836370474250704778
:10C7F0002831405880B27047436823F4400323F443
:10C800000073194341607047416282627047436818
:10C8100023F01F03194341607047054B9A6810B11C
:10C8200042F4000201E022F400029A60704700BF67
:10C8300000240140036819420CBF0020012070470A
:10C84000C943016070474368006810EA112004D0B2
:10C85000C9B219420CBF0020012070476FEA1121B4
:10C860000160704708B54FF00070012101F074FAC3
:10C87000BDE808404FF00070002101F06DBA2E4B6A
:10C8800001221A605A6812F0010252D00278012A7D
:10C890001A680CBF42F0800222F080021A604378CE
:10C8A000012B254B1A680CBF42F0400222F04002D7
:10C8B0001A608278012A1A680CBF42F0200222F026
:10C8C00020021A60C378012B1B4B1A680CBF42F080
:10C8D000100222F010021A600279012A1A680CBFB5
:10C8E00042F0080222F008021A604379012B124B31
:10C8F0001A680CBF42F0040222F004021A60827926
:10C90000C379920742EA0362037A42EA0342437A16
:10C9100042EA03524389013B1A43074BDA611A6822
:10C9200022F001021A60586800F0010080F0010056
:10C9300070471046704700BF006400400378012133
:10C940009940354B70B5D3F8002289B242F001020C
:10C95000C3F80022D3F81C22CC432240C3F81C2287
:10C960008278A2B9D3F80C2246892240C3F80C225F
:10C970000278C588483245EA064543F83250838834
:10C980000289057843EA0242244BED005A5183782C
:10C99000012B15D1204B8688D3F80C22C5880A4379
:10C9A000C3F80C22027845EA0645483243F8325073
:10C9B00043890289057843EA0242184BED005A5137
:10C9C0004378154A1BB9D2F80432234002E0D2F86A
:10C9D00004320B438589C2F804320F4B2DB9D2F8CB
:10C9E00014522C40C2F8144206E0012D04D1D3F8B1
:10C9F00014220A43C3F81422827B012A04D1D3F8FB
:10CA00001C221143C3F81C12D3F8002222F00102A9
:10CA1000C3F8002270BD00BF0064004044660040BF
:10CA20000023037043708370C3700371437183717B
:10CA3000C3710323037202234372012343817047AE
:10CA4000044B5A6909B1104301E022EA0000586121
:10CA5000704700BF00640040334A03469168F0B558
:10CA6000480107D49168090106D49268D20005D420
:10CA70000420F0BD002002E0012000E002200101BE
:10CA800001F1804202F5C842D2F8804104F001046D
:10CA9000C2F880411C7A5D7A3CB91E6876051E603A
:10CAA000D2F8804125432E4307E05E682C43F60010
:10CAB0005E60D2F8807126433E43C2F880619C7A62
:10CAC00001F1804104F00F049C72D2F8844101F519
:10CAD000C84124F00F04C2F884419D7AD2F8844101
:10CAE0002C43C2F884415D7B9C7B2D0445EA0465A0
:10CAF000DC7A25431C7B45EA0425C1F8885101F501
:10CB0000C474597C9D7C090441EA0561DD7B1B7C72
:10CB1000294341EA03236360D2F8803143F00103E3
:10CB2000C2F88031F0BD00BF0064004001281DD074
:10CB30000FD3022829D1174A9368916803F48033F0
:10CB4000926801F400319B0B43EA1143C2F3007277
:10CB500019E0104A91689368926801F0010103F0AE
:10CB6000020343EA8103C2F380620CE0094A93683E
:10CB7000916803F48073926801F400719B0943EAA1
:10CB80001123C2F3C062134300E00023024AD05CC9
:10CB9000704700BF0064004027150108012808D035
:10CBA00002D302280AD07047074B9A6842F08002ED
:10CBB00008E0054B9A6842F4004203E0024B9A6891
:10CBC00042F400029A60704700640040034B202248
:10CBD00008B9DA6070471A61704700BF006400400E
:10CBE00010B9064BD86803E0012804D1034B18693B
:10CBF00000F0030070470020704700BF0064004051
:10CC0000020102F1804303F5C84310B5D3F8B041E7
:10CC100004F00404E4B20C7224B9D3F8B041640DFA
:10CC20000C6003E0D3F8B041E4084C60D3F8B041A5
:10CC300004F002044C72D3F8B44104F00F048C7277
:10CC4000D3F8B4311B0ACB7402F1804303F5C84317
:10CC5000D3F8B84103F5DC72CC72D3F8B841240A9A
:10CC60000C73D3F8B841240C4C73D3F8B831BDE839
:10CC700010401B0E8B735368CB7353681B0A0B74E5
:10CC800053681B0C4B7453681B0E8B74FFF79EBFCD
:10CC9000044B1A6842F002021A601868C0F34000A0
:10CCA000704700BF00640040054B1A6822F0020282
:10CCB0001A60186880F00200C0F34000704700BF9F
:10CCC00000640040034B9B6918420CBF0020012008
:10CCD000704700BF00640040024B9A6922EA0000DE
:10CCE0009861704700640040202838D010D806288A
:10CCF00028D006D804282FD0052848D1254B98687D
:10CD000033E0072823D0082841D1224BD86836E0E9
:10CD1000B0F5007F2CD007D8402823D0B0F5807F15
:10CD200035D11C4B986920E0B0F5803F2AD0B0F592
:10CD3000003F22D0B0F5806F29D1164B9869C0F31F
:10CD400080007047134B9868C0F300207047114B68
:10CD50009868C0F3004070470E4BD86814E00D4B44
:10CD6000186911E00B4B186909E000F001007047E9
:10CD7000084B9869C0F340007047064B5868C0F3F1
:10CD800000107047034B5868C0F3C0007047002084
:10CD9000704700BF00640040202835D00CD806281A
:10CDA00024D004D8042829D005281DD0704707288E
:10CDB00021D0082824D07047B0F5007F2FD005D8A7
:10CDC000402823D0B0F5807F24D07047B0F5803F55
:10CDD0002BD0B0F5003F2AD0B0F5806F2AD1164B8A
:10CDE0009A6922F004021EE0012201E04FF48072F1
:10CDF000114B9A6070474FF48032F9E7082200E047
:10CE000010220D4BDA607047082200E010220A4B16
:10CE10001A617047084B9A6922F0010203E0064B41
:10CE20009A6922F002029A617047082200E01022FB
:10CE3000014B5A60704700BF00640040036823F054
:10CE4000010303600023036043608360C3602D4BD4
:10CE5000984234D011D83C3B98422AD006D8283B7F
:10CE6000984222D01433984221D07047264B9842E2
:10CE700021D01433984220D07047244B98422DD0B3
:10CE800008D8A3F5677398421ED003F562739842E1
:10CE90001FD070471E4B984229D0143398422BD094
:10CEA000283B98422DD11B4B1DE01B4B12E01A4B27
:10CEB00015E0194B17E0184B1AE0174B1DE0164B05
:10CEC0005A6842F470021BE0134B5A6842F07062D9
:10CED00016E0104B5A6842F00F0211E00D4B5A68F1
:10CEE00042F0F0020CE05A6842F4706208E0094B2C
:10CEF0005A6842F4704203E0064B5A6842F47022CA
:10CF00005A6070476C000240440002401C0402401A
:10CF10004404024000040240000002408A6810B548
:10CF20000C6A036814430A6923F4FF4314434A69F3
:10CF300023F0700314438A691443CA6914434A6A8C
:10CF400014438A6A224313430360CB6843600B682F
:10CF500083604B68C36010BD00230360436083603F
:10CF6000C360036143618361C3610362436283629F
:10CF70007047036811B143F0010301E023F001039E
:10CF80000360704703680AB1194301E023EA010115
:10CF900001607047406880B27047C3004CBF044BCB
:10CFA000044B1B6803420CBF00200120704700BFE8
:10CFB0000004024000000240C3004CBF014B024B82
:10CFC000586070470004024000000240C3004CBF9C
:10CFD000034B044B1B6803420CBF00200120704729
:10CFE0000004024000000240C3004CBF014B024B52
:10CFF000586070470004024000000240044B0022C9
:10D000001A605A609A60DA60024A5A61704700BF3B
:10D0100000040140FFFF0700837930B50168027901
:10D0200043B3194BCC431D6802F1804225401D607B
:10D030005D6802F582322C405C6014682143116007
:10D0400002689C68D1430C409C60DC682140D96038
:10D050004179102906D1996811439960D9680A432A
:10D06000DA6030BD01F1804303F5823319680A4369
:10D070001A6030BD02F1804303F582331A6822EA58
:10D080000101196030BD00BF0004014000230C22E3
:10D0900003600371427183717047024B1A69104338
:10D0A0001861704700040140034B5B6918420CBFD4
:10D0B00000200120704700BF00040140014B58616F
:10D0C000704700BF00040140054B1A685B690340CC
:10D0D00004D010420CBF0020012070471846704752
:10D0E00000040140014B5861704700BF000401403B
:10D0F000044B1A6802F038021A601A68104318606C
:10D10000704700BF00200240044B1A6822F008025A
:10D110001A601A6810431860704700BF0020024070
:10D12000044B1A6822F010021A601A681043186043
:10D13000704700BF00200240034B044A5A6002F1CE
:10D1400088325A60704700BF0020024023016745C3
:10D15000024B1A6942F080021A61704700200240B7
:10D16000014BD8698008704700200240014B186AC3
:10D17000704700BF00200240024BD869C0F3400056
:10D18000704700BF00200240024B1868C0F34010F7
:10D19000704700BF00200240044B1A6909B11043D8
:10D1A00001E022EA00001861704700BF0020024041
:10D1B0000128064B03D1D86900F001007047DB68F5
:10D1C00018420CBF00200120704700BF0020024021
:10D1D000014BD860704700BF00200240084BDA685E
:10D1E000D10709D4DA68520708D4DB6813F0100FAE
:10D1F0000CBF0420032070470120704702207047B5
:10D200000020024013B50446FFF7E8FF01280FD1C4
:10D2100064B100230193FF230193019B13B1019B90
:10D22000013BF9E7FFF7DAFF013CEFE7052002E0F9
:10D23000002C08BF052002B010BD38B5054640F6E9
:10D24000FF70FFF7DFFF042814D10B4C40F6FF708E
:10D25000236943F0020323616561236943F04003BE
:10D260002361FFF7CFFF012804D0226941F6FD7347
:10D270001340236138BD00BF0020024010B540F6C6
:10D28000FF70FFF7BFFF042813D10A4C40F6FF7070
:10D29000236943F004032361236943F040032361BE
:10D2A000FFF7B0FF012804D0226941F6FB73134059
:10D2B000236110BD0020024010B540F6FF70FFF75B
:10D2C000A1FF042829D1154C154B40F6FF70A3602F
:10D2D00003F18833A360236943F0200323612369AA
:10D2E00043F040032361FFF78DFF04280ED122692C
:10D2F00041F6DF73134023612369A52243F0100335
:10D300002361084B0F201A80FFF77CFF012804D00F
:10D31000226941F6EF731340236110BD00200240E3
:10D320002301674500F8FF1F70B505460F200E4624
:10D33000FFF768FF042817D10C4C0F20236943F036
:10D3400001032361B3B22B80FFF75CFF042804D1F3
:10D35000360C6E800F20FFF755FF012804D022699C
:10D3600041F6FE731340236170BD00BF00200240F0
:10D3700070B505460F200E46FFF744FF04280FD175
:10D38000084C0F20236943F0010323612E80FFF72F
:10D3900039FF012804D0226941F6FE73134023614E
:10D3A00070BD00BF0020024070B505460F200E463C
:10D3B000FFF728FF042814D10A4C0B4B0F20A36061
:10D3C00003F18833A360236943F0100323612E80A7
:10D3D000FFF718FF012804D0226941F6EF731340CC
:10D3E000236170BD002002402301674510B504464B
:10D3F0000F20FFF707FF04283ED1204B2049E443CC
:10D40000996001F1883199601969E2B241F0100127
:10D41000FF2A196104D1C4F30723FF2B08D10EE0C2
:10D42000184B0F201A81FFF7EDFE04281CD1F2E7FC
:10D43000144A0F205381FFF7E5FE042814D1C4F3EA
:10D440000743FF2B06D00F4A0F209381FFF7DAFE28
:10D45000042809D1240EFF2C01D1042006E0094B39
:10D460000F20DC81FFF7CEFE012805D0034A41F6EC
:10D47000EF7311690B40136110BD00BF0020024023
:10D480002301674500F8FF1F38B5054640F6FF70D9
:10D49000FFF7B8FE042836D11B4C1C4B40F6FF703A
:10D4A000A36003F18833A360236943F02003236161
:10D4B000236943F040032361FFF7A4FE04281BD136
:10D4C000226941F6DF7313402361236943F010039F
:10D4D00023610F4B0DB1002200E0A5221A8040F617
:10D4E000FF70FFF78FFE01280DD0074A41F6EF735A
:10D4F00011690B40136138BD012804D0226941F63F
:10D50000DF731340236138BD0020024023016745CB
:10D5100000F8FF1FF8B5114C114B0546A36003F14D
:10D520008833A3600F200E461746FFF76BFE0428D2
:10D5300013D1236947F0F80743F0100323613E43FA
:10D54000084B35435D800F20FFF75CFE012804D0B7
:10D55000226941F6EF7313402361F8BD00200240B9
:10D560002301674500F8FF1F08B5264B98422FD0CE
:10D5700011D8A3F5006398421ED003F5806398424A
:10D5800020D0A3F5006398423AD10420012100F095
:10D59000D7FB04202FE01C4B98421FD003F580637B
:10D5A000984221D0A3F50063984229D1402001215F
:10D5B00000F0C6FB40201EE00820012100F0C0FB67
:10D5C000082018E01020012100F0BAFB102012E022
:10D5D0002020012100F0B4FB20200CE0802001215C
:10D5E00000F0AEFB802006E04FF48070012100F0D7
:10D5F000A7FB4FF480700021BDE8084000F0A0BBFD
:10D6000008BD00BF00140140001C014008B5012006
:10D61000014600F095FBBDE808400120002100F024
:10D620008FBBCB78F0B5DA0648BF8A78098803F05B
:10D630000F0548BF154311F0FF0F1DD004680022ED
:10D640000127974007EA0106BE4211D197004FF02B
:10D650000F0C0CFA07FC05FA07F724EA0C04282B38
:10D6600044EA070401D1466102E0482B08BF066185
:10D670000132082AE4D10460FF291FD9446800223E
:10D6800002F108060127B74007EA0106BE4211D1A0
:10D6900097004FF00F0C0CFA07FC05FA07F724EA85
:10D6A0000C04282B44EA070401D1466102E0482B10
:10D6B00008BF06610132082AE2D14460F0BD4FF68E
:10D6C000FF730380022383700423C3707047836851
:10D6D00019420CBF002001207047806880B270475B
:10D6E000C36819420CBF002001207047C06880B297
:10D6F000704701617047416170470AB1016170472D
:10D7000041617047C160704741F48033836181613A
:10D710008361836983697047054B1A6822F07F0231
:10D720001204120C114341EA00101860704700BF48
:10D7300000000140014B1860704700BF1C002042F0
:10D7400030B5134A00F44015B5F5401F536884B254
:10D7500006D1556823F0706325F0706555600FE0C1
:10D76000C20205D5C0F30342032505FA02F203E025
:10D77000420D120104FA02F223EA020343F070633D
:10D7800019B1400D000184402343014A536030BD6C
:10D790000000014001F003039B000F229A409840D3
:10D7A00001F0FC0101F1804101F5803110B58C6878
:10D7B00024EA02028A608A6802438A6010BD00BFC0
:10D7C0000B4B6FF070424FF0FF31C3F88010C3F87D
:10D7D0008420C3F88011C3F88421002202F1C00123
:10D7E000013200200F2A43F82100F7D1704700BF13
:10D7F00000E100E0094B4FF0206209495A60002225
:10D800009A60D9601A615A619A61DA611A625A6241
:10D810004FF0FF329A62DA621A63704700ED00E05F
:10D820000000FA0540F0BF60024B40F40030D860C1
:10D83000704700BF00ED00E0C27830B503785AB3FE
:10D840001B4A4478D2688578D243C2F30222C2F1DF
:10D85000040104FA01F10F24D4402C400C4303F0DE
:10D860000301C9002401FF228C408A4003F0FC031D
:10D8700003F1604303F56143D3F8005325EA020145
:10D8800022400A43C3F8002303780122590903F018
:10D890001F0302FA03F306E05909012203F01F03F4
:10D8A00002FA03F32031034A42F8213030BD00BFB1
:10D8B00000ED00E000E100E000230370437083709E
:10D8C000C3707047F6F749BCF6F749BCF6F749BC98
:10D8D000F6F749BC0001F6F748BCF6F749BC024B25
:10D8E0005868C0F30930704700ED00E000F01F03F6
:10D8F000012202FA03F34009044A403052F82000A2
:10D900001840C31A58425841704700BF00E100E078
:10D91000014B1860704700BF00EF00E0420901238F
:10D9200000F01F0003FA00F0024B603243F82200BF
:10D93000704700BF00E100E0024B5868C0F30900E7
:10D94000704700BF00ED00E000F01F03012202FA63
:10D9500003F34009044A803052F820001840C31AEB
:10D9600058425841704700BF00E100E0014B186881
:10D97000704700BF00ED00E021F0604121F07F0121
:10D98000014B08439860704700ED00E0014A024BEC
:10D99000DA6070470400FA0500ED00E0014A024B2E
:10D9A000DA6070470100FA0500ED00E0044B1A69E7
:10D9B00009B1104301E022EA00001861704700BF7E
:10D9C00000ED00E0012300F01F0003FA00F0044B1B
:10D9D0005A6A09B1104301E022EA00005862704718
:10D9E00000ED00E0114B30B5DB68DB43C3F30223ED
:10D9F000C3F10404A140FF2424FA03F31A401143A5
:10DA0000C0F30122D2009440090101FA02F2C0F3EE
:10DA10008110800000F1604000F56D40836923EAC9
:10DA20000404846185692A43826130BD00ED00E011
:10DA3000C0F3832001238340034A506A1840C31A6D
:10DA400058425841704700BF00ED00E000F01F0051
:10DA5000012101FA00F0024B5A6802435A607047F4
:10DA600000ED00E000F01F00411E012000FA01F16E
:10DA7000024B5A680A435A60704700BF00ED00E04D
:10DA8000C0F3833001238340034A506A1840C31A0D
:10DA900058425841704700BF00ED00E0C0F381429A
:10DAA000094B0AB9D86A7047012A0AD1C0F301525A
:10DAB000986AD300D840022A14BF00F00F00C0B209
:10DAC0007047186B704700BF00ED00E0034B10F487
:10DAD000800F0CBF586B986B704700BF00ED00E0E3
:10DAE0000C4B1A6842F001021A6059680A4A0A404F
:10DAF0005A601A6822F0847222F480321A601A681E
:10DB000022F480221A605A6822F4FE025A6000222F
:10DB10009A607047001002400000FFF80C4BB0F50F
:10DB2000803F1A6822F480321A601A6822F4802238
:10DB30001A6003D0B0F5802F04D070471A6842F401
:10DB4000803202E01A6842F4A0221A60704700BFD7
:10DB500000100240034B1A6822F0F80242EAC000AB
:10DB60001860704700100240014B1860704700BFFA
:10DB700000004242034B5A6822F47C1211430843CE
:10DB80005860704700100240014B1860704700BF9A
:10DB900060004242034B5A6822F00302104358606F
:10DBA000704700BF00100240024B586800F00C00A4
:10DBB000704700BF00100240034B5A6822F0F00289
:10DBC00010435860704700BF00100240034B5A6872
:10DBD00022F4E06210435860704700BF001002401A
:10DBE000034B5A6822F4605242EAC0005860704702
:10DBF00000100240044B1A7809B1104301E022EAF8
:10DC000000001870704700BF09100240014B1860F7
:10DC1000704700BFD8004242034B5A6822F440428A
:10DC200010435860704700BF00100240064B0022AE
:10DC300001281A701A7002D0042802D07047187098
:10DC4000704705221A70704720100240014B18607F
:10DC5000704700BF80044242024B1A6A10431862A8
:10DC6000704700BF00100240014B1860704700BFB2
:10DC70003C0442421C4B10B55A6802F00C02042AC4
:10DC800001D0082A01D0194A0EE05A685968C2F337
:10DC90008342CC0302F1020202D55968890301D5FF
:10DCA000134900E011494A4302605968114AC1F31F
:10DCB0000311545C0168E14041605C68C4F30224D4
:10DCC000145D21FA04F484605C68C4F3C224145D1A
:10DCD000E140C1605B68C3F381331A44137CB1FB3C
:10DCE000F3F1016110BD00BF0010024000127A0084
:10DCF00000093D002F150108044B5A6909B1104372
:10DD000001E022EA00005861704700BF00100240A5
:10DD1000044B9A6909B1104301E022EA00009861BE
:10DD2000704700BF00100240044BDA6909B110438C
:10DD300001E022EA0000D861704700BF00100240F5
:10DD4000044BDA6809B1104301E022EA0000D86010
:10DD5000704700BF00100240044B1A6909B110431C
:10DD600001E022EA00001861704700BF0010024085
:10DD7000014B1860704700BF40044242014B1860DD
:10DD8000704700BF4C004242014B1870704700BF03
:10DD9000071002404309012B074A01D1136803E031
:10DDA000022B0CBF136A536A00F01F0023FA00F025
:10DDB00000F00100704700BF0010024008B531209C
:10DDC000FFF7E8FF094B18705A6801325A601A7859
:10DDD00022B95A6840F2FF139A42F0D13120FFF77E
:10DDE000D9FF003018BF012008BD00BF8C0A0020F9
:10DDF000024B5A6A42F080725A6270470010024029
:10DE0000034B9B6818420CBF00200120704700BFE5
:10DE100000100240014B1870704700BF0A1002400A
:10DE200008B5164B98421BD003F5744398420BD0AB
:10DE3000A3F5784398421FD14FF480400121FFF7AA
:10DE40008BFF4FF4804012E04FF480500121FFF728
:10DE500077FFBDE808404FF480500021FFF770BF06
:10DE60004FF400400121FFF777FF4FF400400021FD
:10DE7000BDE80840FFF770BF08BD00BF003C004090
:10DE80000B8810B54C88028823438C8802F44152D9
:10DE90002343CC8823430C8923434C8923438C8917
:10DEA0002343CC89234313439BB20380838B23F406
:10DEB00000631B041B0C83830B8A038210BD838BBE
:10DEC000F0B523F47B6323F00F031B041B0C838347
:10DED000022303840B89868B022B87B005460C46F0
:10DEE000B6B223D08B8801A8002B14BF02270127CC
:10DEF000FFF7C0FEE3882289B3F5007F019B4FF056
:10DF00000A011CBF7F017A4301FB03F308BF120221
:10DF1000B3FBF2F305330A229BB2B3FBF2F303F037
:10DF200001021202C3F34F0392B200E00022991ED5
:10DF300089B2FE2928BF0022E18828BF02231343AB
:10DF40000B439BB22B8423886288334343F40063E2
:10DF50001343A2881343628913439BB2AB8307B078
:10DF6000F0BD0023038043808380C380038143810D
:10DF70008381C38107230382704700230222038029
:10DF800043808380C380028143817047038819B135
:10DF90009BB243F0400303E023F040031B041B0C3F
:10DFA00003807047838B19B19BB243F4806303E015
:10DFB00023F480631B041B0C83837047090901232E
:10DFC0008B409BB21AB1828892B2134303E08288DD
:10DFD00092B222EA03038380704783889BB20AB11E
:10DFE000194301E023EA0101818070478181704774
:10DFF000808980B270474FF6FF639942038803D04F
:10E000009BB243F4807303E023F480731B041B0C66
:10E0100003807047838819B19BB243F0040303E087
:10E0200023F004031B041B0C83807047038823F434
:10E0300000631B041B0C038003889BB219430180FF
:10E04000704703889BB243F4805303807047038872
:10E0500019B19BB243F4005303E023F400531B04B3
:10E060001B0C03807047012914BF008B808A80B28B
:10E070007047008A80B27047B1F5804F038803D1A2
:10E080009BB243F4804303E023F480431B041B0C46
:10E0900003807047038919420CBF0020012070479C
:10E0A000202906D1038903889BB243F040030380F3
:10E0B0007047402901D0082901D103897047C9431D
:10E0C00089B20181704701F00F02012303FA02F2C5
:10E0D00010B584880089A4B280B2104005D0090927
:10E0E0008B401C420CBF0020012010BD552906D1D9
:10E0F000038903889BB243F040030380704756298D
:10E1000001D0532901D10389704701F00F01012388
:10E1100003FA01F1C94389B201817047044B042815
:10E120001A680CBF42F0040222F004021A60704721
:10E1300010E000E0014B5860704700BF10E000E0C5
:10E140000128084B03D11A6842F0010204E00230B2
:10E1500004D11A6822F001021A60704700229A6006
:10E16000704700BF10E000E0044B1A6810B142F0A5
:10E17000020201E022F002021A60704710E000E0A3
:10E18000014B9868704700BF10E000E0C308022B05
:10E19000044B0CBF1B68DB6823FA00F000F00100A1
:10E1A000704700BF10E000E030B5048C24F001049B
:10E1B0002404240C0484058B048CADB225F0F305F3
:10E1C000A4B22A4324F0020442EA031344F00104F7
:10E1D0009DB221430583018430BD30B5048C24F009
:10E1E00010042404240C0484058B048C25F440754D
:10E1F000A4B22D052D0D24F0200444F0100445EAAE
:10E20000022242EA033344EA01119BB28CB2038337
:10E21000048430BD08B52E4B98423AD010D8A3F5EF
:10E220000063984225D003F5806398422BD0B0F16B
:10E23000804F4CD101200146FFF78EFD01201DE0EB
:10E24000244B984231D004D8A3F58063984226D05D
:10E2500008BD214B984204D003F5006398422AD0B0
:10E2600008BD4FF400600121FFF76AFD4FF4006024
:10E2700028E002200121FFF76FFD02200021BDE808
:10E280000840FFF769BD04200121FFF765FD042068
:10E29000F4E708200121FFF75FFD0820EEE71020DA
:10E2A0000121FFF759FD1020E8E720200121FFF7A9
:10E2B00053FD2020E2E74FF400500121FFF740FD1D
:10E2C0004FF400500021BDE80840FFF739BD08BDFC
:10E2D000000C004000140040002C01400388CA8854
:10E2E00003F08F03038003889BB213434A881343D0
:10E2F0009BB203808B8883850B880385054B9842EE
:10E3000003D003F50063984201D10B7A0386012301
:10E3100083827047002C0140038C70B523F0010309
:10E320001B041B0C0384038C8488028B0D8822F051
:10E3300070021204120C4E882A430D8923F0020346
:10E340001B043543ADB21B0C2B43CD88A4B285868C
:10E350000D4DA84203D005F50065A8420FD14D89A7
:10E3600023F008032B438D8823F004032B4347F647
:10E37000FF452540CC8989890C43A4B22C43848075
:10E380000283038470BD00BF002C0140038C30B5B4
:10E3900023F010031B041B0C0384038C8288048B62
:10E3A0000D8824F4E0442404240C23F0200344EAE0
:10E3B00005241B040D891B0C43EA05134D8892B2FA
:10E3C00043EA0513CD88A4B20587114D9BB2A8423C
:10E3D00003D005F50065A84216D14D8923F08003CE
:10E3E0009BB243EA05134FF6BF751D408B8845EA83
:10E3F000031347F2FF3515408A899BB245EA82052F
:10E40000CA8945EA820292B282800483038430BDC5
:10E41000002C0140038C30B523F480731B041B0CCB
:10E420000384038C8288848B0D8824F07004240478
:10E43000240C23F400732C431B040D891B0C43EAAA
:10E4400005234D8892B243EA0523CD889BB2858788
:10E45000104DA84203D005F50065A84216D14D899C
:10E4600023F400639BB243EA05234FF6FF351D40BA
:10E470008B8845EA032344F6FF7515408A899BB2D1
:10E4800045EA0215CA8945EA021292B28280848363
:10E49000038430BD002C0140038C30B523F480533D
:10E4A0001B041B0C0384038C8488828B0D8822F44C
:10E4B000E0421204120C23F4005342EA05221B042A
:10E4C0000D891B0C43EA05334D88A4B243EA05339A
:10E4D000CD8892B2A0F84050084D9BB2A84203D01C
:10E4E00005F50065A84205D18989C4F30D0444EA05
:10E4F0008114A4B284808283038430BD002C014047
:10E500004A880B8813438A881343CA8813430A89AD
:10E5100013434A8913438A8913439BB2A0F84430BA
:10E5200070474FF6FF73838000230380C3804380CE
:10E53000037270470023038043808380C38003817C
:10E5400043818381C381704700230122038043807C
:10E550008280C380038170470023038043808380CF
:10E56000C3800381438183817047038819B19BB2C3
:10E5700043F0010303E023F001039B059B0D03809F
:10E580007047B0F8443029B16FEA43436FEA534310
:10E590009BB201E0C3F30E03A0F8443070478389B7
:10E5A0009BB20AB1194301E023EA0101818170475E
:10E5B000818270470A43A0F84820704783899BB244
:10E5C0000AB1194301E023EA0101818170470389FF
:10E5D00023F007031B041B0C03817047038923F0FE
:10E5E00070031B041B0C1943018103899BB243F088
:10E5F00007030381704738B50D46602D1146044668
:10E600004FF0010202D1FFF7E8FD01E0FFF7CCFD7A
:10E61000238923F070031B041B0C2B4323812389C4
:10E620009BB243F00703238138BD10B5048942EA49
:10E630000323E4B21C43A4B22143018110BD10B5F1
:10E640000446FFF7F2FF238923F077031B041B0C1A
:10E6500043F07703238110BD10B50446FFF7E5FFB3
:10E6600023899BB243F48043238110BD01858282BC
:10E670007047038823F070039B059B0D19430180AD
:10E680007047038923F070031B041B0C194301819D
:10E69000704770B50589048B068C24F44074B6B2BB
:10E6A00024F0030426F0220625F007052404324353
:10E6B0002D04240C2D0C44F4807442EA03132943E6
:10E6C00044F001049EB201810483068470BD038B73
:10E6D00023F070031B041B0C194301837047038B49
:10E6E00023F4E0431B041B0C43EA01218BB2038398
:10E6F0007047838B23F070031B041B0C1943818329
:10E700007047838B23F4E0431B041B0C43EA012175
:10E710008BB283837047038819B19BB243F08003A7
:10E7200003E023F080039B059B0D038070478388E3
:10E7300019B19BB243F0040303E023F004031B046C
:10E740001B0C83807047838819B19BB243F0080388
:10E7500003E023F008031B041B0C838070478388AD
:10E7600019B19BB243F0010303E023F001031B0442
:10E770001B0C83807047038B23F008031B041B0CC6
:10E78000194301837047038B23F400631B041B0CA4
:10E7900043EA01218BB203837047838B23F0080384
:10E7A0001B041B0C194381837047838B23F4006384
:10E7B0001B041B0C43EA01218BB283837047038B3C
:10E7C00023F004031B041B0C194301837047038BC4
:10E7D00023F480631B041B0C43EA01218BB20383E7
:10E7E0007047838B23F004031B041B0C19438183A4
:10E7F0007047838B23F480631B041B0C43EA0121C5
:10E800008BB283837047038B23F080031B041B0CA4
:10E81000194301837047038BC3F30E0343EA0121BD
:10E820008BB203837047838B23F080031B041B0C84
:10E83000194381837047838BC3F30E0343EA01219D
:10E840008BB283837047038C23F002031B041B0CE1
:10E85000194301847047038C23F008031B041B0C2D
:10E86000194301847047038C23F020031B041B0C05
:10E8700043EA01118BB203847047038C23F08003B9
:10E880001B041B0C43EA01118BB203847047038CF9
:10E8900023F400731B041B0C43EA01218BB2038495
:10E8A0007047038C23F400631B041B0C43EA012113
:10E8B0008BB203847047038C23F400531B041B0C9E
:10E8C00043EA01318BB20384704701238B408A40B5
:10E8D00010B5048CA4B224EA03030384038C13430D
:10E8E0009BB2038410BD04238B408A4010B5048C76
:10E8F000A4B224EA03030384038C13439BB203846E
:10E9000010BD01238B4010B5048C1830A4B224EA4A
:10E910000303038121F008033BB9490844584FF62B
:10E920008F732340435043580AE00439C1F34E012A
:10E93000445848F6FF73234043501202435892B2A2
:10E940001A43425010BD038819B19BB243F0020331
:10E9500003E023F002039B059B0D038070470388AF
:10E9600019B19BB243F0040303E023F004039B05B9
:10E970009B0D03807047838819B19BB243F08003DD
:10E9800003E023F080031B041B0C83807047038883
:10E9900023F008039B059B0D038003889BB219435A
:10E9A00001807047838823F070031B041B0C838055
:10E9B00083889BB2194381807047038923F0070342
:10E9C0001B041B0C038103899BB21943018170470F
:10E9D000038923F080031B041B0C038103899BB272
:10E9E0001943018170478184704781857047818612
:10E9F00070470187704781877047A0F840107047C3
:10EA0000038B23F00C031B041B0C0383038B9BB2AF
:10EA1000194301837047038B23F440631B041B0CD1
:10EA20000383038B9BB243EA01218BB203837047BC
:10EA3000F8B50C464988A2880029B4F800E014BF54
:10EA400000270227012A054614BF01260226238932
:10EA5000BEF1000F11D1FFF7A7FB2846E188FFF7B1
:10EA6000CFFF2846394632462389FFF7B6FB2846B2
:10EA7000E188BDE8F840FFF7CEBFFFF7AEFB2846C0
:10EA8000E188FFF7C8FF2846394632462389FFF759
:10EA90008BFB2846E188BDE8F840FFF7B1BF838BC8
:10EAA00023F00C031B041B0C8383838B9BB2194341
:10EAB00081837047838B23F440631B041B0C838387
:10EAC000838B9BB243EA01218BB283837047F8B5F5
:10EAD0000E880D4604464988AA882B893EB9FFF75F
:10EAE00063FB2046E988BDE8F840FFF789BF042EA4
:10EAF00007D1FFF772FB2046E988BDE8F840FFF731
:10EB00008ABF082EEF88068C1CD126F48076360446
:10EB1000360C0684858B068CADB225F0F30545EAEC
:10EB20000313B6B29BB21A4326F4007343EA0121E1
:10EB300089B241F48071828301843946BDE8F8408E
:10EB4000FFF7ADBF26F480563604360C0684858B5D
:10EB5000068C25F440752D05B6B22D0D45EA02252B
:10EB600026F4005242EA013145EA033389B29BB2EE
:10EB700041F48051838301843946BDE8F840FFF7B2
:10EB800099BF0388DBB2038003889BB219430180DD
:10EB90007047808E80B27047008F80B27047808F40
:10EBA00080B27047B0F8400080B27047808C80B26D
:10EBB0007047008D80B27047038A19420CBF002055
:10EBC00001207047C94389B201827047038A828954
:10EBD00011EA030092B203D011420CBF00200120C1
:10EBE0007047C94389B20182704700BF08B5224B04
:10EBF00098422CD008D8A3F50063984217D003F5AB
:10EC0000806398421BD008BD1C4B984227D003F567
:10EC1000684398422FD14FF480400121FFF790F8CC
:10EC2000BDE808404FF480400021FFF789B84FF459
:10EC300000300121FFF790F84FF4003016E04FF458
:10EC400080200121FFF788F84FF480200EE04FF478
:10EC500000200121FFF780F84FF4002006E04FF478
:10EC600080100121FFF778F84FF480100021BDE8F3
:10EC70000840FFF771B808BD004C0040005000404C
:10EC8000038ACA889BB223F44053134330B50382EE
:10EC90000D4682890989AB8892B20B43698922F4B7
:10ECA000B0520B4322F00C0213439BB28381838A40
:10ECB000AA899BB223F4407387B01343044683822E
:10ECC00001A8FEF7D7FF049A039B0E498C4208BFA8
:10ECD000134619214B432A689200B3FBF2F16423D7
:10ECE000B1FBF3F21201100903FB101109013231DB
:10ECF000B1FBF3F303F00F031A4392B2228107B082
:10ED000030BD00BF003801404FF4165303600C22A1
:10ED100000238380C38003814281838170470B88F5
:10ED200010B54C88028A23438C88C98892B2234349
:10ED30000B4322F4706213439BB2038210BD002385
:10ED4000038043808380C3807047838919B19BB25D
:10ED500043F4005303E023F400531B041B0C838192
:10ED60007047C1F3421310B5012401F01F01A34203
:10ED700004FA01F101D10C3003E0022B0CBF10307A
:10ED8000143003680AB1194301E023EA010101606C
:10ED900010BD838A9BB20AB1194301E023EA010145
:10EDA00081827047038A23F00F031B041B0C03822C
:10EDB000038A9BB2194301827047838923F400635D
:10EDC0001B041B0C838183899BB21943818170478B
:10EDD000838919B19BB243F0020303E023F00203DD
:10EDE0001B041B0C83817047038A23F020031B0440
:10EDF0001B0C0382038A9BB2194301827047038A6A
:10EE000019B19BB243F4804303E023F480431B0415
:10EE10001B0C03827047C1F3080181807047808812
:10EE2000C0F30800704783899BB243F001038381DC
:10EE30007047038BDBB20383038B9BB243EA012150
:10EE400001837047038B03F47F430383038B9BB2DF
:10EE5000194301837047838A19B19BB243F02003A1
:10EE600003E023F020031B041B0C83827047838A7A
:10EE700019B19BB243F0100303E023F010031B040D
:10EE80001B0C83827047838A19B19BB243F008033D
:10EE900003E023F008031B041B0C83827047838A62
:10EEA00023F004031B041B0C8382838A9BB2194347
:10EEB00081827047838A19B19BB243F0020303E059
:10EEC00023F002031B041B0C838270470388194242
:10EED0000CBF002001207047C94389B201807047F0
:10EEE00010B5C1F3421401F01F030122012C02FAF4
:10EEF00003F201D1838903E0022C0CBF038A838AC9
:10EF00009BB21340028892B243B10123090A03FA6B
:10EF100001F111420CBF0020012010BD184610BDA8
:10EF2000090A01238B40DB439BB20380704700BF7B
:10EF3000684620F007018D4601B500230B4A0C49B5
:10EF40009818884204D20B49595899500433F5E770
:10EF5000094B0A4A934203D2002243F8042BF8E7F4
:10EF600002F036F8BDE801408546704700000020F9
:10EF70006005002074160108600500208C15002033
:10EF800010B5064C18B9236801221A8210BD044B33
:10EF90001B681B68984720680A3010BDD8140020F1
:10EFA0009414002010B5064C18B9236801221A8267
:10EFB00010BD044B1B689B68984720680C3010BD3F
:10EFC000D81400209414002010B5204B18B91B68E9
:10EFD00002221A8210BD1E4A1968002010800C7887
:10EFE000134614F07F040DD14A7A910644BF0221E2
:10EFF000197012F0400F1A7814BF22F0010242F08B
:10F00000010214E0012C1FD0022C1ED1497901F01D
:10F010000F02920002F1804202F5B84211F0800F17
:10F02000126806D002F03002102A07D101221A70AD
:10F0300004E002F44052B2F5805FF6E7054B1B682E
:10F040001B699847024810BD104610BDD814002017
:10F050008415002094140020234A2DE9F8431468F5
:10F060009046238A267A214FA3B9042E12D1204933
:10F070000A78012A0AD11F4A10681F4A80B2024446
:10F080005200136030223A800B7027E010233B803F
:10F09000072623E0A58AAB428CBF022604269D42A8
:10F0A00028BF1D462846A36998478146002000F0E6
:10F0B0006BFE2A460146484600F06EFC29460020B9
:10F0C00000F07EFE238A4FF440525B1B2382638A4A
:10F0D0001D4430233B80094B65821A80D8F80030EC
:10F0E0001E72BDE8F88300BFD814002088150020E8
:10F0F000940A0020505C0040023000208615002059
:10F1000010B50A4B0A491B684978DA7891420AD34C
:10F11000997841B99C8834B99A72064B1B685B6830
:10F120009847204610BD022010BD00BFD814002013
:10F13000D40000209414002038B50E4A0E4C1268FA
:10F14000236892695879D978904723689A7A7AB176
:10F1500070B91A7962B99D7855B9084B1B68DB689C
:10F160009847236828465A79DA72DA781A7338BDD4
:10F17000022038BD70140020D81400209414002000
:10F1800038B52F4B1B68187810F07F0004D15A7ADD
:10F1900022F020025A7238BD02284ED15A88002A25
:10F1A0004CD11A79002A49D15A79264D22F0800093
:10F1B000840004F1804101F5B84109682D7812F00E
:10F1C000800F14BF01F0300101F44051A84234D245
:10F1D000002932D09B7A83B304F1804404F5B8440B
:10F1E000120623680CD503F03003102B1FD1C4B2D4
:10F1F000204600F080FD2046302100F055FC16E04E
:10F2000003F44053B3F5805F11D128B90E4B93F846
:10F210002C1000F0F6FD01E000F05DFD236823F402
:10F22000804323F070039BB283F440532360074B69
:10F230001B685B699847002038BD022038BD00BFBD
:10F24000D8140020D40000204C000020941400208A
:10F2500038B51D4B1D4D19682D784A7922F0800470
:10F26000A30003F1804000F5B840006812F0800F61
:10F2700014BF00F0300000F44050AC4222D24C8861
:10F2800004BBF8B1897AE9B103F1804303F5B843CF
:10F2900012F0800F1A6807D022F4E04222F04002F8
:10F2A00092B282F0100206E022F4804222F0700254
:10F2B00092B282F480521A60054B1B689B69984792
:10F2C000002038BD022038BDD8140020D400002012
:10F2D0009414002008B5064B1B685A7A42F02002AD
:10F2E0005A72044B1B68DB699847002008BD00BFB9
:10F2F000D814002094140020054B1A68538A18B9BA
:10F300008988CB1A1382704708681844704700BF79
:10F31000D814002008B50B4B002093F82C1000F0F7
:10F3200070FD094B1B68187A082806D1074B4FF46B
:10F3300080521A80064B10221A80B0F109035842FD
:10F34000584108BD4C000020D8140020861500202C
:10F3500088150020F7B5914F914B3A68914D92B2C4
:10F3600013442E685B001C68337A092B15D0A4B2B5
:10F37000640004F1804404F5C0442378337063785A
:10F380007370A08800F0E8FE708020892E6800F07D
:10F39000E3FEB080A2892B68DA802B6801221A7202
:10F3A000DA885C78002A61D11A7812F07F023AD1AB
:10F3B000092C02D1FFF7A4FE44E0052C0FD193F9EC
:10F3C0000320002A01DA08234DE09A78002AFAD1B6
:10F3D0009A88002AF7D19B7A002B37D0F3E7032CC9
:10F3E00013D1DA78012A07D06F4B20461B685B697E
:10F3F0009847032828D135E09A88002AF4D15B7A0F
:10F400009806F1D5FFF766FF1CE0012CECD1DA7805
:10F41000012AE9D19A88002AE6D15B7A9906E3D5D8
:10F42000FFF7AEFE0EE0012A04D10B2CDCD1FFF772
:10F4300083FE07E0022AD7D1012CF1D0032CD3D1CF
:10F44000FFF706FF10B1CFE70028BCD13A68574B51
:10F4500092B213445B0000221A60554B30221A808E
:10F46000062300E009232A681372D0E0062C13D18A
:10F470001A78520678D19A784B4B012A02D11B6830
:10F48000DB6968E0022A02D11B681B6A63E0032A79
:10F490006AD11B685B6A5EE0002C3DD15988002967
:10F4A00062D15A6822F47F42B2F5003F5CD11A78EB
:10F4B00012F07F0204D19B88002B00F0AC8053E057
:10F4C000012A0DD1384A587912689269904700286C
:10F4D0004AD1344B1B689B7A002B40F09C8043E060
:10F4E000022A41D15B79334803F00F018A0002F10F
:10F4F000804202F5B8421268007813F0800F14BF02
:10F5000002F0300202F4405281422DD213F0700F0B
:10F510002AD1002A7FD127E0082C03D11B785B0673
:10F520007BD021E00A2C1FD11A7802F07F02012A39
:10F530001AD19A7AC2B15988B1B95A6822F47F4275
:10F54000B2F5803F10D1184A5879126892699047F5
:10F55000002864D008E03BB12A68002454829361FB
:10F560002046984720460AE00F4B1A682B6812691C
:10F5700058789047032802D10A4B1B6805E02B6896
:10F580004FF6FF711A8A8A4201D1092203E002284C
:10F5900000D08AB908221A7239E000BF505C0040DE
:10F5A00004300020D8140020701400200230002005
:10F5B00088150020D400002093F90010002920DADB
:10F5C000D988019101988242164802D9019A1A827B
:10F5D00010E08A420ED2016891F82C108A4201D2C2
:10F5E000002105E092FBF1F401FB142212B9012184
:10F5F0000D4A1170026892F82C209A82FFF72CFDB8
:10F6000005E003221A72094B4FF440521A80FFF7AB
:10F6100081FE03B0F0BD064B9EE7064B9CE7064B10
:10F620009AE700BF70140020940A0020861500207D
:10F63000C9EF000881EF0008A5EF0008F8B52B4DD1
:10F640002C68237A032B01D0052B41D1A369228A90
:10F65000ABB1A2B1A68A964228BF1646304698475B
:10F66000238A07469B1B2382638A002033446382DC
:10F6700000F098FB32460146384600F0A5F9238A8F
:10F6800053B11B4B00204FF4405201461A8000F04A
:10F6900097FB184B30221A80238AA28A9A4202D8FA
:10F6A0002B68032202E01BB12B6805221A720CE0C2
:10F6B0002A6806211172104A1168104A89B20A4458
:10F6C000520013600B4B30221A802B681B7A06E025
:10F6D000072B03D10A4B1B68DB68984708232A686D
:10F6E0001372BDE8F840FFF715BE00BFD814002024
:10F6F0008615002088150020505C00400230002054
:10F700007014002030B50B4B1C780023A3420CD2A0
:10F7100003F1805202F5B85291000D6848F68F72DD
:10F720002A401A430A600133F0E7034B40F080009F
:10F73000186030BDD40000204C5C004010B5134C64
:10F7400023681A7A022A01D0042A04D1FFF784FC24
:10F7500023681B7A13E0062A10D15A78052A09D1AA
:10F760001A78520606D1D878FFF7CCFF084B1B68F1
:10F770001B6A9847074B1B689B68984708232268B9
:10F780001372BDE81040FFF7C5BD00BFD8140020BC
:10F790009414002070140020704700BF08B5074A79
:10F7A000074B0849136002221A72074B074A13607D
:10F7B000074A1B681160984708BD00BFD814002095
:10F7C00078140020B00000204C00002070140020AD
:10F7D0009414002070B54C4A4C4B116888B20C044C
:10F7E000188040F1908047F6FF7111601A88484CEC
:10F7F00002F00F022270002A5FD1464C464D22686B
:10F80000464E02F440522A80226802F030023280D2
:10F81000226822F4804222F0700292B282F40052F6
:10F820002260226822F4E04222F0400292B282F08A
:10F83000200222601B88D80602D52368190607D546
:10F84000226848F60F7313402360FFF777FF12E03A
:10F850001A0507D5226840F68F7313402360FFF71F
:10F8600079FD08E01804B6D5226840F68F7313407E
:10F870002360FFF7E3FE23682A8823F4804323F004
:10F8800070039BB2D10448BF83F480539504214A8E
:10F8900048BF83F4005313601368318823F4E043B6
:10F8A00023F040039BB2CC0648BF83F010038806C8
:10F8B00048BF83F02003136070BD930003F18043C1
:10F8C00003F5B8431D68290409D5186840F68F71FF
:10F8D00001401960124B013A53F8223098472B0629
:10F8E0007FF579AF217848F60F728B0003F18043E2
:10F8F00003F5B8431868013902401A60094B53F800
:10F900002130984767E770BD445C00406E140020CA
:10F9100074140020005C004086150020881500202B
:10F92000D8000020F400002008B5164A164B1168D4
:10F9300088B20904188024D547F6FF7111601A882F
:10F94000124B02F00F021A70930003F1804303F58B
:10F95000B8431968080407D5186840F68F7101404C
:10F960001960013A0A4B08E00906DED5186848F626
:10F970000F7101401960074B013A53F82230984744
:10F98000D3E708BD445C00406E14002074140020CE
:10F99000D8000020F400002030B501F10051013200
:10F9A00001F54051521049000023934200F102003A
:10F9B00009D010F8015C10F8024C44EA052421F843
:10F9C00023400133F1E730BD10B501F100510132A0
:10F9D00001F54051521049000023934205D051F8DF
:10F9E000234020F813400133F7E710BD014B1860A6
:10F9F000704700BF405C0040014B186880B2704700
:10FA0000405C0040014B1860704700BF445C004000
:10FA1000014B186880B27047445C0040014B186885
:10FA200080B27047485C0040014B1860704700BFCF
:10FA30004C5C0040014B186880B270474C5C004041
:10FA40004FF6F873014A034013607047505C004062
:10FA5000014B186880B27047505C0040800000F194
:10FA6000804000F5B84001607047800000F18040A0
:10FA700000F5B840006880B27047800000F1804017
:10FA800000F5B840036823F4EC4323F070031943F6
:10FA90008BB203607047800000F1804000F5B840F1
:10FAA000006800F4C0607047800000F1804000F5FD
:10FAB000B8400368CA0623F4E04323F040039BB236
:10FAC00048BF83F010038A0648BF83F02003036019
:10FAD0007047800000F1804000F5B8400368CA0418
:10FAE00023F4804323F070039BB248BF83F4805318
:10FAF0008A0448BF83F4005303607047800000F11C
:10FB0000804000F5B8400129026802D14EF6FF732B
:10FB100003E0022903D14FF6EF73134003607047EF
:10FB2000800000F1804000F5B840006800F030002F
:10FB30007047800000F1804000F5B840006800F494
:10FB400040507047800000F1804000F5B8400368E5
:10FB500023F4E04323F040039BB283F030030360BF
:10FB60007047800000F1804000F5B840036823F43E
:10FB7000804323F070039BB283F4405303607047CB
:10FB8000800000F1804000F5B840036823F4E043B2
:10FB900023F0700343F480739BB2036070478000CE
:10FBA00000F1804000F5B840036823F4E24323F0FD
:10FBB00070031B041B0C03607047800000F1804041
:10FBC00000F5B840036823F4E24323F070031B04FC
:10FBD0001B0C03607047800000F1804000F5B840C6
:10FBE000036823F4E04323F0700343F480739BB273
:10FBF00003607047800000F1804000F5B840036862
:10FC000023F4E04323F0700343F480739BB203605A
:10FC10007047800000F1804000F5B840036823F48D
:10FC2000E24323F070031B041B0C03607047800049
:10FC300000F1804000F5B840006800F03000B0F1FD
:10FC40001003584258417047800000F1804000F591
:10FC5000B840006800F44050B0F580535842584115
:10FC60007047800000F1804000F5B840036823F041
:10FC700070031B051B0D03607047800000F180407E
:10FC800000F5B840036823F4E14323F070031B043C
:10FC90001B0C03607047800000F1804000F5B84005
:10FCA000036823F4E04323F070031B041B0C43F4AC
:10FCB000804303607047800000F1804000F5B84049
:10FCC000036823F4E04323F070031B041B0C43F090
:10FCD000400303607047800000F1804000F5B840A9
:10FCE00003685B0406D5026848F68F73134043F43B
:10FCF000804303607047800000F1804000F5B84009
:10FD000003685B0606D5026848F68F73134043F01C
:10FD1000400303607047800000F1804000F5B84068
:10FD2000036823F4E04323F070031B041B0C194306
:10FD300001607047800000F1804000F5B840006825
:10FD400000F00F007047074B49081B6849009BB241
:10FD500003EBC00000F1005000F54050400001608E
:10FD6000704700BF505C0040054B49081B684900C4
:10FD70009BB203EBC000034B03445B001960704768
:10FD8000505C004004300020054B1B689BB203EB25
:10FD9000C00000F1005000F540504000008870475E
:10FDA000505C0040044B1B689BB203EBC000034B4C
:10FDB00003445B0018887047505C0040043000200A
:10FDC000044B1B689BB203EBC000034B03445B0076
:10FDD00019607047505C0040023000203E2909D96C
:10FDE0004B09C90604BF03F1FF339BB29B0243F4E6
:10FDF000004304E04B08CA0748BF01339B0203607D
:10FE000070470E4B3E291B689BB203EBC0000C4BA6
:10FE100003444FEA430209D94B09C80604BF03F162
:10FE2000FF339BB29B0243F4004304E04B08C90735
:10FE300048BF01339B021360704700BF505C004015
:10FE400006300020054B1B689BB203EBC000044B3F
:10FE500003445B001868C0F309007047505C004021
:10FE600002300020054B1B689BB203EBC000044B23
:10FE700003445B001868C0F309007047505C004001
:10FE80000630002010B50B4CC000236849089BB217
:10FE9000034403F1005303F540535B00490019602C
:10FEA000236852089BB21844034B520003445B0082
:10FEB0001A6010BD505C004004300020064B490819
:10FEC0001B6849009BB203EBC00000F1005000F535
:10FED0004050400001607047505C0040054B4908AD
:10FEE0001B6849009BB203EBC000034B03445B005B
:10FEF00019607047505C004004300020054B1B68BF
:10FF00009BB203EBC00000F1005000F540504000F0
:10FF100000887047505C0040044B1B689BB203EBA9
:10FF2000C000034B03445B0018887047505C0040DE
:10FF300004300020012910B52FD1254CC0002168C4
:10FF4000244B89B201440B443E2A4FEA43010AD9AB
:10FF5000530912F01F0F04BF03F1FF339BB29B0242
:10FF600043F4004305E0530812F0010F18BF0133BA
:10FF70009B020B6023683E2A9BB21844164B034435
:10FF80004FEA43031CD95109D00604BF01F1FF31E8
:10FF900089B2890241F4004117E0022917D10C49C6
:10FFA000C0000C680B4BA4B2044423445B001A60ED
:10FFB0000B689BB21844084B03445B001A6010BDE9
:10FFC0005108D20748BF01318902196010BD10BD28
:10FFD000505C0040023000200630002001291BD177
:10FFE000134B3E2A1B689BB203EBC000114B03442A
:10FFF0004FEA430109D95309D00604BF03F1FF3387
:020000040801F1
:100000009BB29B0243F4004304E05308D20748BF6D
:1000100001339B020B607047022908D1044B1B6817
:100020009BB203EBC000034B03445B001A607047B4
:10003000505C00400230002001291BD1134B3E2AA6
:100040001B689BB203EBC000114B03444FEA430112
:1000500009D95309D00604BF03F1FF339BB29B02B9
:1000600043F4004304E05308D20748BF01339B0226
:100070000B607047022908D1044B1B689BB203EB4D
:10008000C000034B03445B001A607047505C0040A3
:1000900006300020054B1B689BB203EBC000044BED
:1000A00003445B001868C0F309007047505C0040CF
:1000B00002300020054B1B689BB203EBC000044BD1
:1000C00003445B001868C0F309007047505C0040AF
:1000D000063000200D4AC00013689BB2C1180C4BBB
:1000E0000B445B001B8813F47C4F0DD113689BB24B
:1000F0001844084B03445B001B88C3F30903002B1F
:100100000CBF00200220704701207047505C004067
:10011000063000200230002001290BD1800000F1C0
:10012000804000F5B840026848F68F73134043F0F2
:1001300040030CE002290BD1800000F1804000F563
:10014000B840026848F68F73134043F4804303605D
:10015000704741EA00207047C3B2000A40EA03201A
:10016000704700BF81F0004102E000BF83F0004310
:1001700030B54FEA41044FEA430594EA050F08BF42
:1001800090EA020F1FBF54EA000C55EA020C7FEA06
:10019000645C7FEA655C00F0E2804FEA5454D4EB83
:1001A0005555B8BF6D420CDD2C4480EA020281EA4D
:1001B000030382EA000083EA010180EA020281EA85
:1001C0000303362D88BF30BD11F0004F4FEA0131D7
:1001D0004FF4801C4CEA113102D0404261EB4101E6
:1001E00013F0004F4FEA03334CEA133302D052426C
:1001F00063EB430394EA050F00F0A780A4F1010428
:10020000D5F1200E0DDB02FA0EFC22FA05F2801861
:1002100041F1000103FA0EF2801843FA05F3594147
:100220000EE0A5F120050EF1200E012A03FA0EFCC6
:1002300028BF4CF0020C43FA05F3C01851EBE371F0
:1002400001F0004507D54FF0000EDCF1000C7EEB0D
:1002500000006EEB0101B1F5801F1BD3B1F5001F4B
:100260000CD349085FEA30004FEA3C0C04F101046A
:100270004FEA445212F5800F80F09A80BCF1004F93
:1002800008BF5FEA500C50F1000041EB045141EA15
:10029000050130BD5FEA4C0C404141EB010111F416
:1002A000801FA4F10104E9D191F0000F04BF0146C1
:1002B0000020B1FA81F308BF2033A3F10B03B3F19F
:1002C00020020CDA0C3208DD02F1140CC2F10C022F
:1002D00001FA0CF021FA02F10CE002F11402D8BF8D
:1002E000C2F1200C01FA02F120FA0CFCDCBF41EA59
:1002F0000C019040E41AA2BF01EB0451294330BD28
:100300006FEA04041F3C1CDA0C340EDC04F1140404
:10031000C4F1200220FA04F001FA02F340EA0300DB
:1003200021FA04F345EA030130BDC4F10C04C4F121
:10033000200220FA02F001FA04F340EA0300294601
:1003400030BD21FA04F0294630BD94F0000F83F44B
:10035000801306BF81F480110134013D4EE77FEA2E
:10036000645C18BF7FEA655C29D094EA050F08BF7A
:1003700090EA020F05D054EA000C04BF194610465B
:1003800030BD91EA030F1EBF0021002030BD5FEA9F
:10039000545C05D14000494128BF41F0004130BDC7
:1003A00014F580043CBF01F5801130BD01F000451B
:1003B00045F0FE4141F470014FF0000030BD7FEA8E
:1003C000645C1ABF194610467FEA655C1CBF0B4689
:1003D000024650EA013406BF52EA033591EA030FA0
:1003E00041F4002130BD00BF90F0000F04BF002198
:1003F000704730B54FF4806404F132044FF00005CB
:100400004FF0000150E700BF90F0000F04BF002143
:10041000704730B54FF4806404F1320410F00045A9
:1004200048BF40424FF000013EE700BF42004FEAA4
:10043000E2014FEA31014FEA02701FBF12F07F4321
:1004400093F07F4F81F06051704792F0000F14BF1E
:1004500093F07F4F704730B54FF4607401F0004562
:1004600021F0004120E700BF50EA010208BF7047B9
:1004700030B54FF000050AE050EA010208BF7047AE
:1004800030B511F0004502D5404261EB41014FF417
:10049000806404F132045FEA915C3FF4DCAE4FF01B
:1004A00003025FEADC0C18BF03325FEADC0C18BF02
:1004B000033202EBDC02C2F1200300FA03FC20FA53
:1004C00002F001FA03FE40EA0E0021FA02F11444A0
:1004D000C1E600BF70B54FF0FF0C4CF4E06C1CEAB5
:1004E00011541DBF1CEA135594EA0C0F95EA0C0F2A
:1004F00000F0DEF82C4481EA030621EA4C5123EA9D
:100500004C5350EA013518BF52EA033541F48011CB
:1005100043F4801338D0A0FB02CE4FF00005E1FB7E
:1005200002E506F00042E0FB03E54FF00006E1FBC8
:1005300003569CF0000F18BF4EF0010EA4F1FF040B
:10054000B6F5007F64F5407404D25FEA4E0E6D414B
:1005500046EB060642EAC62141EA55514FEAC5205C
:1005600040EA5E504FEACE2EB4F1FD0C88BFBCF5D8
:10057000E06F1ED8BEF1004F08BF5FEA500E50F189
:10058000000041EB045170BD06F0004646EA01014F
:1005900040EA020081EA0301B4EB5C04C2BFD4EB81
:1005A0000C0541EA045170BD41F480114FF0000E7A
:1005B000013C00F3AB8014F1360FDEBF002001F0E8
:1005C000004170BDC4F10004203C35DA0C341BDC62
:1005D00004F11404C4F1200500FA05F320FA04F034
:1005E00001FA05F240EA020001F0004221F0004168
:1005F00010EBD37021FA04F642EB06015EEA430EDB
:1006000008BF20EAD37070BDC4F10C04C4F120050A
:1006100000FA04F320FA05F001FA04F240EA0200BD
:1006200001F0004110EBD37041F100015EEA430E8E
:1006300008BF20EAD37070BDC4F1200500FA05F2AE
:100640004EEA020E20FA04F301FA05F243EA02032D
:1006500021FA04F001F0004121FA04F220EA02003C
:1006600000EBD3705EEA430E08BF20EAD37070BD82
:1006700094F0000F0FD101F00046400041EB010162
:1006800011F4801F08BF013CF7D041EA060195F044
:10069000000F18BF704703F00046520043EB0303FE
:1006A00013F4801F08BF013DF7D043EA06037047EB
:1006B00094EA0C0F0CEA135518BF95EA0C0F0CD0F6
:1006C00050EA410618BF52EA4306D1D181EA03013C
:1006D00001F000414FF0000070BD50EA410606BF36
:1006E0001046194652EA430619D094EA0C0F02D17B
:1006F00050EA013613D195EA0C0F05D152EA0336C0
:100700001CBF104619460AD181EA030101F00041DD
:1007100041F0FE4141F470014FF0000070BD41F026
:10072000FE4141F4780170BD70B54FF0FF0C4CF400
:10073000E06C1CEA11541DBF1CEA135594EA0C0F1F
:1007400095EA0C0F00F0A7F8A4EB050481EA030E6C
:1007500052EA03354FEA013100F088804FEA033353
:100760004FF0805545EA131343EA12634FEA022221
:1007700045EA111545EA10654FEA00260EF00041E2
:100780009D4208BF964244F1FD0404F5407402D234
:100790005B084FEA3202B61A65EB03055B084FEAC5
:1007A00032024FF480104FF4002CB6EB020E75EBC2
:1007B000030E22BFB61A754640EA0C005B084FEAEA
:1007C0003202B6EB020E75EB030E22BFB61A754667
:1007D00040EA5C005B084FEA3202B6EB020E75EBB2
:1007E000030E22BFB61A754640EA9C005B084FEA2A
:1007F0003202B6EB020E75EB030E22BFB61A754637
:1008000040EADC0055EA060E18D04FEA051545EA25
:1008100016754FEA06164FEAC30343EA52734FEACE
:10082000C2025FEA1C1CC0D111F4801F0BD141EA47
:1008300000014FF000004FF0004CB6E711F4801FAC
:1008400004BF01430020B4F1FD0C88BFBCF5E06F8C
:100850003FF6AFAEB5EB030C04BFB6EB020C5FEA9C
:10086000500C50F1000041EB045170BD0EF0004EF1
:100870004EEA113114EB5C04C2BFD4EB0C0541EA23
:10088000045170BD41F480114FF0000E013C90E620
:1008900045EA060E8DE60CEA135594EA0C0F08BFE4
:1008A00095EA0C0F3FF43BAF94EA0C0F0AD150EAE3
:1008B00001347FF434AF95EA0C0F7FF425AF104676
:1008C00019462CE795EA0C0F06D152EA03353FF49E
:1008D000FDAE1046194622E750EA410618BF52EA1B
:1008E00043067FF4C5AE50EA41047FF40DAF52EAEF
:1008F00043057FF4EBAE12E74FEA410212F5001216
:1009000015D211D56FF47873B3EB625212D94FEA56
:10091000C12343F0004343EA505311F0004F23FA40
:1009200002F018BF404270474FF00000704750EA95
:10093000013005D111F0004008BF6FF00040704752
:100940004FF00000704700BF4FEA4102B2F1E043B0
:1009500024BFB3F5001CDCF1FE5C0DD901F0004CA6
:100960004FEAC0024CEA5070B2F1004F40EB8300F6
:1009700008BF20F00100704711F0804F21D113F122
:100980003872BCBF01F00040704741F480114FEA5B
:100990005252C2F11802C2F1200C10FA0CF320FAE4
:1009A00002F018BF40F001004FEAC1234FEAD32301
:1009B00003FA0CFC40EA0C0023FA02F34FEA43036B
:1009C000CCE77FEA625307D150EA01331EBF4FF0F4
:1009D000FE4040F44000704701F0004040F0FE400F
:1009E00040F40000704700BF80F0004002E000BF0C
:1009F00081F0004142001FBF5FEA410392EA030F0A
:100A00007FEA226C7FEA236C6AD04FEA1262D2EB53
:100A10001363C1BFD218414048404140B8BF5B4258
:100A2000192B88BF704710F0004F40F4000020F0F1
:100A30007F4018BF404211F0004F41F4000121F007
:100A40007F4118BF494292EA030F3FD0A2F1010251
:100A500041FA03FC10EB0C00C3F1200301FA03F18F
:100A600000F0004302D5494260EB4000B0F5000FB2
:100A700013D3B0F1807F06D340084FEA310102F171
:100A80000102FE2A51D2B1F1004F40EBC25008BF23
:100A900020F0010040EA03007047490040EB0000ED
:100AA00010F4000FA2F10102EDD1B0FA80FCACF11C
:100AB000080CB2EB0C0200FA0CF0AABF00EBC2501B
:100AC00052421843BCBFD0401843704792F0000F09
:100AD00081F4000106BF80F400000132013BB5E75C
:100AE0004FEA41037FEA226C18BF7FEA236C21D0D2
:100AF00092EA030F04D092F0000F08BF0846704737
:100B000090EA010F1CBF0020704712F07F4F04D104
:100B1000400028BF40F00040704712F100723CBF17
:100B200000F50000704700F0004343F0FE4040F441
:100B3000000070477FEA226216BF08467FEA2363FF
:100B40000146420206BF5FEA412390EA010F40F4EA
:100B5000800070474FF0000304E000BF10F0004336
:100B600048BF40425FEA000C08BF704743F096431D
:100B700001464FF000001CE050EA010208BF704738
:100B80004FF000030AE000BF50EA010208BF7047BF
:100B900011F0004302D5404261EB41015FEA010CD4
:100BA00002BF84460146002043F0B64308BFA3F1CC
:100BB0008053A3F50003BCFA8CF2083AA3EBC253AE
:100BC00010DB01FA02FC634400FA02FCC2F12002CD
:100BD000BCF1004F20FA02F243EB020008BF20F004
:100BE0000100704702F1200201FA02FCC2F120026A
:100BF00050EA4C0021FA02F243EB020008BF20EA5F
:100C0000DC7070474FF0FF0C1CEAD0521EBF1CEA8C
:100C1000D15392EA0C0F93EA0C0F6FD01A4480EA7A
:100C2000010C400218BF5FEA41211ED04FF0006363
:100C300043EA501043EA5111A0FB01310CF000408F
:100C4000B1F5000F3EBF490041EAD3715B0040EAB5
:100C5000010062F17F02FD2A1DD8B3F1004F40EB85
:100C6000C25008BF20F00100704790F0000F0CF058
:100C7000004C08BF49024CEA502040EA51207F3A1C
:100C8000C2BFD2F1FF0340EAC250704740F40000F7
:100C90004FF00003013A5DDC12F1190FDCBF00F0E8
:100CA00000407047C2F10002410021FA02F1C2F196
:100CB000200200FA02FC5FEA310040F1000053EA32
:100CC0004C0308BF20EADC70704792F0000F00F080
:100CD000004C02BF400010F4000F013AF9D040EA86
:100CE0000C0093F0000F01F0004C02BF490011F41A
:100CF000000F013BF9D041EA0C018FE70CEAD15318
:100D000092EA0C0F18BF93EA0C0F0AD030F0004C97
:100D100018BF31F0004CD8D180EA010000F000404B
:100D2000704790F0000F17BF90F0004F084691F009
:100D3000000F91F0004F14D092EA0C0F01D1420243
:100D40000FD193EA0C0F03D14B0218BF084608D10C
:100D500080EA010000F0004040F0FE4040F4000056
:100D6000704740F0FE4040F4400070474FF0FF0CE9
:100D70001CEAD0521EBF1CEAD15392EA0C0F93EA30
:100D80000C0F69D0A2EB030280EA010C49024FEA82
:100D9000402037D04FF0805343EA111143EA10133B
:100DA0000CF000408B4238BF5B0042F17D024FF4F3
:100DB000000C8B4224BF5B1A40EA0C00B3EB510FCE
:100DC00024BFA3EB510340EA5C00B3EB910F24BFB7
:100DD000A3EB910340EA9C00B3EBD10F24BFA3EB3C
:100DE000D10340EADC001B0118BF5FEA1C1CE0D104
:100DF000FD2A3FF650AF8B4240EBC25008BF20F0B7
:100E0000010070470CF0004C4CEA50207F32C2BF0A
:100E1000D2F1FF0340EAC250704740F400004FF0A7
:100E20000003013A37E792F0000F00F0004C02BFD8
:100E3000400010F4000F013AF9D040EA0C0093F0A2
:100E4000000F01F0004C02BF490011F4000F013BFC
:100E5000F9D041EA0C0195E70CEAD15392EA0C0F64
:100E600008D142027FF47DAF93EA0C0F7FF470AF9C
:100E7000084676E793EA0C0F04D14B023FF44CAFDF
:100E800008466EE730F0004C18BF31F0004CCAD174
:100E900030F000427FF45CAF31F000437FF43CAFB0
:100EA0005FE700BF4FF0FF3C06E000BF4FF0010CD2
:100EB00002E000BF4FF0010C4DF804CD4FEA4002B4
:100EC0004FEA41037FEA226C18BF7FEA236C11D0FE
:100ED00001B052EA530C18BF90EA010F58BFB2EBB1
:100EE000030088BFC81738BF6FEAE17018BF40F031
:100EF000010070477FEA226C02D15FEA402C05D1E5
:100F00007FEA236CE4D15FEA412CE1D05DF8040B69
:100F1000704700BF844608466146FFE70FB5FFF7FC
:100F2000C9FF002848BF10F1000F0FBD4DF808EDB4
:100F3000FFF7F4FF0CBF012000205DF808FB00BFA5
:100F40004DF808EDFFF7EAFF34BF012000205DF8FF
:100F500008FB00BF4DF808EDFFF7E0FF94BF01204C
:100F600000205DF808FB00BF4DF808EDFFF7D2FF49
:100F700094BF012000205DF808FB00BF4DF808ED8C
:100F8000FFF7C8FF34BF012000205DF808FB00BF59
:100F900042000ED2B2F1FE4F0BD34FF09E03B3EBE3
:100FA000126209D44FEA002343F0004323FA02F00F
:100FB00070474FF00000704712F1610F01D14202FB
:100FC00002D14FF0FF3070474FF00000704700BF74
:100FD0002DE9F341774EFCF783FD00244FF4803078
:100FE0003470FCF79BFDFCF7E9FE0128054626D18D
:100FF0001020FCF795F82046FCF7DEFD2046FCF7B4
:10100000EFFD4FF48060FCF7E1FD4FF440304FF40A
:10101000E011FCF7AFFD2846FCF7B6FD3920FCF7E0
:10102000B9FE0028FAD00220FCF762F80220FCF793
:10103000B1FDFCF7B9FD0828FBD101233370042072
:101040000121FCF765FE4FF48073ADF804300323F3
:1010500001A98DF80630584818238DF80730FCF7A1
:10106000E0FA0620FCF790FE01200146FCF750FE56
:101070004FF0C0500121FCF757FE4FF480414FF074
:101080000060FCF779FC4FF44070FCF7CBFBF3F702
:10109000A5F8F3F729FBF3F773F8F3F79CFAF8F7E1
:1010A00043F9F8F723F9F7F7F5FBF3F76FF9F3F7DF
:1010B000C1FA424C28B1F3F7BDFA6070F3F7BAFAFF
:1010C000A060F3F7E5FA3E4F2078F7F765FCE0788B
:1010D000F7F7AEFD3B78394D23B96879A9682A69DD
:1010E000F7F7E0FE3B780BB1F8F71AFCF8F798FE3B
:1010F000FAF700FFF3F7CCFAF3F7E0FADFF8B8807D
:10110000D0F1010538BF0025F6F7A0FCF8F780FC08
:10111000F9F7F0F94FF40073C8F81030294BC022EA
:101120005A61F8F7FBF80646F6F7B4FDF9F7F6F959
:10113000F8F76FFCF8F7F2F8801B0028B8BF4042C0
:10114000B0F57A7F23DD3B781D4E8BB1D8F808309F
:1011500013F4004318D13370F8F712FCF8F7FEFBD4
:10116000F3F70EF86079A1682269F7F79BFE0BE0B0
:10117000D8F808301B0407D5F7F7D2FF01233370E6
:10118000F2F7FEFFF8F7CCFBF8F7C8F80646F3F7DE
:101190007FFAF3F79DFA0028C6D00DB1FAF7AAFE40
:1011A000F8F73EFE0025F6F751FCF9F7A3F9F8F73A
:1011B00047FCB9E7F01200200008014004000020BD
:1011C000EC100020000C014000210A2200F0ACB815
:1011D0000F4B30B405461C6802E0D01A16D1ABB1F3
:1011E00015F8013BE21850781A4600F00300012878
:1011F00008BF03F1200211F8013BE018407800F02D
:1012000003000128E9D12033D01AE9D030BC70475F
:101210005C0500202DE9F00F424C82B0D4F800C0EC
:1012200001900E4600E02646344614F8015B0CEBB4
:101230000500407800F0080000F0FF0A0028F2D115
:101240002D2D5BD02B2D04BF7578B41C33F010000E
:101250003CD09946BAF1000F0CBF6FF0004B4FF035
:10126000004BBBFBF9F8002709FB18BB38460CE024
:10127000303DAB4219DD7E1C05D0404523D820D03F
:1012800009FB0050012714F8015B0CEB050676788A
:1012900016F0040FECD116F0030606D0012E14BF91
:1012A00057263726AD1BAB42E5DC7B1C15D0BAF1C7
:1012B000000F21D10AB1EFB9116002B0BDE8F00F03
:1012C00070475D45DCDD4FF0FF37DCE7302D1AD08D
:1012D000002BBED10A239946BCE70199BAF1000F51
:1012E0004FF022030CBF6FF000404FF000400B6046
:1012F000002AE2D0611EDFE74042DBE7B41C7578CC
:101300004FF0010AA2E7207800F0DF00582803D050
:10131000002B9ED108239CE7102365789946023460
:1013200098E700BF5C05002030B4044C0D4613461E
:1013300001462A46206830BCFFF76CBF58050020E4
:10134000F4010000640000000180080800000000B3
:10135000000200000000000000000000C8000000C3
:101360000000000000000000010003E80000000091
:1013700000000003E800000000000200FA0600037D
:101380000000000000370600000000000000000020
:1013900032035400720069006E0061006D00690044
:1013A0006300200053007400650070007000650049
:1013B000720020004400650076006900630065004B
:1013C000200026035400720069006E0061006D0069
:1013D000690063004D006F00740069006F006E00CB
:1013E0002000430074006C00040309040902430058
:1013F000020100C0320904000001020201000524BC
:101400000010010524010001042402020524060045
:1014100001070582030800FF09040100020A000019
:10142000000705030240000007058102400000128A
:10143000011001020000403C2A0001012A010203C0
:1014400001010203040506524F5200000106524FEB
:101450004C000002064D5354000003024D5650004C
:1014600000040753415000000507474150000006A3
:101470000353544150000703525341500008035393
:1014800047500000090747475000000A03535447DC
:1014900050000B0352534750000C035246530000B8
:1014A0000D0353494F00000E0747494F00000F033B
:1014B00053414300001D0753434F00001E0747439D
:1014C0004F00001F0343434F0000200341434F00E0
:1014D00000270355463000004007554631000041C3
:1014E0000755463200004207554633000043075572
:1014F000463400004407554635000045075546363A
:10150000000046075546370000470752554E000079
:10151000810553544F5000800042494E00008B001B
:1015200000000000000000020000000000000100B8
:101530000000000102030401020304060708090277
:1015400004060836313130563134320041425300FE
:1015500052454C00434F4F524400535441525400A3
:1015600053544F500053544154555300430000000E
:101570000020202020202020202028282828282063
:10158000202020202020202020202020202020205B
:1015900020881010101010101010101010101010C3
:1015A00010040404040404040404041010101010B3
:1015B000101041414141414101010101010101017D
:1015C00001010101010101010101010110101010CF
:1015D000101042424242424202020202020202024F
:1015E00002020202020202020202020210101010A3
:1015F00020000000000000000000000000000000CB
:1016000000000000000000000000000000000000DA
:1016100000000000000000000000000000000000CA
:1016200000000000000000000000000000000000BA
:1016300000000000000000000000000000000000AA
:10164000000000000000000000000000000000009A
:10165000000000000000000000000000000000008A
:10166000000000000000000000000000000000007A
:041670000000000076
:1016740043150108000102000008000001000000F9
:101684000200000000000000000000000000000054
:101694000000000000000000000000000000000046
:1016A4000000000000000000000000000000000036
:1016B4000000000000C2010000000800F9970008C3
:1016C400B5950008B5940008C9940008CB940008A7
:1016D4002595000849950008919600089D960008F4
:1016E400A996000800000000400000002F14010823
:1016F40012000000EC13010843000000E813010885
:1017040004000000C2130108260000009013010821
:1017140032000000100100201A0000000100000047
:1017240099F700089194000899F7000899F70008C0
:1017340099F7000899F7000899F7000899F7000845
:10174400A99400080401000099F7000899F700081B
:101754008995000899F7000899F7000899F7000897
:1017640099F700088594000899F7000899F700088C
:1017740099F7000899F7000899F7000899F7000805
:101784001A0354004D004300530054004500500018
:101794000000000000000000000000000000000045
:1017A400000000001C04002084040020EC0400203D
:1017B4000000000000000000000000000000000025
:1017C4000000000000000000000000000000000015
:1017D400000000006C15010800000000000000007B
:1017E40000000000000000000000000000000000F5
:1017F40000000000000000000000000000000000E5
:1018040000000000000000000000000000000000D4
:1018140000000000000000000000000000000000C4
:1018240000000000000000000000000000000000B4
:1018340000000000000000000000000000000000A4
:101844000000000000000000010000000000000093
:101854000E33CDAB34126DE6ECDE05000B00000058
:101864000000000000000000000000000000000074
:101874000000000000000000000000000000000064
:101884000000000000000000000000000000000054
:101894000000000000000000000000000000000044
:101BC4000000000000000000300100207015010832
:04000005080041109E
:00000001FF
